:100000000C9458120C9489120C9489120C94891235
:100010000C9489120C9489120C9489120C948912F4
:100020000C9489120C9489120C9489120C948912E4
:100030000C9489120C9422720C9489120C948912DB
:100040000C9489120C94A1420C9489120C9489127C
:100050000C9489120C9489120C94647A0C94FEB25C
:100060000C9489120C948F410C9489120C9489126F
:100070000C9489120C9489120C9489120C94891294
:100080000C9489120C9489120C9489120C94891284
:100090000C9489120C9489120C9489120C94891274
:1000A0000C9489120C9489120C9489120C94891264
:1000B0000C9489120C9489120C9489120C94891254
:1000C0000C9489120C9489120C9489120C94891244
:1000D0000C9489120C9489120C942E420C94EF41CA
:1000E0000C948912102C2D2C5E2C7B2C902CB92C6E
:1000F000262D8C2D352E2E313C3135315C31603141
:100100007A313C358F31DB310D3234325D32B232EF
:10011000C332D432E532F63207333C3549343C350C
:100120005234C234C834E83417AF1AAF09AF0DAF38
:1001300013AF51AF1EAF22AF28AF2CAF30AF36AFE9
:100140003AAF3EAF51AF44AF48AF4CAF1AB21FB257
:1001500024B22EB238B2B1B242B24AB252B25CB29A
:1001600066B270B27FB289B2B1B293B29DB2A7B299
:10017000084AD73B3BCE016E84BCBFFDC12F3D6C0E
:1001800074319ABD56833DDA3D00C77F11BED9E474
:10019000BB4C3E916BAAAABE000000803F05A84C54
:1001A000CDB2D44EB93836A9020C50B99186880820
:1001B0003CA6AAAA2ABE000000803F004E414E493C
:1001C0004E495459494E46CDCCCC3D0AD7233C1715
:1001D000B7D13877CC2B329595E6241FB14F0A0062
:1001E0000020410000C84200401C4620BCBE4CCA52
:1001F0001B0E5AAEC59D74434F4D4D554E4943415C
:1002000054494F4E0044525952554E004552524F98
:10021000525300494E464F004543484F0047322F46
:1002200047332062616420706172616D657465722C
:10023000730A00206F6620004D424C20473239205F
:10024000706F696E74200059206F7574206F66207E
:1002500072616E67652028312D35292E0A005820DD
:100260006F7574206F662072616E67652028312D6E
:1002700035292E0A004D6573682070726F62696EB1
:100280006720646F6E652E0A005374617274206D6E
:100290006573682070726F62696E67207769746831
:1002A0002022473239205331222066697273742E1E
:1002B0000A004732380A47323920533200537461FA
:1002C00074653A20004D65736820626564206C6532
:1002D00076656C696E6720686173206E6F2064615B
:1002E00074612E0A0053206F7574206F662072614E
:1002F0006E67652028302D35292E0A004D657368FC
:1003000020706F696E742063616E6E6F7420626519
:10031000207265736F6C7665640A00456E642066B2
:10032000696C65206C6973740A00426567696E20A8
:1003300066696C65206C6973740A00286E6F2066AC
:10034000696C6529005344207072696E74696E6728
:10035000206279746520004E6F74205344207072BF
:10036000696E74696E670A0043757272656E7420F7
:1003700066696C653A200046696C652064656C6549
:100380007465643A0044656C6574696F6E206661DB
:10039000696C65642C2046696C653A200025697398
:1003A0000025696D20256973002569682025696D20
:1003B0002025697300256964202569682025696DF9
:1003C00020256973002569792025696420256968DD
:1003D0002025696D20256973005072696E74207440
:1003E000696D653A2000180213020C020502F7013C
:1003F0006F66660044454255473A004B494C4C45B0
:10040000442E20004D3131332053006F6B002C20DF
:10041000002C2000544845524D414C5F50524F54DF
:10042000454354494F4E004155544F5245504F5249
:10043000545F53445F53544154555300454D455206
:1004400047454E43595F5041525345520043415333
:10045000455F4C494748545F4252494748544E45CE
:10046000535300544F47474C455F4C4947485453FA
:1004700000534F4654574152455F504F5745520025
:100480004255494C445F50455243454E54004C45FB
:1004900056454C494E475F44415441005A5F5052C3
:1004A0004F4245004155544F4C4556454C00505223
:1004B000494E545F4A4F420050524F4752455353A2
:1004C000004155544F5245504F52545F54454D5082
:1004D00000564F4C554D45545249430045455052E6
:1004E0004F4D0053455249414C5F584F4E5F584F56
:1004F0004646004649524D574152455F4E414D4593
:100500003A4D61726C696E20312E312E39202847A8
:1005100069746875622920534F555243455F434FB4
:1005200044455F55524C3A68747470733A2F2F6784
:1005300069746875622E636F6D2F4D61726C696EA0
:100540004669726D776172652F4D61726C696E20BC
:1005500050524F544F434F4C5F56455253494F4EA4
:100560003A312E30204D414348494E455F54595051
:10057000453A3344205072696E7465722045585470
:1005800052554445525F434F554E543A31205555CC
:1005900049443A63656465326132662D34316132B3
:1005A0002D343734382D396231322D633535633689
:1005B000326633363766660A002F2F20002054003B
:1005C000205200416363656C65726174696F6E3AB5
:1005D0002050005741524E494E4721204C6F772002
:1005E0005A204A65726B206D6179206C65616420C8
:1005F000746F20756E77616E7465642070617573B9
:1006000065732E0A0020466C6F773A200000013691
:100610003726032BFFFFFF3C3D382AFFFFFFFF2E4D
:10062000303E12FFFFFFFFFFFFFF0809FF2C071AF4
:100630001C18FFFFFF08440A2C4324221E20643AA2
:100640000020693A0020703A00496E76616C696456
:100650002065787472756465720A0043290A006126
:10066000626C656420286D696E2074656D70200071
:10067000436F6C6420657874727564657320617271
:1006800065200020643A0020693A0020703A004E4C
:100690006F2063617365206C696768740A00454563
:1006A00050524F4D204F4B0A00205A004475616C48
:1006B00020456E6473746F702041646A7573746D45
:1006C000656E7420286D6D293A20003F4B207661BD
:1006D0006C7565206F7574206F662072616E67653A
:1006E0002028302D3130292E0A00416476616E6356
:1006F00065204B3D004163746976652045787472CE
:10070000756465723A2000496E76616C6964206593
:10071000787472756465720A0043616E6E6F74203E
:10072000656E746572207375626469723A20004D5B
:10073000353031005370656369616C204D656E75AD
:100740003A205265616420454550524F4D0A004D94
:10075000353030005370656369616C204D656E758E
:100760003A205361766520454550524F4D0A004767
:1007700032380A473239005370656369616C204D25
:10078000656E753A204175746F20426564204C6532
:1007900076656C696E670A004D333033204338202C
:1007A00053323030005370656369616C204D656E63
:1007B000753A204175746F2054756E652050494418
:1007C0000A003C5370656369616C5F4D656E753EF0
:1007D000003C5370656369616C5F4D656E753E00EA
:1007E0002F002F002F002F2E2E0A002F2E2E002F2D
:1007F0002E2E003C5370656369616C5F4D656E75AC
:100800003E0A003C5370656369616C204D656E75EE
:100810003E003C5370656369616C204D656E753EAA
:10082000003C5265616420454550524F4D3E003CAE
:100830005265616420454550524F4D3E003C536126
:10084000766520454550524F4D3E003C53617665DC
:1008500020454550524F4D3E003C4175746F20423B
:100860006564204C6576656C696E673E003C417539
:10087000746F20426564204C6576656C696E673ED6
:10088000003C4175746F2054756E6520486F746527
:100890006E64205049443E003C4175746F2054758D
:1008A0006E6520486F74656E64205049443E003C7C
:1008B000457869743E003C457869743E0056313194
:1008C00036004A333320004D3530300A4D34323053
:1008D0002053310A4731205A313020463234300A11
:1008E0004731205830205930204636303030004AC9
:1008F0003232004A3232004731205A3520463234F3
:10090000300A4731205831393020593230204636AC
:100910003030300A4731205A3020463234300047D8
:1009200031205A3520463234300A47312058313987
:100930003020593139302046363030300A473120A6
:100940005A302046323430004731205A3520463262
:1009500034300A473120583139302059323020465E
:10096000363030300A4731205A3020463234300099
:100970004739310A4731205A313020463234300A63
:100980004739300A4732380A4732390A4731205846
:100990003230205932302046363030300A4731204C
:1009A0005A302046323430004A3032004A31320068
:1009B0004731205A3130004F4B004731205A3130F7
:1009C0000047393000473120452569463530300031
:1009D000473120452D302E314625690047312045CD
:1009E000302E31462569004731205A256946256950
:1009F000004731205A2D302E3146256900473120DD
:100A00005A302E314625690047312059256946253F
:100A10006900473120592D302E3146256900473174
:100A20002059302E31462569004731205825694626
:100A3000256900473120582D302E31462569004761
:100A4000312058302E314625690047393100473270
:100A50003800473238205A00473238205900473290
:100A6000382058004132305620004731205A31306A
:100A7000004A3034004A3231004A3230004B494C8F
:100A80004C45442E20004A303400454E4400464E2A
:100A900020004A3032003939393A393939004D00AD
:100AA00048004137562000413656202D2D2D004A52
:100AB00030320041365620005A3A2000593A200080
:100AC000583A2000413556004134562000413356F3
:100AD000200041325620004131562000413056203E
:100AE000004D3834004A3136004A31380047393138
:100AF0000A4731205A313020463234300A473930E3
:100B0000004A3134004A3030004A3031004A313036
:100B100000656E7175657565696E672022004B49C9
:100B20004C4C45442E20005072696E7465722073DF
:100B3000746F707065642064756520746F206572D1
:100B4000726F72732E204669782074686520657212
:100B5000726F7220616E6420757365204D3939396A
:100B600020746F20726573746172742E202854652E
:100B70006D7065726174757265206973207265733A
:100B800065742E20536574206974206166746572E3
:100B90002072657374617274696E67290A004E6F02
:100BA00020436865636B73756D2077697468206C8A
:100BB000696E65206E756D6265722C204C61737470
:100BC000204C696E653A20004E6F20436865636B68
:100BD00073756D2077697468206C696E65206E7519
:100BE0006D6265722C204C617374204C696E653A9D
:100BF0002000636865636B73756D206D69736D614B
:100C00007463682C204C617374204C696E653A20C3
:100C1000004C696E65204E756D62657220697320A7
:100C20006E6F74204C617374204C696E65204E7534
:100C30006D6265722B312C204C617374204C696E8F
:100C4000653A20004D313130004D3331005344209E
:100C500072656164206572726F720A00446F6E651E
:100C6000207072696E74696E672066696C650A002F
:100C700024F4D43050C38E20C2A24017828B70114E
:100C8000127A910D816CD90AA861E108C7586607EC
:100C9000615143061E4B5D05C145A7041A4111046D
:100CA000093D9803713931034036DB026533910207
:100CB000D4305402802E1D02632CEE01752AC5012A
:100CC000B028A001102781018F2564012B244B013E
:100CD000E0223401AC211F018D200D01801FFC009A
:100CE000841EED00971DDF00B81CD200E61BC60075
:100CF000201BBC00641AB200B219A8000A19A00097
:100D00006A189900D117910040178B00B51684001E
:100D100031167E00B31579003A157300C7146F00C1
:100D200058146A00EE1366008813630025135E00F2
:100D3000C7125B006C12570015125400C11151000C
:100D400070114F0021114B00D61049008D10470043
:100D50004610440002104200C00F4000800F3E00C9
:100D6000420F3C00060F3B00CB0E3800930E3700BD
:100D70005C0E3500270E3400F30D3200C10D31003A
:100D8000900D3000600D2E00320D2D00050D2C0051
:100D9000D90C2B00AE0C2900850C29005C0C270017
:100DA000350C27000E0C2600E80B2400C40B240091
:100DB000A00B23007D0B23005A0B2100390B2100CF
:100DC000180B2000F80A1F00D90A1E00BB0A1E00DB
:100DD0009D0A1D00800A1D00630A1C00470A1B00B3
:100DE0002C0A1B00110A1A00F7091A00DD09190064
:100DF000C4091900AB091900920917007B091800F2
:100E0000630917004C091600360916002009160060
:100E10000A091500F5081500E0081400CC081400B4
:100E2000B8081400A4081400900813007D081200EC
:100E30006B0813005808120046081200340811000D
:100E4000230811001208110001081100F00710001A
:100E5000E0071000D0071000C0071000B0070F0017
:100E6000A107100091070E0083070F0074070F0001
:100E700065070E0057070E0049070E003B070D00DF
:100E80002E070E0020070D0013070D0006070D00AA
:100E9000F9060C00ED060D00E0060C00D4060C006F
:100EA000C8060C00BC060C00B0060C00A4060B0023
:100EB00099060C008D060B0082060B0077060B00CE
:100EC0006C060B0061060A0057060B004C060A0070
:100ED00042060A0038060A002E060A0024060A0006
:100EE0001A060A001006090007060A00FD05090097
:100EF000F4050900EB050900E2050900D905090020
:100F0000D0050900C7050900BE050900B5050800A0
:100F1000AD050800A50509009C050800940508001A
:100F20008C050800840508007C050800740508008D
:100F30006C050700650508005D05070056050800FB
:100F40004E05070047050700400508003805070063
:100F5000310507002A050700230507001C050600C8
:100F6000160507000F050700080506000205070023
:100F7000FB040600F5040700EE040600E804060082
:100F8000E2040700DB040600D5040600CF040600D7
:100F9000C9040600C3040600BD040600B704060029
:100FA000B1040500AC040600A6040600A004050078
:100FB0009B04060095040500900406008A040500C1
:100FC00085040500800406007A0405007504050008
:100FD000700405006B04050066040500610405004B
:100FE0005C04050057040500520405004D0405008B
:100FF00048040500430405003E0404003A040500CB
:1010000035040500300404002C0405002704040006
:10101000230405001E0404001A040400160405003D
:10102000110404000D040400090405000404040074
:1010300000040400FC030400F8030400F4030400AB
:10104000F0030400EC030400E8030400E4030400DC
:10105000E0030400DC030400D8030400D40304000C
:10106000D0030400CC030400C8030300C50303003D
:1010700024F404D9201BC40C5C0E9804C4095F023C
:1010800065077101F405F900FB04B300480487000B
:10109000C10369005803550003034500BE023A002E
:1010A0008402310053022A00290225000402200094
:1010B000E4011C00C8011900AF01170098011400D9
:1010C00084011300710110006101100051010E0034
:1010D00043010D0036010B002B010B0020010B001A
:1010E000150109000C01090003010800FB000800BC
:1010F000F3000800EB000700E4000600DE00060035
:10110000D8000600D2000600CC000500C70005008C
:10111000C2000500BD000400B9000400B5000400D1
:10112000B1000400AD000400A9000400A500030004
:10113000A20003009F0004009B000300980003002E
:101140009500020093000300900003008D00020050
:101150008B00030088000200860002008400030068
:10116000810002007F0002007D0002007B0002007F
:10117000790002007700010076000200740002008E
:1011800072000100710002006F0002006D0001009A
:101190006C0002006A0001006900020067000100A3
:1011A00066000100650001006400020062000100A9
:1011B00061000100600001005F0002005D000100AD
:1011C0005C0001005B0001005A00010059000100B1
:1011D00058000100570001005600010055000100B1
:1011E00054000100530000005300010052000100B0
:1011F00051000100500001004F0001004E000000AE
:101200004E0001004D0001004C0001004B000000A9
:101210004B0001004A0001004900010048000000A5
:1012200048000100470001004600000046000100A0
:10123000450000004500010044000100430000009B
:101240004300010042000000420001004100000094
:1012500041000100400001003F0000003F0001008C
:101260003E0000003E0001003D0000003D00010086
:101270003C0000003C0000003C0001003B0000007E
:101280003B0001003A0000003A0001003900000074
:10129000390001003800000038000000380001006B
:1012A0003700000037000100360000003600000063
:1012B0003600010035000000350000003500010057
:1012C000340000003400000034000100330000004E
:1012D0003300000033000100320000003200000043
:1012E0003200010031000000310000003100010037
:1012F0003000000030000000300001002F0000002E
:101300002F0000002F0000002F0001002E00000021
:101310002E0000002E0001002D0000002D00000016
:101320002D0000002D0001002C0000002C0000000A
:101330002C0000002C0001002B0000002B000000FE
:101340002B0000002B0001002A0000002A000000F2
:101350002A0000002A0001002900000029000000E6
:1013600029000000290000002900010028000000D9
:1013700028000000280000002800000028000100CC
:1013800027000000270000002700000027000000C1
:1013900027000100260000002600000026000000B3
:1013A00026000000260001002500000025000000A6
:1013B0002500000025000000250000002500010098
:1013C000240000002400000024000000240000008D
:1013D000240001002300000023000000230000007F
:1013E0002300000023000000230000002300010070
:1013F0002200000022000000220000002200000065
:101400002200000022000100210000002100000055
:101410002100000021000000210000002100000048
:10142000210001002000000020000000200000003A
:10143000200000002000000020000000200000002C
:10144000200001001F0000001F0000001F0000001E
:101450001F0000001F0000001F0000001F0001000F
:101460001E0000001E0000001E0000001E00000004
:10147000C23100001C260000F4190000D80F000043
:10148000EB080000C00400007502000040010000ED
:10149000526573656E643A20006F6B0020746F6F45
:1014A000206C6F6E6720657874727573696F6E203B
:1014B00070726576656E7465640A0020636F6C6493
:1014C00020657874727573696F6E207072657665C9
:1014D0006E7465640A00627573793A207061757381
:1014E000656420666F7220696E7075740A0062759B
:1014F00073793A2070617573656420666F72207528
:101500007365720A00627573793A2070726F636551
:101510007373696E670A004A3135004B494C4C457C
:10152000442E20004B494C4C206361757365642048
:101530006279204B494C4C20627574746F6E2F7029
:10154000696E0A004B494C4C45442E20004B494CD7
:101550004C2063617573656420627920746F6F201D
:101560006D75636820696E6163746976652074695E
:101570006D65202D2063757272656E7420636F6DCA
:101580006D616E643A20004A3131005072696E74A8
:1015900065722068616C7465642E206B696C6C28C0
:1015A000292063616C6C6564210A000000A0C00002
:1015B000000000000000005761726E696E673A20FB
:1015C000486F6D696E672042756D70204469766959
:1015D000736F72203C20310A000202040000A04018
:1015E0000000A040000000400000574300005243AC
:1015F00000004D43FFFFFF20746F6F206C6F6E671C
:1016000020657874727573696F6E20707265766587
:101610006E7465640A0020636F6C64206578747270
:101620007573696F6E2070726576656E7465640A95
:1016300000454550524F4D206461746173697A656D
:10164000206572726F722E0A00290A002062797476
:1016500065733B20637263200053657474696E6721
:10166000732053746F726564202800290A00206279
:10167000797465733B2063726320002073746F720A
:1016800065642073657474696E6773207265747223
:101690006965766564202800202863616C63756C39
:1016A0006174656429210A0020213D2000454550D0
:1016B000524F4D20435243206D69736D61746368CE
:1016C000202D202873746F726564292000205369CF
:1016D0007A653A2000496E6465783A2000204D61B1
:1016E000726C696E3D563535290A002845455052C1
:1016F0004F4D3D00454550524F4D20766572736900
:101700006F6E206D69736D617463682000024A31E9
:1017100035004A3132004A3137002020506C616E6A
:101720006E657242756666657242797465733A20B9
:10173000002046726565204D656D6F72793A200014
:10174000436F6D70696C65643A204E6F7620313658
:1017500020323031380A00207C20417574686F7265
:101760003A2028646176696472616D69726F2C2019
:10177000666F7220416E79637562696320693320F8
:101780004D656761290A00323031392D31312D31F3
:101790003500204C61737420557064617465643A3F
:1017A0002000312E312E390A004D61726C696E00B5
:1017B00020536F6674776172652052657365740A91
:1017C00000205761746368646F67205265736574A5
:1017D0000A002042726F776E206F75742052657315
:1017E00065740A002045787465726E616C205265DC
:1017F0007365740A00506F77657255700A007374D0
:101800006172740A004D3234004D3233202573006A
:101810006175746F25692E67006572726F7220772B
:10182000726974696E6720746F2066696C650A005E
:10183000205A3A0020593A0020583A00656E6473E5
:10184000746F7073206869743A2000446F6E65206D
:10185000736176696E672066696C652E0A004D3289
:1018600039006F70656E206661696C65642C204676
:10187000696C653A200043616E6E6F74206F70650D
:101880006E2073756264697220004A3035004A32F6
:1018900033004739310A4731205A2D313020463242
:1018A00034300A4739300053442063617264206F3A
:1018B0006B0A006F70656E526F6F74206661696CA1
:1018C00065640A00766F6C756D652E696E697420AB
:1018D0006661696C65640A004572726F723A005302
:1018E0004420696E6974206661696C0A00656368EA
:1018F0006F3A001000C90210012C01400122017052
:10190000011801B0010E01F00104015002FA00B00B
:1019100002F0003003E600D003DC009004D2007037
:1019200005C800A006BE000008B400B009AA00D097
:101930000BA000600E960060118C00001582002044
:10194000197800C01D6E00A0226400B0275A0090D4
:101950002C500000314600E0343C0010383200903A
:101960003A2800603C1E00A03D1400803E0A002082
:101970003F00002CFFFFFFFFFF000101010101629A
:1019800065640A002C2073797374656D2073746F1D
:101990007070656421204865617465725F49443ADE
:1019A00020004265642068656174696E6720666125
:1019B000696C65640048656174696E672066616979
:1019C0006C65640045312048656174696E67206606
:1019D00061696C65640048656174696E6720666161
:1019E000696C65640070012C0190012701B001222F
:1019F00001C0011D01F00118011002130130020E97
:101A0000016002090190020401C002FF000003FA14
:101A1000004003F5008003F000D003EB002004E653
:101A2000007004E100E004DC004005D700C005D2EE
:101A3000004006CD00D006C8008007C3003008BEB5
:101A400000F008B900C009B400B00AAF00B00BAA9A
:101A500000D00CA500000EA000500F9B00C01096F7
:101A6000005012910000148C00C0158700B017823E
:101A700000B0197D00D01B7800001E730040206E5E
:101A80000090226900F024640040275F0090295AEA
:101A900000E02B5500102E500020304B0010324635
:101AA00000E033410090353C001037370070383289
:101AB00000A0392D00B03A2800A03B2300603C1E56
:101AC00000103D1900903D1400103E0F00703E0ABA
:101AD00000C03E0500003F0000403FFBFF803FF696
:101AE000FFC03FF1FF453120544845524D414C2045
:101AF00052554E41574159004245442054484552A1
:101B00004D414C2052554E41574159005468657221
:101B10006D616C2052756E617761790045312045A9
:101B200072723A204D415854454D50004572723AF8
:101B3000204D415854454D5020424544004D415898
:101B400054454D502074726967676572656400453D
:101B500031204572723A204D494E54454D50004552
:101B600072723A204D494E54454D50204245440032
:101B70004D494E54454D50207472696767657265D2
:101B800064004D383420582059205A204500202F19
:101B9000002042403A0020403A003A004361703A47
:101BA00000205A00205900580020204D61783A202A
:101BB00000205A00205900580020204D696E3A201C
:101BC000004F6E20004F666600536F667420656E8E
:101BD0006473746F70733A20004B64200023646553
:101BE00066696E652044454641554C545F004B691B
:101BF000200023646566696E652044454641554C66
:101C0000545F004B70200023646566696E65204454
:101C1000454641554C545F00504944204175746F0E
:101C200074756E652066696E6973686564212050FD
:101C3000757420746865206C617374204B702C205F
:101C40004B6920616E64204B6420636F6E73746116
:101C50006E74732066726F6D2062656C6F77206999
:101C60006E746F20436F6E66696775726174696F19
:101C70006E2E680A00504944204175746F74756E69
:101C800065206661696C6564212074696D656F7596
:101C9000740A00453120544845524D414C2052555C
:101CA0004E415741590042454420544845524D4108
:101CB0004C2052554E4157415900546865726D6130
:101CC0006C2052756E6177617900453120486561FD
:101CD00074696E67206661696C65640042656420A2
:101CE00068656174696E67206661696C6564004847
:101CF000656174696E67206661696C65640050494E
:101D000044204175746F74756E65206661696C65F9
:101D100064212054656D70657261747572652074FC
:101D20006F6F20686967680A00204B643A200020C2
:101D30004B693A2000204B703A20000A20436C6126
:101D40007373696320504944200A002054753A2077
:101D500000204B753A2000206D61783A2000206DFC
:101D6000696E3A200020643A200020626961733A6B
:101D70002000504944204175746F74756E6520666B
:101D800061696C65642120426164206578747275B4
:101D9000646572206E756D6265720A005049442058
:101DA0004175746F74756E652073746172740A0086
:101DB0004F66660A00466164652048656967687415
:101DC0002000426564204C6576656C696E67200072
:101DD0004661696C656420746F20656E61626C6534
:101DE00020426564204C6576656C696E670A004D1B
:101DF00065736820426564204C6576656C2064617B
:101E000074613A0A004D65736820706F696E7420C2
:101E100063616E6E6F74206265207265736F6C769D
:101E200065640A004D34323120696E636F727265E9
:101E3000637420706172616D657465722075736181
:101E400067650A002066697273740A005A005900B7
:101E50005800486F6D652000546F6F2066617220D6
:101E600066726F6D207265666572656E636520705F
:101E70006F696E740A007C3C3E5E2B3D3F2F5B5DBC
:101E80003B2C2A225C0020496E76616C69642065D7
:101E90007874727564657220000000A0C0000000B4
:101EA0000000000000000052430000524300004DBB
:101EB00043486F6D696E67206661696C65640020D8
:101EC0006E6F7420656E74657265642E0A005072C0
:101ED0006F7465637465642050696E0A004A303619
:101EE000004A3034004A30370020573A004A303830
:101EF000004A30390020573A00205A3A0020593A17
:101F00000020436F756E7420583A0020453A002037
:101F10005A3A0020593A00583A0048617264636F97
:101F20006465642044656661756C742053657474DF
:101F3000696E6773204C6F616465640A00B80B00BA
:101F400000B80B00003C000000102700000000FA61
:101F5000430000FA430000C040000070420000A0AF
:101F6000420000A0420000C8433333B94220286D2C
:101F70006D290020204D393030204B004C696E65B2
:101F8000617220416476616E63653A0A0020440004
:101F900020490020204D33303420500020440020C0
:101FA000490020204D3330312050005049442073E7
:101FB000657474696E67733A0A00205A0020204DD8
:101FC00036363600456E6473746F702061646A75CE
:101FD00073746D656E743A0A00205A00205900200F
:101FE00020473239205333205800205A0020204DFA
:101FF0003432302053004D65736820426564204CB4
:102000006576656C696E673A0A00205A00205900AF
:1020100020204D323036205800486F6D65206F66A5
:10202000667365743A0A00204500205A0020590062
:1020300020580020540020530020204D32303520FD
:10204000510020453C6D61785F655F6A65726B3E4B
:102050000020583C6D61785F785F6A65726B3E2046
:10206000593C6D61785F795F6A65726B3E205A3CBE
:102070006D61785F7A5F6A65726B3E00416476617C
:102080006E6365643A20513C6D696E5F7365676D80
:10209000656E745F74696D655F75733E20533C6D4A
:1020A000696E5F66656564726174653E20543C6D5F
:1020B000696E5F74726176656C5F66656564726196
:1020C00074653E0020540020520020204D323034F0
:1020D000205000416363656C65726174696F6E20A6
:1020E00028756E6974732F7332293A20503C7072D0
:1020F000696E745F616363656C3E20523C72657407
:10210000726163745F616363656C3E20543C7472FA
:102110006176656C5F616363656C3E0A0020450013
:10212000205A0020590020204D3230312058004DD7
:102130006178696D756D20416363656C657261746A
:10214000696F6E2028756E6974732F7332293A0A8D
:1021500000204500205A0020590020204D32303305
:102160002058004D6178696D756D206665656472F3
:10217000617465732028756E6974732F73293A0A28
:1021800000204500205A0020590020204D393220DF
:10219000580053746570732070657220756E697491
:1021A0003A0A0020204D3230302044300A002020EE
:1021B0004D3230302044002044697361626C6564A4
:1021C0000A0046696C616D656E742073657474698C
:1021D0006E67733A002020473231202020203B00D8
:1021E000545249474745524544006F70656E003A66
:1021F00020007A325F6D696E007A5F6D696E0079DA
:102200005F6D696E00785F6D696E005265706F7208
:1022100074696E6720656E6473746F702073746187
:102220007475730A000A4D65617375726564207078
:102230006F696E74733A0A005A206F66667365742C
:102240003A20004E756D20582C593A20352C350A0D
:10225000004572726F722077726974696E672074BC
:102260006F20454550524F4D210A000000210024A7
:102270000027002A002D0030003300010100000477
:102280000107010A0100002200250028002B002E72
:10229000003100340002010000050108010B0100BB
:1022A0000020002300260029002C002F003200000F
:1022B00001000003010601090105050505070508E0
:1022C000080808020202020A0A08080404040401B9
:1022D00001010101010101030303030303030304DB
:1022E0000707070C0C0C0C0C0C0C0C02020202066B
:1022F000060606060606060B0B0B0B0B0B0B0B015B
:102300000210202008081020401020408002010206
:1023100001080402010102040810204080804020CE
:102320001008040201800402018040201008040209
:102330000108040201010204081020408001020487
:10234000081020408000000A0B02090C0D0E08073F
:102350000304010000000000000000000000000075
:10236000000000000000000000000000000000006D
:10237000001211100000000000000000000000002A
:102380000000000000000000000000556E6B6E6F42
:10239000776E20636F6D6D616E643A2022000000DD
:1023A0004842000048420000804000000000577290
:1023B0006974696E6720746F2066696C653A2000E5
:1023C0006F70656E206661696C65642C2046696C6F
:1023D000653A20006F70656E206661696C65642CDB
:1023E0002046696C653A200046696C652073656C0F
:1023F00065637465640A002053697A653A20004673
:10240000696C65206F70656E65643A2000206669AE
:102410006C653A2000646F696E6700667265736868
:10242000004E6F772000454E4420535542524F5581
:1024300054494E450A002220706F730022207061BB
:1024400072656E743A2200535542524F5554494EAC
:10245000452043414C4C207461726765743A2200F8
:102460004B494C4C45442E2000747279696E6720AC
:10247000746F2063616C6C207375622D67636F6489
:10248000652066696C6573207769746820746F6F66
:10249000206D616E79206C6576656C732E204D41E0
:1024A00058206C6576656C2069733A0084BFC4B9A6
:1024B00011241FBECFEFD1E2DEBFCDBF00E00CBFC5
:1024C00013E0A0E0B2E0ECE9FAE901E00BBF02C0E2
:1024D00007900D92A03AB107D9F726E1A0EAB3E040
:1024E00001C01D92AF3BB207E1F712E1C7E5D2E1AF
:1024F00000E006C021970109802FFE010E94A6CCB2
:10250000C635D10780E00807A9F70E94E5B90C9409
:102510003DCD0C9400002F923F924F925F926F92AC
:102520007F928F929F92AF92BF92CF92DF92EF9263
:10253000FF920F931F93CF93DF93CDB7DEB7CB56A8
:10254000D1090FB6F894DEBF0FBECDBF91E09093D6
:10255000BF0A809174168D3411F40C944F1C84358D
:1025600011F40C943629873411F00C9482292090B0
:102570007216309073162CE12216310409F43EC60F
:10258000A4F444E0241631044CF452E0251631043E
:102590000CF046C037FE3DC00C944B1C64E0261680
:1025A000310409F4ECC50C944B1C7AE52716310470
:1025B00011F40C94841B6CF49DE12916310409F488
:1025C00022C6AAE22A16310411F40C94F91A0C94CA
:1025D0004B1CBBE52B16310411F40C94881BECE565
:1025E0002E16310411F00C944B1C9FE4292E92E01E
:1025F000392E2DECE22E2AE0F22E6DEB73E079AF4E
:1026000068AF30EAC32E33E0D32E00E010E00C9424
:10261000C71B8091410281110C9489290C94842953
:1026200080914102882311F40C9484290E94EA9736
:1026300082E50E94613D882309F450C10E94E13C7B
:102640004B015C0120E030E0A9010E9464C58823B1
:1026500009F474C12091BD033091BE034091BF03C2
:102660005091C00328AF39AF4AAF5BAF4091C1036F
:102670005091C2036091C3037091C4034CAF5DAF2E
:102680006EAF7FAF6091DA0A7091DB0A8091DC0A4D
:102690009091DD0A2C966CAF7DAF8EAF9FAF2C97DB
:1026A0008091DE0A9091DF0AA091E00AB091E10AE0
:1026B00028968CAF9DAFAEAFBFAF28972C962CADB0
:1026C0003DAD4EAD5FAD2C9768AD79AD8AAD9BAD9C
:1026D0000E9464C581110FC028962CAD3DAD4EAD52
:1026E0005FAD28976CAD7DAD8EAD9FAD0E9464C58A
:1026F000882309F423C111E092E02916310409F07E
:1027000010E020E030E0A901C501B4010E9464C5D9
:10271000881F8827881F181759F020E030E040E80C
:102720005FEB64962CAF3DAF4EAF5FAF64970AC0CE
:1027300040E050E060E87FE364964CAF5DAF6EAF81
:102740007FAF649728AD39AD4AAD5BAD2C966CADCB
:102750007DAD8EAD9FAD2C970E948DC960966CAFFC
:102760007DAF8EAF9FAF60972CAD3DAD4EAD5FADF1
:1027700028966CAD7DAD8EAD9FAD28970E948DC91A
:102780006B017C0160962CAD3DAD4EAD5FAD6097A9
:10279000CA01B9010E94C9C52B013C01A7019601DC
:1027A000C701B6010E94C9C59B01AC01C301B201BA
:1027B0000E948EC90E94F9CB24966CAF7DAF8EAF7C
:1027C0009FAF249720E030E040E05FE30E94C9C55E
:1027D0002B013C01A5019401C501B4010E94C9C5AA
:1027E0004B015C01A3019201C301B2010E94C9C562
:1027F0009B01AC01C501B4010E948DC90E94F9CBB7
:1028000064962CAD3DAD4EAD5FAD64970E94C9C5D9
:102810004B015C01C701B601905824962CAD3DAD2B
:102820004EAD5FAD24970E946ACAA50194010E9433
:10283000C9C56B017C012C962CAD3DAD4EAD5FAD95
:102840002C9768AD79AD8AAD9BAD0E948EC920E012
:1028500030E040E05FE30E94C9C59B01AC01C701C5
:10286000B6010E948EC928AD39AD4AAD5BAD0E945C
:102870008DC96B017C0128962CAD3DAD4EAD5FAD91
:1028800028976CAD7DAD8EAD9FAD0E948EC920E0C6
:1028900030E040E05FE30E94C9C52B013C01249673
:1028A0002CAD3DAD4EAD5FAD249760966CAD7DAD6A
:1028B0008EAD9FAD60970E946ACAA50194010E94E7
:1028C000C9C59B01AC01C301B2010E948EC92CADE8
:1028D0003DAD4EAD5FAD0E948DC914C089E40E942C
:1028E000613D882329F00E94E13C6B017C0103C01B
:1028F000C12CD12C76018AE40E94613D882309F124
:102900000E94E13C2C966CAF7DAF8EAF9FAF2C97B1
:1029100020E030E0A901C701B6010E9464C5811121
:102920001FC020E030E0A9012C966CAD7DAD8EADCE
:102930009FAD2C970E9464C5811112C0E8EDF8E1AB
:102940000AC420E030E0A901C701B6010E9464C5B5
:102950008823A1F32C961CAE1DAE1EAE1FAE2C9785
:10296000C701B601905868AF79AF8AAF9BAF2C967C
:102970008CAD9DADAEADBFAD2C97B0588CAF9DAFBB
:10298000AEAFBFAF28AD39AD4AAD5BADCA01B9013D
:102990000E94C9C54B015C012CAD3DAD4EAD5FAD94
:1029A000CA01B9010E94C9C59B01AC01C501B401AE
:1029B0000E948EC90E94F9CBA0966CAF7DAF8EAFFE
:1029C0009FAFA0972091BD033091BE034091BF03FC
:1029D0005091C00328962CAF3DAF4EAF5FAF289704
:1029E000A701960128966CAD7DAD8EAD9FAD289761
:1029F0000E948EC964966CAF7DAF8EAF9FAF649717
:102A00004091C1035091C2036091C3037091C4030C
:102A100060964CAF5DAF6EAF7FAF60972C962CADDC
:102A20003DAD4EAD5FAD2C9760966CAD7DAD8EAD7E
:102A30009FAD60970E948EC9A4966CAF7DAF8EAF9C
:102A40009FAFA4976091DA0A7091DB0A8091DC0A4B
:102A50009091DD0A68966CAF7DAF8EAF9FAF68979F
:102A600064962CAD3DAD4EAD5FAD64970E948DC9AF
:102A70006B017C018091DE0A9091DF0AA091E00A4F
:102A8000B091E10A6C968CAF9DAFAEAFBFAF6C97C3
:102A9000A4962CAD3DAD4EAD5FADA497BC01CD016C
:102AA0000E948DC94B015C012091C5033091C60382
:102AB0004091C7035091C803A8962CAF3DAF4EAFCD
:102AC0005FAFA8976091E20A7091E30A8091E40AEF
:102AD0009091E50A0E948DC924966CAF7DAF8EAFB0
:102AE0009FAF2497A701960168AD79AD8AAD9BADE4
:102AF0000E94C9C52B013C01A50194016CAD7DADBF
:102B00008EAD9FAD0E94C9C59B01AC01C301B2014E
:102B10000E948EC92B013C01A501940168AD79ADDD
:102B20008AAD9BAD0E94C9C54B015C01A70196010E
:102B30006CAD7DAD8EAD9FAD0E94C9C59B01AC0152
:102B4000C501B4010E948DC9A30192010E9401CA6E
:102B50006B017C0120E030E0A9010E9464C587FF81
:102B60000AC02BED3FE049EC50E4C701B6010E94DA
:102B70008EC96B017C0132E02316310451F42BED38
:102B80003FE049EC50E4C701B6010E948DC96B01DA
:102B90007C0120E030E0A901C701B6010E9464C5B4
:102BA000811128C068962CAD3DAD4EAD5FAD6897E4
:102BB00028966CAD7DAD8EAD9FAD28970E9464C503
:102BC000811118C06C962CAD3DAD4EAD5FAD6C97CC
:102BD00060966CAD7DAD8EAD9FAD60970E9464C573
:102BE000811108C01BEDC12E1FE0D12E19ECE12E82
:102BF00010E4F12EA7019601A0966CAD7DAD8EADCF
:102C00009FADA0970E94C9C54B015C0120E030E058
:102C1000A90124966CAD7DAD8EAD9FAD24970E9429
:102C200064C58823E9F0A5019401C501B4010E949F
:102C3000C9C54B015C0124962CAD3DAD4EAD5FADD9
:102C40002497CA01B9010E94C9C59B01AC01C50105
:102C5000B4010E948EC90E94F9CB4B015C010DC0EA
:102C600020E030E0A901C501B4010E94B4CB87FF88
:102C700004C0B7FAB094B7F8B0942FE632E143E855
:102C80005AE3C501B4010E9464C587FF02C00C94D9
:102C90008429C501B4010E9403CB0E94D7CA2E9695
:102CA0007FAF6EAF2E97672B31F441E050E02E9648
:102CB0005FAF4EAF2E974090C9035090CA0360900B
:102CC000CB037090CC032E96AEADBFAD2E97BD0159
:102CD00080E090E00E9468C54B015C019B01AC0163
:102CE000C701B6010E946ACA28966CAF7DAF8EAF4D
:102CF0009FAF2897A501940124966CAD7DAD8EAD54
:102D00009FAD24970E946ACAA0966CAF7DAF8EAF2C
:102D10009FAFA097A30192016091E60A7091E70A24
:102D20008091E80A9091E90A0E948DC9A501940159
:102D30000E946ACAAC966CAF7DAF8EAF9FAFAC9766
:102D400028962CAD3DAD4EAD5FAD2897CA01B901B7
:102D50000E94C9C520E030E040E05FE30E94C9C5A1
:102D60009B01AC0160E070E080E89FE30E948DC9A8
:102D700068966CAF7DAF8EAF9FAF6897A8962CAD6D
:102D80003DAD4EAD5FADA89729873A874B875C87ED
:102D90004D865E866F86788A60910202709103028A
:102DA000072E000C880B990B0E946AC520914B02DC
:102DB00030914C0240914D0250914E020E94C9C583
:102DC0002AE037ED43E25CE30E94C9C56CAB7DAB02
:102DD0008EAB9FAB0E94F2B29B01AC0128533F4FD8
:102DE0004F4F5F4F6C962CAF3DAF4EAF5FAF6C97C0
:102DF00048AC59AC6AAC7BAC22242394312C39E129
:102E000021963FAF21972E964EAD5FAD2E9742157E
:102E1000530509F44DC10E949F7F0E94F2B2DC016C
:102E2000CB016C962CAD3DAD4EAD5FAD6C97821B6A
:102E3000930BA40BB50BB7FD10C00E94F2B29B011F
:102E4000AC0128533F4F4F4F5F4F6C962CAF3DAFB7
:102E50004EAF5FAF6C970E94BE4E21963FAD21975B
:102E6000315021963FAF2197332309F445C02CAD53
:102E70003DAD4EAD5FAD68966CAD7DAD8EAD9FAD99
:102E800068970E94C9C56B017C019201A301289635
:102E90006CAD7DAD8EAD9FAD28970E94C9C5A701D1
:102EA00096010E948EC97B018C019201A301689654
:102EB0006CAD7DAD8EAD9FAD68970E94C9C54B01CD
:102EC0005C012CAD3DAD4EAD5FAD28966CAD7DADDA
:102ED0008EAD9FAD28970E94C9C59B01AC01C5016D
:102EE000B4010E948DC92B013C01C701D8018CAFF0
:102EF0009DAFAEAFBFAF55C0B10180E090E00E9482
:102F000068C528962CAD3DAD4EAD5FAD28970E94AB
:102F1000C9C54B015C010E9467CA6B017C01C501F8
:102F2000B4010E94EFCB4B015C01A701960168AD93
:102F300079AD8AAD9BAD0E94C9C52B013C012C9691
:102F40002CAD3DAD4EAD5FAD2C97C501B4010E94D7
:102F5000C9C5A30192010E948EC92B013C01A501A4
:102F6000940168AD79AD8AAD9BAD0E94C9C54B0196
:102F70005C012C962CAD3DAD4EAD5FAD2C97C701DD
:102F8000B6010E94C9C59B01AC01C501B4010E94F4
:102F90008DC96CAF7DAF8EAF9FAF49E121964FAF2A
:102FA00021979201A30164966CAD7DAD8EAD9FAD6E
:102FB00064970E948EC969837A838B839C832CAD2E
:102FC0003DAD4EAD5FADA4966CAD7DAD8EAD9FAD0C
:102FD000A4970E948EC96D837E838F839887A09665
:102FE0002CAD3DAD4EAD5FADA09769857A858B85E3
:102FF0009C850E948EC969877A878B879C87AC964F
:103000002CAD3DAD4EAD5FADAC976D857E858F85AA
:1030100098890E948EC96D877E878F87988B809153
:103020002102882321F0CE0101960E94894CE09074
:10303000BE0A1CA61DA61EA61FA689819A81AB8169
:10304000BC8188A399A3AAA3BBA38D819E81AF81D4
:10305000B8858CA39DA3AEA3BFA389859A85AB85B4
:10306000BC8588A799A7AAA7BBA7AE01485D5F4FFB
:10307000BE016C5D7F4FCE0180960E94C4A7BE0149
:10308000645D7F4F6B018E010C5C1F4F9E01235FBF
:103090003F4FAE01485D5F4F68507109CE01809689
:1030A0000E94BA56882321F07FEF271A370AABCE49
:1030B000E090BE0A18AA19AA1AAA1BAA8091DA0AD5
:1030C0009091DB0AA091DC0AB091DD0A88A399A354
:1030D000AAA3BBA38091DE0A9091DF0AA091E00A27
:1030E000B091E10A8CA39DA3AEA3BFA38091E20A95
:1030F0009091E30AA091E40AB091E50A88A799A704
:10310000AAA7BBA7AE01485D5F4FBE016C5D7F4FB4
:10311000CE0180960E94C4A7CE01C0966C018E019C
:103120000C5C1F4F26EE3AE0AE01485D5F4FBE01DA
:103130006C5D7F4F40970E94BA5680E1EAEDFAE05D
:10314000ADEBB3E001900D928A95E1F70C948429E0
:103150000E947D3DF80184918F010F5F1F4F811107
:10316000F7CFEDE1F2E084918F010F5F1F4F8823CD
:1031700011F40C9484290E947D3DF801F4CF80E580
:103180000E94613D882379F08091AC039091AD035A
:10319000009749F04AE050E060E070E00E94E3C32D
:1031A0006B017C0103C0C12CD12C760183E50E9408
:1031B000613D882361F00E94E13C20E030E04AE775
:1031C00054E40E94C9C50E94D7CA6B017C010E94C9
:1031D000DD660E94F2B2C60ED71EE81EF91E0E94DE
:1031E000F2B2DC01CB018C199D09AE09BF09B7FD14
:1031F00002C00C9484290E94BE4EF1CF80E00E9450
:103200008A990C94842983E50E94613D882321F1E9
:103210000E94C13C182F863070F0E5EEF2E08491F8
:103220008F010F5F1F4F882311F40C9484290E9493
:103230007D3DF801F4CF833009F44AC130F4813088
:1032400091F1823009F43FC008C0843009F49FC175
:10325000853009F4ACC101C010E00E943D99811194
:1032600003C0E5ECF2E013C080913B16882319F00F
:103270006BE073E002C06FE073E08DEB92E00E94C0
:10328000074C8AE00E947D3D0E94FEA796C1849172
:103290007F019FEFE91AF90A882309F48EC10E9481
:1032A0007D3DF701F4CF0E94B1A810920102109267
:1032B000000282EB92E09093FC0C8093FB0C0E9446
:1032C000A93D0C948429809100029091010297FFFE
:1032D0000EC0E9E8F2E084918F010F5F1F4F882351
:1032E00011F40C9484290E947D3DF801F4CF0097DD
:1032F000A1F4809121028093B30319821A821B8268
:103300001C8218A219A21AA21BA2BE016F5F7F4FD6
:10331000CE0180960E945DB027C0815065E00E947A
:1033200056CC80FF03C024E0291B922FA5E09A020F
:10333000F0011124E80FF11D87FDFA95EE0FFF1F34
:10334000EE0FFF1FED53FA4E8091C5039091C60317
:10335000A091C703B091C80380839183A283B383F4
:103360008091B30380932102809100029091010229
:10337000893191050CF067C0109221029C012F5FEA
:103380003F4F309301022093000265E00E9456CC2B
:1033900080FF03C024E0291B922F4091C503509168
:1033A000C6036091C7037091C80348A359A36AA3D9
:1033B0007BA319821A821B821C82B4E08B029001CB
:1033C0001124F901EF5BF04F4F01208131814281DF
:1033D0005381F4E09F02C0011124BC016B5A704F6D
:1033E0005B01DB016D917D918D919C91FE01319688
:1033F0006F01E12CF12C00EA10E40E948DAF1982DC
:103400001A821B821C82B601CE0180960E945DB09A
:10341000F50180819181A281B3818093BD03909356
:10342000BE03A093BF03B093C003F40180819181D8
:10343000A281B3818093C1039093C203A093C3037D
:10344000B093C403BCC080E090E0A0EAB0E48093F5
:10345000C5039093C603A093C703B093C8030E940B
:10346000779A0E94DD668FEF9FEF90930102809321
:103470000002E5E7F2E084918F010F5F1F4F882380
:1034800021F00E947D3DF801F6CF83E992E09A8316
:10349000898304E610E019A308A3BE016F5F7F4F84
:1034A000CE0180960E9410B18AEB92E09A838983C4
:1034B00019A308A3BE016F5F7F4FCE0180960E94C3
:1034C00010B181E00E948A9981E00E946A9977C0D8
:1034D00088E50E94613D8823A1F00E94B13C1FEF66
:1034E000160F1530A8F0EEE5F2E084918F010F5F22
:1034F0001F4F882311F40C9484290E947D3DF8010C
:10350000F4CF88E50E947D3D0E9455C10C9484292A
:1035100089E50E94613D8823A1F00E94B13C0FEF34
:10352000060F0530A8F0E7E4F2E084918F010F5F09
:103530001F4F882311F40C9484290E947D3DF801CB
:10354000F4CF89E50E947D3D0E9455C10C948429E9
:103550008AE50E94613D882399F00E94E13C25E0C4
:10356000129FF0011124E00FF11DEE0FFF1FEE0F6F
:10357000FF1FED53FA4E608371838283938335C0BE
:103580008AE50E947D3D0E9455C10C9484298AE5FC
:103590000E94613D8823A1F30E94E13C6093BF1526
:1035A0007093C0158093C1159093C2151EC080E022
:1035B0000E946A990E94B1A818C01230B1F46091BB
:1035C0000002709101026931710514F069E170E047
:1035D00088E392E00E94EE4B69E170E083E392E0C1
:1035E0000E94EE4B8AE00E947D3D0E9445950C941E
:1035F000842980914102882311F40C94842989E460
:103600000E94613DE82E882321F00E94B13C062FE4
:1036100001C000E08AE40E94613DF82E882321F079
:103620000E94B13C162F01C010E0EE2011F00530D1
:1036300020F4FF2081F0153070F0ECEFF2E084917F
:103640008F010F5F1F4F882311F40C9484290E946F
:103650007D3DF801F4CF0E94733DEE2091F034E0FF
:103660000302F0011124EB5AF04F80819181A28175
:10367000B3818093DA0A9093DB0AA093DC0AB093BB
:10368000DD0AFF2091F044E01402F0011124EF5B09
:10369000F04F80819181A281B3818093DE0A909363
:1036A000DF0AA093E00AB093E10A80E50E94613D41
:1036B000882319F00E94D23C03C080E50E94183D87
:1036C00086E40E94613D8823D9F00E94E13C6B01B1
:1036D0007C0120E030E0A9010E94B4CB181684F4EC
:1036E00020E030E040E752E4C701B6010E946ACA18
:1036F00060934B0270934C0280934D0290934E0264
:103700000E947E520C9484291092B2030C94842956
:103710009093B2030C9484290E94E13C2B013C015C
:10372000133049F0F60120813181428153810E949A
:103730008DC92B013C01A8ADB9AD2D913D914D91A5
:103740005C91C301B2010E948DC94B015C012DEB5C
:1037500037E346E855EB0E94B4CB87FD20C02DEB44
:1037600037E346E855E3C501B4010E9464C5181665
:10377000B4F01F5FB4E0EB0EF11CE8ADF9AD349688
:10378000F9AFE8AFF4E0CF0ED11C143039F1D1011C
:103790008D911D010E94613D882359F3BDCF1330E7
:1037A00051F44092C9035092CA036092CB037092C5
:1037B000CC0301E0DECFA5019401F70160817181A6
:1037C000828193810E948EC9D7016D937D938D93E1
:1037D0009C931397812F0E94CE9ACBCF002309F49C
:1037E00004CFC090C903D090CA03E090CB03F090FF
:1037F000CC0320E030E0A901C701B6010E948EC9C8
:103800002091B5163091B6164091B7165091B81662
:103810000E94C9C50E94BFCB60933D0F70933E0FBD
:1038200080933F0F9093400FC0922D0FD0922E0F98
:10383000E0922F0FF092300F90910B0F80910C0FB0
:10384000981719F00E947F66D0CE0E94DD668091A5
:103850006F00982F927081FF05C080916F008D7F5F
:1038600080936F0040913D0F50913E0F60913F0F4C
:103870007091400F4093311550933215609333157A
:1038800070933415992309F4B0CE80916F00826053
:1038900080936F00AACE0E9444B10C948429809139
:1038A0007216909173168637910509F4AAC70CF029
:1038B000CEC08D34910509F4D1C40CF05AC08A31C0
:1038C000910509F43DC264F58531910509F4F6C10D
:1038D000C4F48231910509F432C68431910509F4AA
:1038E000ADC1419711F00C9433295F988A9847989D
:1038F00080910801817080930601479812980C947A
:1039000084298731910509F4E3C10CF4DBC18831C6
:10391000910509F4F3C1499709F4FBC10C943329CB
:103920008F31910509F49AC384F48C31910509F41F
:10393000ADC20CF413C28D31910511F40C9484299D
:103940004E9709F4ADC20C9433298A32910509F4DB
:1039500038C42CF4809709F435C30C9433298B3484
:10396000910509F462C48C34910509F462C40C9485
:1039700033298B36910509F4B4C50CF042C0853566
:10398000910509F40BC6FCF48235910509F4D0C504
:1039900084F48135910511F00C9433290E94DF7C69
:1039A0000E946FA31092CE031092CD0300E010E0AE
:1039B000A8C58335910509F4BEC58435910509F480
:1039C000BEC50C9433298836910509F44BC47CF4A8
:1039D0008C35910511F00C943329FFE4CF2EF2E0E1
:1039E000DF2EA9EAEA2EA6E1FA2E10E0F0C589360C
:1039F000910509F4FAC48A36910509F456C50C9468
:103A000033298037910509F4BFC484F48D369105BC
:103A100009F42BC50CF4B5C48E36910509F44BC4DA
:103A20008F36910509F45AC40C94332982379105D5
:103A300009F44DC60CF4AFC48337910509F4FBC0FB
:103A40008537910511F40C9484290C9433298E3216
:103A500021E0920711F40C946F270CF06EC08B3CA0
:103A6000910509F48CC7ACF58C38910509F400C5B3
:103A70008CF48837910509F413C70CF40EC7893705
:103A8000910511F00C9433291092680B1092670B7A
:103A90000C9484298E3B910509F404C534F48B39C8
:103AA000910509F4BDC40C943329883C910509F4AF
:103AB000FDC6893C910511F00C9433297FE4E72E73
:103AC00072E0F72E09E816E1E9E9CE2EE6E1DE2EF6
:103AD0003DC78C3D910511F40C940326A4F48D3C54
:103AE000910509F4DDC70CF466C78E3C910511F40D
:103AF0000C94DD25833D910511F00C9433290E942F
:103B0000AB8C0C948429823E910511F40C947D2693
:103B10003CF48D3D910511F40C9410260C9433293E
:103B20008C3241E0940711F40C94A6268D3291401A
:103B300011F40C94CF260C943329853F61E096074D
:103B400011F40C945C28E4F58A39A1E09A0709F491
:103B50001FC4BCF48033E1E09E0711F40C94C62727
:103B600014F40C94C327833621E0920709F45FC054
:103B70008039914011F00C9433290E94DD660C9439
:103B80008429853A41E0940711F40C9459284CF4A7
:103B9000843A914011F00C9433290E946F850C9463
:103BA00084298C3A71E0970711F40C940026843F25
:103BB000914011F00C9433290E94246D0C948429B7
:103BC0008A39B2E09B0711F40C949B28B4F4873F28
:103BD000F1E09F0711F40C94622814F40C945F2810
:103BE000883F31E0930711F40C946E288C3092409A
:103BF00011F40C9492280C9433298B3853E09507D8
:103C000011F40C9484293CF48438934011F40C94FE
:103C1000C8280C943329803AA3E09A0709F411C20A
:103C2000873E934011F40C9420290C943329E8ED3D
:103C3000F8E10C944628E3EFF4E088C5EAE2F3E00B
:103C400084918F010F5F1F4F882321F00E947D3DDB
:103C5000F801F6CF109207128AEB9FE00E942290A3
:103C60008BE1EAEBFFE0DE01159601900D928A955B
:103C7000E1F78091B80F9091B90F9C838B8385EE0B
:103C800092E09A83898340E050E0BE016F5F7F4FEE
:103C900080E090E00E945976CE0101960E94544E39
:103CA000EBE1F3E084918F010F5F1F4F882311F444
:103CB0000C9484290E947D3DF801F4CF0E94287461
:103CC0000C9484291092890F10928A0F0C948429E5
:103CD000E0917016F09171168081882329F080326E
:103CE00009F410823196F8CF40E061E080917016BF
:103CF000909171160E945AB30C94842980918A0F76
:103D0000882319F081E08093890F0E94A87C0C948D
:103D100084291092890F80913915813011F00C940B
:103D2000842982E0809339150E94F2B260933515A0
:103D30007093361580933715909338150C94842919
:103D400080918A0F882311F40C94842983E50E94C2
:103D5000613D81110C948E290C94842983E40E9486
:103D6000183D882309F450C0E8E6F3E084918F0100
:103D70000F5F1F4F882321F00E947D3DF801F6CF91
:103D800080915511811103C0EBE3F3E012C0BE0135
:103D90006F5F7F4F82E591E10E94EA8E8E010F5F97
:103DA0001F4FF80181918F01882349F10E947D3DC9
:103DB000F8CF84918F010F5F1F4F882301F10E947C
:103DC0007D3DF801F6CFB6EECB2EB3E0DB2EE12C35
:103DD000F12C20E08091510B90E00E2C02C09595C3
:103DE00087950A94E2F780FDA9C29FEFE91AF90AC4
:103DF000A2E0CA0ED11CB5E0EB16F10459F78AE037
:103E00000E947D3D0C94842980918A0F882339F08B
:103E10008091890F882319F0E5E4F3E003C0E7E51A
:103E2000F3E028C084918F010F5F1F4F882321F09A
:103E30000E947D3DF801F6CF60910312709104124B
:103E400080910512909106124AE00E9499408FE2FB
:103E50000E947D3D6091FF117091001280910112CE
:103E6000909102124AE00E9499408AE00E947D3DB2
:103E70000C94842984918F010F5F1F4F882311F4C4
:103E80000C9484290E947D3DF801F4CF40E060E06D
:103E900080917016909171160E945AB30C948429E7
:103EA00080918A0F882311F40C94842982E591E192
:103EB0000E943BAD82E591E10E94C58E1092880F71
:103EC0001092870F80918A0F882311F40C94842913
:103ED00000917016109171160E944C76B801CE01B7
:103EE00080960E9460788C01892B11F40C948429AF
:103EF00068A179A16115710511F06C5F7F4F19827E
:103F00001C8222E0A801CE0101960E9458948111E2
:103F100002C0F12C14C0CE0101960E94BA7588230C
:103F2000C1F361E0CE0101960E94CE8E009789F325
:103F300025EEDC012C931C820E94E4AAF82ECE010F
:103F400001960E946D3DF11003C0E5E8F3E022C048
:103F5000E7E7F3E084917F01BFEFEB1AFB0A8823C8
:103F600021F00E947D3DF701F5CFF80181918F018D
:103F7000882319F00E947D3DF8CF8AE00E947D3DA4
:103F8000109203121092041210920512109206124F
:103F90000C94842984917F012FEFE21AF20A88237E
:103FA00021F00E947D3DF701F5CFD8018D918D0163
:103FB000882319F00E947D3DF8CF8EE20E947D3D5E
:103FC0000C9484298091890F81110E94DD66809173
:103FD0008A0F882311F40C94842980E50E94613DA6
:103FE000882319F00E94D23C03C080E50E94183D4E
:103FF000182F482F61E080917016909171160E94E1
:104000005AB383E50E94613D882381F00E94B13C50
:10401000AB01BC014093031250930412609305124C
:104020007093061282E591E10E94DB8D80918A0FE8
:10403000882319F081E08093890F11110C94842951
:1040400064CE809170169091711621E02093880FB4
:1040500040E060E00E945AB30C9484290E94597C8D
:104060007B018C0120E831E541E050E00E9452C91B
:10407000C9016DE671E00E9463CC4B015C01C8018F
:10408000B70120E13EE040E050E00E9452C9CA0181
:10409000B90128E130E040E050E00E9452C9762E9C
:1040A000672EC62ED72E8CE3282E312C412C512C76
:1040B000C801B701A20191010E9452C9F62EE72E54
:1040C000CA01B901A20191010E9452C9CB018E011E
:1040D0000F5F1F4F81149104D1F0EF92FF927F93F5
:1040E0006F936F927F92BF92AF929F928F9285EC67
:1040F00093E09F938F931F930F930E9436C50FB643
:10410000F894DEBF0FBECDBFEDEEF8E145C0A114BF
:10411000B10489F0EF92FF927F936F936F927F9239
:10412000BF92AF9285EB93E09F938F931F930F9372
:104130000E9436C5E4CFCD2879F0EF92FF927F93AD
:104140006F936F927F9289EA93E09F938F931F936F
:104150000F930E9436C5D3CF892B69F0EF92FF925F
:104160007F936F9381EA93E09F938F931F930F93B5
:104170000E9436C5C4CFEF92FF928DE993E09F93E2
:104180008F931F930F930E9436C50F900F900F903F
:104190000F900F900F90B8CF84917F017FEFE71AB7
:1041A000F70A882321F00E947D3DF701F5CFB80181
:1041B00089ED93E00E94074C8AE00E947D3D0C94BB
:1041C000842983E50E94613D882311F40C9484299D
:1041D0000E94C13CE82E80E50E94613D882339F0B1
:1041E0000E94C13C182F87FF03C00C9484291DE056
:1041F00089E40E94613D882341F00E94D23C8111F4
:104200000C94FC29EDE0F6E00BC089E40E94183D17
:10421000F6CF319686E0ED33F80711F40C94FC29C3
:1042200084911813F6CF0C94D1290E94A87C0C9489
:10423000842980913915813011F00C94842982E011
:10424000809339150E94F2B260933515709336153C
:1042500080933715909338150C9484290E94CA7C5A
:104260000C94842988E690E00E940E9B81110C94A6
:1042700084298091510B83FF02C00C94842983E52B
:104280000E94613D882399F00E94E13C0E94D2CABD
:10429000CB010E94C1720E94E13C20E030E044EB7F
:1042A00052E40E9464C5181614F00E94CA7C0E9451
:1042B000524C0C9484298EE40E94613D882311F4B1
:1042C0000C9484290E94B13C60934E1670934F1653
:1042D00080935016909351160C94842983E50E9484
:1042E000183D882359F083E50E94613D882319F029
:1042F0000E94C13C01C080E08093510BEDEEF8E1DB
:1043000084918F010F5F1F4F811103C0E4EFF3E031
:1043100004C00E947D3DF801F3CF84918F010F5FAF
:104320001F4F882321F00E947D3DF801F6CF809138
:10433000510B811148CDE0EFF3E018C0BB24B394DA
:10434000B20E222319F08CE20E947D3DF601859188
:104350009491FC0184918F010F5F1F4F882321F0FE
:104360000E947D3DF801F6CF2B2D3FCD84918F012A
:104370000F5F1F4F882309F442CD0E947D3DF80155
:10438000F5CF10924002C0C78BEF93E00E94774EAA
:104390000E943687B9C783E50E94613D811103C041
:1043A000EDEEF8E10BC00E94C13C8D3318F4809310
:1043B0002202AAC78CE380932202A6C784918F01B0
:1043C0000F5F1F4F882321F00E947D3DF801F6CF3B
:1043D0004091220250E060E070E084E094E00E94AE
:1043E000B44B8AE00E947D3D8FC789E690E00E9431
:1043F0000E9B811111C0EBE0F4E084918F010F5FFF
:104400001F4F882321F00E947D3DF801F6CF0E94C6
:10441000E1798AE00E947D3D1092BF0A0C94112A36
:1044200083E50E94613D882309F46EC70E94C13C68
:10443000182F8D3308F01CE31093CC0A0E94F2B2BF
:104440006B017C01212F30E0A8EEB3E00E947EC911
:10445000C60ED71EE81EF91EC092C80AD092C90A1D
:10446000E092CA0AF092CB0A4FC70E94509B4CC7F9
:104470008091510B83FD48C783E50E94613D8823ED
:1044800009F442C70E94E13C0E94D2CA6E3671050F
:1044900014F06EE670E07093D0036093CF030E9437
:1044A0009B7A32C70E940F962FC780E50E94613D1C
:1044B000811106C083E50E94613D882359F005C043
:1044C0000E94C13C811120C7F5CF0E94B13C6F3FD3
:1044D000710510F06FEF70E07093CE036093CD0321
:1044E00013C780E50E94613D811105C01092CE0383
:1044F0001092CD0309C70E94B13C672B09F004C795
:10450000F5CF62E370E080E090E00E94BAB20E94D2
:104510009F7F0F5F1F4F0331110599F762E370E032
:1045200080E090E00E94BAB20E949F7F94D7ECC6D0
:104530001092B103E9C681E08093B103E5C683E53B
:104540000E94613D882399F00E94E13C20E030E028
:104550004AE754E40E94C9C50E94D7CA6093230267
:10456000709324028093250290932602CDC688E59D
:104570000E94183D8111E3C689E50E94183D811112
:10458000DEC68AE50E94183D8111D9C685E40E94E5
:10459000183D8111D4C60E946FA3B6C683E50E9460
:1045A000183D882309F4B0C60E94E13C20E030E0C9
:1045B0004AE754E40E94C9C50E94D7CA6093C40A5E
:1045C0007093C50A8093C60A9093C70A9DC6F601E8
:1045D00081916F010E94183D882309F46EC0133049
:1045E00009F063C00E94E13C4B015C0120E030E037
:1045F00040EA51E40E9464C587FF4EC0A5019401C2
:104600006091B5167091B6168091B7169091B81654
:104610000E946ACA2B013C019B01AC016091200BF6
:104620007091210B8091220B9091230B0E94C9C5A0
:104630006093200B7093210B8093220B9093230B9C
:10464000A30192016091400B7091410B8091420B4C
:104650009091430B0E94C9C56093400B7093410B2E
:104660008093420B9093430B609185167091861650
:1046700080918716909188160E9468C5A3019201C7
:104680000E94C9C50E94D7CA60938516709386168A
:1046900080938716909388168092B5169092B616DE
:1046A000A092B716B092B81608C00E94E13CD7019C
:1046B0006D937D938D939C9313971F5FB4E0EB0EE6
:1046C000F11C143009F083CF0E9453B91DC60E941B
:1046D000DD6683E50E94613D882311F40C94F51A90
:1046E0000E94B13C6230710511F00C94F51A0E94E1
:1046F0005A568BE50E947D3D6091B20A7091B30AD3
:104700008091B40A9091B50A42E00E941E41409106
:10471000B60A5091B70A6091B80A7091B90A81E15E
:1047200094E00E94D14B4091BA0A5091BB0A60912B
:10473000BC0A7091BD0A8EE094E00E94D14B8DE5D9
:104740000E947D3D8AE00E947D3DDEC584918F01FF
:104750000F5F1F4F882321F00E947D3DF801F6CFA7
:1047600060E083EE94E00E94898D61E08CED94E03E
:104770000E94898D61E081ED94E00E94898D61E065
:1047800081EC94E00E94898D60E088EB94E00E94C7
:10479000898D61E08EEA94E00E94898D60E084EA70
:1047A00094E00E94898D60E08CE994E00E94898DFC
:1047B00061E08EE894E00E94898D60E080E894E0FA
:1047C0000E94898D60E081E794E00E94898D60E01D
:1047D00083E694E00E94898D60E08DE494E00E947D
:1047E000898D60E08CE394E00E94898D60E087E22F
:1047F00094E00E94898D61E084E194E00E94898DBB
:1048000083C5009170161091711683E0D12C40E0A1
:104810008150E1F0F8019081292F2B7F2134C1F7DD
:1048200021812133A9F7913421F0953421F441E01D
:1048300002C0DD24D39498012E5F3F4F89012F5F82
:104840003F4FD8019C919032C9F3E2CF442369F0E5
:10485000EDEEF8E184917F01BFEFEB1AFB0A8823AC
:1048600021F00E947D3DF701F5CFDD2069F0E9EBF5
:10487000F5E084917F012FEFE21AF20A882321F0FC
:104880000E947D3DF701F5CFD8018D918D018823E0
:1048900009F4B5CA0E947D3DF7CF0E9449A934C5ED
:1048A00081E08093680B8093670B2EC588EC90E0C5
:1048B0000E940E9B811128C584E40E94183D882324
:1048C00009F441C00E94E13C6B017C0111E020E051
:1048D00030E0A9010E9464C5811101C010E010936D
:1048E000271620E030E0A901C701B6010E9464C587
:1048F000882349F10E94E13CE0915C15B4E0EB9F14
:10490000F0011124E45DF94E608371838283938307
:1049100020E030E0A90160912C1670912D16809155
:104920002E1690912F160E9464C581110CC080E054
:1049300090E0A0EEBFE380932C1690932D16A093E9
:104940002E16B0932F160E94ADA3DEC4F7018191FD
:104950007F010E94183D882351F00E94E13C0E9493
:10496000D7CAD8016D937D938D939C9313970C5F59
:104970001F4FC016D10651F70E94E2B7C5C46FE4BD
:10498000E62E62E0F62E04E31BE0F70181917F0141
:104990000E94183D882341F00E94E13CD8016D93AC
:1049A0007D938D939C9313970C5F1F4FBBE0043452
:1049B0001B0759F7A9C483E50E94613D8823A1F034
:1049C0000E94E13C60932C0B70932D0B80932E0B77
:1049D00090932F0B6093280B7093290B80932A0BD5
:1049E00090932B0B10E001C011E080E50E94613D27
:1049F000882359F00E94E13C60932C0B70932D0B9F
:104A000080932E0B90932F0B10E082E50E94613D66
:104A1000882359F00E94E13C6093300B7093310B76
:104A20008093320B9093330B10E084E50E94613D3C
:104A3000882359F00E94E13C6093280B7093290B66
:104A400080932A0B90932B0B5FC4112309F45CC451
:104A500040912C0B50912D0B60912E0B70912F0BD0
:104A600083EC95E00E94D14B4091300B5091310B7B
:104A70006091320B7091330B80EC95E00E94D14B2A
:104A80004091280B5091290B60912A0B70912B0BB0
:104A90008DEB95E00E94D14B8AE00E947D3D34C4AD
:104AA00081E50E94183D8823C1F08091AC0390916C
:104AB000AD03009739F04AE050E060E070E00E94FA
:104AC000E3C303C060E070E0CB016093440B7093DC
:104AD000450B8093460B9093470B83E50E94183D4E
:104AE000882351F00E94E13C60934C0B70934D0B76
:104AF00080934E0B90934F0B84E50E94183D8823C2
:104B000051F00E94E13C6093480B7093490B8093F5
:104B10004A0B90934B0B88E50E94183D882351F077
:104B20000E94E13C6093140B7093150B8093160B5D
:104B30009093170B89E50E94183D882351F00E943D
:104B4000E13C6093180B7093190B80931A0B9093B0
:104B50001B0B8AE50E94183D8823F1F00E94E13C7E
:104B600060931C0B70931D0B80931E0B90931F0B77
:104B70002DEC3CEC4CEC5DE30E9464C5181664F02F
:104B8000E3EDF5E084918F010F5F1F4F882321F043
:104B90000E947D3DF801F6CF85E40E94183D8823F0
:104BA00009F4B2C30E94E13C6093200B7093210B87
:104BB0008093220B9093230BA7C34FE4C42E42E0B3
:104BC000D42E59E6E52E5BE0F52E10E0F60181913A
:104BD0006F010E94183D882359F00E94E13CD701E3
:104BE0006D937D938D939C931397812F0E94CE9A02
:104BF0001F5FB4E0EB0EF11C133041F70C94F51A73
:104C00000E942B8381C383E50E94613D882309F4C0
:104C10007BC30E94B13C709303026093020274C391
:104C20008DED90E00E940E9B81116EC383E50E9482
:104C3000613D811103C0EDEEF8E139C000915C15D2
:104C400010E00E94B13C000F111FF801E75BFD4F1F
:104C50007183608380915C1590E07C01EE0CFF1CF9
:104C6000EE0CFF1C87010D5C1D4F880F991FFC0186
:104C7000E75BFD4F60817181072E000C880B990B5B
:104C80000E946AC52AE037ED43E25CE30E94C9C591
:104C9000F701E85DF94E20813181428153810E9404
:104CA000C9C5F80160837183828393832DC3849186
:104CB0008F010F5F1F4F882321F00E947D3DF80177
:104CC000F6CF85E40E947D3D80915C15805D0E9459
:104CD0007D3DE0915C15F0E0EE0FFF1FE75BFD4FBF
:104CE0006081718185E096E00E94EE4B85E20E9432
:104CF0007D3D8AE00E947D3D07C380E50E94183D0E
:104D0000882309F401C30E94B13C6B017C0183E557
:104D10000E94613D882321F00E94B13C8B0102C0BA
:104D20000FEF1FEFC8010196039708F0EDC2D7FC03
:104D3000EBC28C2DEDE0F6E09491891709F431C3B4
:104D4000319626E0ED33F207B9F72EC383E50E94D2
:104D5000613D882319F00E94B13C02C064E071E01B
:104D600079A368A380E50E94613D882339F00E9401
:104D7000B13C693833E1730730F402C068EE73E088
:104D80007A83698304C088E893E19A838983BE01AA
:104D9000605E7F4FCE0101960E9410B1B5C285E4DE
:104DA0000E94613D811110C080E50E94183D88235A
:104DB00091F00E94E13C60934A1570934B158093EB
:104DC0004C1590934D1507C00E94C13C882361F398
:104DD000E8EDF8E171C089E40E94183D882381F074
:104DE0000E94E13C2CEA35EC47E25EE30E94C9C533
:104DF0006093461570934715809348159093491515
:104E000084E40E94183D882381F00E94E13C2CEA52
:104E100035EC47E25EE30E946ACA60934E157093D8
:104E20004F158093501590935115EDEEF8E1849154
:104E30008F010F5F1F4F882321F00E947D3DF801F5
:104E4000F6CF40914A1550914B1560914C157091D9
:104E50004D1585E496E00E94D14B2CEA35EC47E2F3
:104E60005EE36091461570914715809148159091C9
:104E700049150E946ACAAB01BC0181E496E00E9418
:104E8000D14B2CEA35EC47E25EE360914E15709110
:104E90004F1580915015909151150E94C9C5AB01D5
:104EA000BC018DE396E00E94D14B8AE00E947D3DDB
:104EB0002BC20E947D3DF80184918F010F5F1F4F2F
:104EC0008111F7CFE9E4F6E084918F010F5F1F4F66
:104ED000882309F419C20E947D3DF801F5CF83E5CE
:104EE0000E94183D182F882371F00E94E13C0E9417
:104EF000D2CA709338026093370221E0672B09F021
:104F000020E02093500B80E50E94183D882359F043
:104F10002091370230913802232B11F00E94D23CAD
:104F20008093500BF1C11111EFC1EDEEF8E18491C6
:104F30008F010F5F1F4F882321F00E947D3DF801F4
:104F4000F6CF8091500B882319F063E173E002C023
:104F500066E173E080E796E00E94074C60913702BB
:104F6000709138028FE596E00E94EE4BEBE5F6E09B
:104F700084918F010F5F1F4F882309F4C5C10E94E0
:104F80007D3DF801F5CF0E947387BEC180E50E9488
:104F9000183D882351F00E94E13C609342157093C4
:104FA0004315809344159093451589E40E94183D5C
:104FB000882381F00E94E13C2CEA35EC47E25EE375
:104FC0000E94C9C560933E1570933F1580934015AC
:104FD0009093411584E40E94183D882381F00E943B
:104FE000E13C2CEA35EC47E25EE30E946ACA60933A
:104FF0003A1570933B1580933C1590933D15EDEE5B
:10500000F8E184918F010F5F1F4F882321F00E94E8
:105010007D3DF801F6CF40914215509143156091C6
:105020004415709145158BE896E00E94D14B2CEA0F
:1050300035EC47E25EE360913E1570913F1580913B
:105040004015909141150E946ACAAB01BC0187E8E6
:1050500096E00E94D14B2CEA35EC47E25EE360918A
:105060003A1570913B1580913C1590913D150E9429
:10507000C9C5AB01BC0183E896E00E94D14B8AE030
:105080000E947D3D41C10E947D3DF80184918F01C8
:105090000F5F1F4F8111F7CFEFE8F6E084918F018A
:1050A0000F5F1F4F882309F42FC10E947D3DF80137
:1050B000F5CF0E94848428C10E94186D25C10E94EA
:1050C000E1A122C183E50E94183D882321F00E94BE
:1050D000D23C91E089270E944D9D16C181E08093CA
:1050E000580B0E940E671092580B882309F40CC1CC
:1050F000EDEEF8E184918F010F5F1F4F811103C026
:10510000EEE9F6E004C00E947D3DF801F3CF849102
:105110008F010F5F1F4F882309F4F6C00E947D3D69
:10512000F801F5CF8091890F882309F4EDC081E063
:1051300080938C0FE9C08AE50E94613D811103C014
:10514000ECEAF6E00BC00E94E13C6093BB15709363
:10515000BC158093BD159093BE15D6C084918F0168
:105160000F5F1F4F882321F00E947D3DF801F6CF8D
:105170004091BB155091BC156091BD157091BE1545
:1051800089EA96E00E94D14B8AE00E947D3DBCC036
:105190008BE40E94613D811103C0EDEEF8E136C061
:1051A0008BE40E94613D8823C1F00E94E13C6B01C9
:1051B0007C0120E030E0A9010E94B4CB87FD0AC049
:1051C00020E030E040E251E4C701B6010E9464C52E
:1051D000181634F4EBECF6E00EC0C12CD12C76019D
:1051E0000E94DD66C092240BD092250BE092260B24
:1051F000F092270B89C084918F010F5F1F4F882386
:1052000009F482C00E947D3DF801F5CF84918F01A1
:105210000F5F1F4F882321F00E947D3DF801F6CFDC
:105220004091240B5091250B6091260B7091270B18
:105230008AEE96E00E94D14B8AE00E947D3D64C0D8
:1052400081E08093410283E50E94613D882339F02B
:105250000E94D23C811158C00E94935655C083E5EC
:105260000E94183DF7CF0E9444B14EC0F0907216D4
:105270000E94DD6610913B1680E00E946A99FF2033
:1052800029F1EDEEF8E184918F010F5F1F4F882324
:1052900021F00E947D3DF801F6CF84E50E947D3D1E
:1052A0006F2D70E080E090E04AE00E94994080E23B
:1052B0000E947D3DE7E0F7E084918F010F5F1F4F73
:1052C000882311F10E947D3DF801F6CF1092BE0AAD
:1052D000812F0E946A99EDEEF8E184918F010F5FB2
:1052E0001F4F882321F00E947D3DF801F6CF609189
:1052F000BE0A70E085EF96E00E94EE4B8AE00E94C5
:105300007D3D02C00E9444B11092BF0A0E947656B1
:1053100088C00E94EA970E947E52F6CF0E94B13C5C
:10532000AB01BC0140930312509304126093051229
:105330007093061282E591E10E94DB8DE5CF0E9419
:10534000DD6688E50E94183D882331F05F9A8091E0
:10535000BC038E7F8093BC0389E50E94183D88239F
:1053600039F08A9A479A8091BC038D7F8093BC0361
:105370008AE50E94183D882361F08091080180959C
:10538000817080930601479A8091BC038B7F809344
:10539000BC0385E40E94183D882309F4B5CF129A16
:1053A000B3CF0E943AC1B0CF0E94DD66BC2C60E052
:1053B0008C2D0E94B7B10F3F4FEF140759F48C2D7D
:1053C0000E9461B131E020E0892B09F030E0032F29
:1053D000122F05C00130110561F401E010E08B2DA2
:1053E0000E9461B18017910709F48ECF0E94BE4ED2
:1053F000F6CF00E010E0F3CF61E0812F0E94B7B15B
:105400006E2D812F0E9489B1F12CB701812F0E944E
:10541000F3B1193009F078CFF092CE03E092CD03CA
:1054200073CFC559DF4F0FB6F894DEBF0FBECDBFA7
:10543000DF91CF911F910F91FF90EF90DF90CF9070
:10544000BF90AF909F908F907F906F905F904F90A4
:105450003F902F9008952F923F924F925F926F92BC
:105460007F928F929F92AF92BF92CF92DF92EF92F4
:10547000FF920F931F93CF93DF93CDB7DEB76F9754
:105480000FB6F894DEBF0FBECDBFC090D703D0904B
:10549000D803E090D903F090DA0320E030E040EA4E
:1054A00050E4C701B6010E9464C587FD19C120E020
:1054B00030E041E953E4C701B6010E94B4CB1816AD
:1054C0000CF40EC11092A6131092A513809109013D
:1054D0004091A413042E000C550B817021E082270B
:1054E00090E04817590709F433C080910901817091
:1054F00028272093A41381111BC00E942874E5E083
:10550000FBE084918F01882351F0082E000C990B49
:105510000E9423740F5F1F4FF8018491F4CF8DE038
:1055200090E00E9423748AE090E00E94237410C0EF
:10553000E9E0FBE084918F01882389F3082E000CB9
:10554000990B0E9423740F5F1F4FF8018491F4CFD1
:1055500080919713833009F44CC02CF4882351F0C8
:105560008130D9F072C0843009F43EC0853009F42E
:105570004DC06BC08091890F882309F466C081E01B
:10558000809397130E94F2B260939B1370939C13C5
:1055900080939D1390939E1358C08091890F811121
:1055A00054C080915511882321F082E08093971395
:1055B0004CC010929713E1E0FBE084918F018823A7
:1055C00051F0082E000C990B0E9423740F5F1F4F9F
:1055D000F8018491F4CF8DE090E00E9423748AE07A
:1055E00090E00E94237431C08091E4138823E9F293
:1055F0002CC08091890F811128C080910B0F909150
:105600000C0F891B8F7009F496C01FC08091890F01
:1056100081111BC080910B0F90910C0F891B8F7013
:1056200009F4ABC012C08DE090E00E9423748AE0C0
:1056300090E00E9423741092971381EE9AE0909369
:10564000FC0C8093FB0C0E94A93D80918C139091DF
:105650008D1303974CF57BEE272E77E0372EE0E68F
:105660008E2EEAEE9E2EA12CB12C82EF94E10E94A8
:105670008A3818161906C4F480918C1390918D13F2
:10568000049794F482EF94E10E944E388093921331
:10569000E0919313F09194138A3019F08D3009F052
:1056A0007DC0309709F083C080918C1390918D1349
:1056B000009711F40C94BF37019790938D1380934A
:1056C0008C1380918E1390918F13019664E070E09B
:1056D0000E9477CC90938F1380938E130C94BF37D6
:1056E0008091A5139091A6138136FAEE9F07E8F0FA
:1056F0001092A6131092A513EDE0FBE084918F01A8
:10570000882351F0082E000C990B0E9423740F5F20
:105710001F4FF8018491F4CF8DE090E00E94237434
:105720008AE090E00E942374D1CE01969093A61354
:105730008093A513CBCE8DEE9AE09093FC0C8093D2
:10574000FB0C0E94A93D8091E413882311F082E0B4
:1057500001C084E080939713E9EEFAE084918F0111
:10576000882309F438CF082E000C990B0E9423746B
:105770000F5F1F4FF8018491F3CFE5EEFAE08491BB
:105780008F01882309F44FCF082E000C990B0E943B
:1057900023740F5F1F4FF8018491F3CF8A3309F40C
:1057A00080CFEF35F10514F40C9458357ACF809101
:1057B00090139091911320E6289F7001299FF00C7F
:1057C00011248701045F1D4EE00FF11F108261E478
:1057D00070E0C8010E94FACC009711F40C943C359B
:1057E0009093961380939513801B910B8E0D9F1DA4
:1057F00060E070E0835F9D4E0E9465C10E94D2CA46
:10580000CB01770FAA0BBB0B8232910510F00C94E1
:105810003C35FC018827EE58FF4F8F4F0C94A6CCE7
:10582000ECEDFAE084918F01882351F0082E000CF2
:10583000990B0E9423740F5F1F4FF8018491F4CFDE
:1058400020E030E040E05FE36091D7037091D8033F
:105850008091D9039091DA031EC0E7EDFAE08491BC
:105860008F01882351F0082E000C990B0E9423749D
:105870000F5F1F4FF8018491F4CF6091D5037091B1
:10588000D603072E000C880B990B0E946AC520E0F6
:1058900030E040E05FE30E948EC90E94D2CACB0193
:1058A0000E94B9410E9492B58DE090E00E9423745D
:1058B0008AE090E00E9423740C943C35E2EDFAE01B
:1058C00084918F01882351F0082E000C990B0E94BF
:1058D00023740F5F1F4FF8018491F4CF20E030E074
:1058E00040E05FE36091D1037091D2038091D303D4
:1058F0009091D403D0CFEDECFAE084918F0188230E
:1059000051F0082E000C990B0E9423740F5F1F4F5B
:10591000F8018491F4CF6091CF037091D003B1CF9F
:105920002091CD033091CE0344E6429FC001439FB6
:10593000900D11246FEF70E00E9477CC8B016536DB
:10594000710510F004E610E0E8ECFAE084917F01C4
:10595000882359F0082E000C990B0E942374FFEF46
:10596000EF1AFF0AF7018491F3CFB80180E090E0CD
:10597000F1C5E4ECFAE084918F01882351F0082E00
:10598000000C990B0E9423740F5F1F4FF801849144
:10599000F4CF80E290E00E942374E0ECFAE084917E
:1059A0008F01882351F0082E000C990B0E9423745C
:1059B0000F5F1F4FF8018491F4CF6091BD03709188
:1059C000BE038091BF039091C0030E9493B580E213
:1059D00090E00E942374ECEBFAE084918F0188231D
:1059E00051F0082E000C990B0E9423740F5F1F4F7B
:1059F000F8018491F4CF6091C1037091C20380914A
:105A0000C3039091C4030E9493B580E290E00E948A
:105A10002374E8EBFAE084918F01882351F0082E7B
:105A2000000C990B0E9423740F5F1F4FF8018491A3
:105A3000F4CF6091C5037091C6038091C703909124
:105A4000C8030E9493B580E290E051C48091890F11
:105A5000882309F450C0E3EBFAE084918F01882396
:105A600051F0082E000C990B0E9423740F5F1F4FFA
:105A7000F8018491F4CF80918A0F882359F18091A5
:105A80005511882329F18091FF1190910012A09166
:105A90000112B09102120097A105B105C1F0BC013D
:105AA000CD016D597F4F8F4F9F4F24E630E040E08E
:105AB00050E00E9452C960910312709104128091CB
:105AC0000512909106120E9452C9822F01C080E0F7
:105AD00090E0E6CEEFEAFAE084918F01882309F4A2
:105AE000E3CE082E000C990B0E9423740F5F1F4F0A
:105AF000F8018491F3CFE7EAFAE084918F018823DB
:105B000009F4D2CE082E000C990B0E9423740F5F6B
:105B10001F4FF8018491F3CFE2EAFAE084918F01FC
:105B2000882351F0082E000C990B0E9423740F5FFC
:105B30001F4FF8018491F4CF80919B1390919C1397
:105B4000A0919D13B0919E13892B8A2B8B2B09F466
:105B500077C00E94F2B2A50194010E9452C9690166
:105B60007A0160919B1370919C1380919D13909189
:105B70009E13A50194010E9452C98601021B130BBA
:105B8000C8016CE370E00E9463CCCB019927EAE086
:105B9000F0E0BF010E9477CC282FCB01BF010E940B
:105BA00077CC805D8093B403205D2093B503109281
:105BB000B60384EB93E00E9492B580E290E00E94ED
:105BC0002374E0EAFAE084917F01882359F0082EDB
:105BD000000C990B0E942374FFEFEF1AFF0AF701E4
:105BE0008491F3CF80E290E00E942374C8016CE3BB
:105BF00070E00E9463CC6AE070E00E9477CC605D48
:105C00006093B403805D8093B5031092B60384EB78
:105C100093E00E9492B580E290E00E942374EEE946
:105C2000FAE084918F01882309F43ECE082E000CFF
:105C3000990B0E9423740F5F1F4FF8018491F3CFDB
:105C400080E290E00E942374E6E9FAE084918F01FB
:105C5000882309F429CE082E000C990B0E94237486
:105C60000F5F1F4FF8018491F3CF1092C5138091FD
:105C7000090180FF11C0E2E9FAE084918F018823D5
:105C800009F412CE082E000C990B0E9423740F5FAA
:105C90001F4FF8018491F3CF83E50E942EB588232E
:105CA00041F00E9449B50E94D7CA70939A1360933D
:105CB0009913EEE8FAE084918F01882351F0082EC1
:105CC000000C990B0E9423740F5F1F4FF801849101
:105CD000F4CF8DE090E00E9423748AE090E00E946F
:105CE00023748091E313882309F4F3C080919913FE
:105CF00090919A13009741F0049709F09EC2EFE249
:105D0000F8E084918F01C1C0E6EBF8E084918F0147
:105D1000882351F0082E000C990B0E9423740F5F0A
:105D20001F4FF8018491F4CF8DE090E00E9423741E
:105D30008AE090E00E942374EFEAF8E084918F01FA
:105D4000882351F0082E000C990B0E9423740F5FDA
:105D50001F4FF8018491F4CF8DE090E00E942374EE
:105D60008AE090E00E942374E8E9F8E084918F01D2
:105D7000882351F0082E000C990B0E9423740F5FAA
:105D80001F4FF8018491F4CF8DE090E00E942374BE
:105D90008AE090E00E942374E1E8F8E084918F01AA
:105DA000882351F0082E000C990B0E9423740F5F7A
:105DB0001F4FF8018491F4CF8DE090E00E9423748E
:105DC0008AE090E00E942374EDE6F8E084918F0170
:105DD000882351F0082E000C990B0E9423740F5F4A
:105DE0001F4FF8018491F4CF8DE090E00E9423745E
:105DF0008AE090E00E942374E9E5F8E084918F0145
:105E0000882351F0082E000C990B0E9423740F5F19
:105E10001F4FF8018491F4CF8DE090E00E9423742D
:105E20008AE090E00E942374EBE4F8E084918F0113
:105E3000882351F0082E000C990B0E9423740F5FE9
:105E40001F4FF8018491F4CF8DE090E00E942374FD
:105E50008AE090E00E942374EDE3F8E084918F01E2
:105E6000882351F0082E000C990B0E9423740F5FB9
:105E70001F4FF8018491F4CF8DE090E00E942374CD
:105E80008AE090E00E942374D8C1882351F0082E44
:105E9000000C990B0E9423740F5F1F4FF80184912F
:105EA000F4CF8DE090E00E9423748AE090E00E949D
:105EB0002374E1E2F8E084918F018823E9F2082E4F
:105EC000000C990B0E9423740F5F1F4FF8018491FF
:105ED000F4CF80918A0F882309F486C181E08093F2
:105EE0000712109209121092081289ED9FE00E9489
:105EF00022908BE1E9EDFFE0DE01159601900D9215
:105F00008A95E1F78091D70F9091D80F9C838B836E
:105F100085EE92E09A83898340E050E0BE016F5F96
:105F20007F4F80E090E00E945976CE0101960E945A
:105F3000544EC0900812D0900912009199131091FC
:105F40009A13C601801B910B049720F06801F3E0BF
:105F5000CF0ED11C52E1452E58E0552E63E0662E3F
:105F600068E0762EC016D10608F467C10115110548
:105F700009F0A1C06DE87FE089ED9FE00E94EA8E04
:105F80006AE173E08DE89FE00E9405CD892B09F05E
:105F90004AC0F201849142E1E42E48E0F42E8823C5
:105FA00059F0082E000C990B0E942374FFEFEF1A92
:105FB000FF0AF7018491F3CF8DE090E00E942374F3
:105FC0008AE090E00E942374F301849133E0E32E91
:105FD00038E0F32E882359F0082E000C990B0E940C
:105FE0002374FFEFEF1AFF0AF7018491F3CF8DE0DE
:105FF00090E00E9423748AE090E00E9423744AE0BB
:1060000060E070E0CB010E949940E3EFF7E08491FB
:106010007F012FEFE21AF20A882309F4E2C00E94FE
:106020007D3DF701F4CFEFEEF7E084917F01882307
:1060300059F0082E000C990B0E942374FFEFEF1A01
:10604000FF0AF7018491F3CF8DE090E00E94237462
:106050008AE090E00E942374F10184912BEEE22EFD
:1060600027E0F22E882359F0082E000C990B0E948D
:106070002374FFEFEF1AFF0AF7018491F3CF8DE04D
:1060800090E00E9423748AE090E00E9423744AE02A
:1060900060E070E0CB010E949940E6EEF7E0849169
:1060A0007F012FEFE21AF20A882309F49AC00E94B6
:1060B0007D3DF701F4CF60E070E0C80101970E94D8
:1060C0001F7880918B0F882309F45FC0E4EEF7E01E
:1060D00084917F01882359F0082E000C990B0E94AF
:1060E0002374FFEFEF1AFF0AF7018491F3CF8DE8D5
:1060F0009FE00E9492B58DE090E00E9423748AE0B8
:1061000090E00E942374E2EEF7E084917F018823FF
:1061100059F0082E000C990B0E942374FFEFEF1A20
:10612000FF0AF7018491F3CF8AE99FE00E9492B5BC
:106130008DE090E00E9423748AE090E00E94237436
:10614000C801A0E0B0E04AE0BC01CD010E94994046
:10615000E0EEF7E084917F012FEFE21AF20A882344
:1061600021F00E947D3DF701F5CF9AE9E92E9FE0ED
:10617000F92EF70181917F01882319F00E947D3D5E
:10618000F8CF8AE00E947D3D2CC08DE89FE00E9400
:1061900092B58DE090E00E9423748AE090E00E9426
:1061A00023748AE99FE00E9492B58DE090E00E94FE
:1061B00023748AE090E00E942374C801A0E0B0E05C
:1061C0004AE0BC01CD010E9499408AE9E82E8FE0A7
:1061D000F82EF70181917F01882399F20E947D3D7D
:1061E000F8CF0F5F1F4FBECEE1EDF7E084918F0136
:1061F000882351F0082E000C990B0E9423740F5F26
:106200001F4FF8018491F4CF8DE090E00E94237439
:106210008AE090E00E942374E2ECF7E084918F0121
:10622000882309F429CE082E000C990B0E942374B0
:106230000F5F1F4FF8018491F3CFEAE8FAE08491F1
:106240008F01882309F430CB082E000C990B0E9493
:1062500023740F5F1F4FF8018491F3CF8091890F52
:10626000882339F00E948B7507C48091890F882399
:10627000E9F00E9477AF00C480919713823019F043
:10628000833609F0F9C30E946A75E6E8FAE0849162
:106290008F01882309F408CB082E000C990B0E946B
:1062A00023740F5F1F4FF8018491F3CF80919713F0
:1062B000833609F0E1C3DDCF8DE79AE00E94774E87
:1062C00080910B0F90910C0F891B8F7009F0D4C334
:1062D00080919713823009F4CFC3833609F000C44C
:1062E000CBC38DE090E00E9423748AE090E00E948E
:1062F0002374DACA80910B0F90910C0F891B8F7059
:1063000009F0BAC380919713823009F4B5C383367C
:1063100009F4B2C380915511811136C4ADC383E530
:106320000E942EB5811126C083E40E942EB58823D9
:1063300009F4A2C380910B0F90910C0F891B8F70F1
:1063400009F09AC320E030E040E251E46091C503D7
:106350007091C6038091C7039091C8030E9464C5E1
:1063600087FF08C08AE69AE09093FC0C8093FB0CB0
:106370000E94A93D0E9449B520E030E0A9010E9499
:1063800064C587FD10C00E9449B520E030E849E8A7
:1063900053E40E94B4CB18164CF00E9449B50E94F9
:1063A000D7CACB0105C080E090E002C083E191E054
:1063B0000E94C17261C383E50E942EB5882309F44F
:1063C0005BC30E9449B520E030E0A9010E9464C58A
:1063D00087FD11C00E9449B520E030E046E153E45A
:1063E0000E94B4CB18164CF00E9449B50E94D7CA3F
:1063F000362F272F04C030E001C036E920E0832F7C
:10640000922F8E36910514F08EE690E09093D00393
:106410008093CF030E949B7A2FC383E50E942EB501
:106420008823D9F00E9449B520E030E04FE753E4DB
:106430000E94C9C520E030E048EC52E40E946ACADC
:106440000E94D7CA6F3F710519F010F06FEF70E02E
:106450007093CE036093CD0327CA8FEF90E09093A3
:10646000CE038093CD0320CA80910B0F90910C0F27
:10647000891B8F7009F018CA8091890F811114CA85
:106480000E9436875F9A8091BC038E7F8093BC0305
:106490008A9A479A8091BC038D7F8093BC03809138
:1064A00008018095817080930601479A8091BC0312
:1064B0008B7F8093BC03129AF7C983E50E942EB5A7
:1064C000882319F10E9449B520E030E040E252E40F
:1064D0000E9464C587FD0FC00E9449B520E030ECE2
:1064E00049E754E40E94B4CB181644F00E9449B521
:1064F0000E94D2CA05C068E270E002C067EE73E095
:106500007093030260930202B7C2E4E6FAE084915A
:106510008F01882351F0082E000C990B0E942374E0
:106520000F5F1F4FF8018491F4CFC0900202D0900A
:1065300003020D2C000CEE08FF08F7FE0DC06DE203
:1065400082EF94E15ED566277727CB016C197D0930
:106550008E099F094AE003C04AE0C701B6010E94C4
:1065600052B5A2C980910B0F90910C0F891B8F70AF
:1065700009F082C280919713823009F47DC283367C
:1065800009F048C279C280910B0F90910C0F891BC2
:106590008F7009F089C980919713823009F484C9FA
:1065A000833609F013C380C980910B0F90910C0FB3
:1065B000891B8F7009F060C280919713823009F4B3
:1065C0005BC2833609F055C457C280910B0F90917E
:1065D0000C0F891B8F7009F04FC280919713823086
:1065E00009F44AC2833609F079C446C280910B0F80
:1065F00090910C0F891B8F7009F03EC28091971308
:10660000823009F439C2833609F09DC435C28091C5
:10661000C513811103C00E94287424C18E3271F504
:106620008091C6138E3209F0A6C080912A1188236A
:1066300009F418C1815080932A11882361F090E0F9
:1066400001974FE1489F9001499F300D1124C901E6
:106650008C50904F02C086EB9FE02BE1FC013496FA
:10666000A9EDBFE001900D922A95E1F7FC0182812E
:1066700093819093D80F8093D70FF4C08C3309F097
:106680007AC06CE173E085EC93E10E9405CD892B23
:1066900021F481E08093E313E5C06BE273E085ECC5
:1066A00093E10E9405CD892B79F4E5EAF7E0849126
:1066B0008F010F5F1F4F882321F00E947D3DF8015D
:1066C000F6CF88E997E044C062E473E085EC93E19B
:1066D0000E9405CD892B79F4E7E7F7E084918F01DB
:1066E0000F5F1F4F882321F00E947D3DF801F6CFF8
:1066F0008FE697E02DC066E573E085EC93E10E949C
:1067000005CD892B79F4E4E5F7E084918F010F5FE3
:106710001F4F882321F00E947D3DF801F6CF8FE4C2
:1067200097E016C064E673E085EC93E10E9405CD26
:10673000892BA9F4E4E3F7E084918F010F5F1F4FE9
:10674000882321F00E947D3DF801F6CF8FE297E08B
:106750009093FC0C8093FB0C0E94A93D83C062E7E0
:1067600073E085EC93E10E9405CD892B09F07AC096
:106770001092E31377C01D8218861C821B8285EE5F
:1067800092E09A8389838091DC0F811103C066EBCC
:106790007FE002C065ED7FE06115710519F06C5F67
:1067A0007F4F02C060E070E021E045EC53E1CE0194
:1067B00005960E945894882361F18BE1FE0135967D
:1067C000A9EDBFE001900D928A95E1F72B813C8104
:1067D0003093D80F2093D70F80912A118A3008F078
:1067E0003DC091E0980F90932A11FFE18F9FC00167
:1067F0001124DC01A850B04F4BE1E9EDFFE001901E
:106800000D924A95E1F7FC01EC50F04F338322835F
:1068100025C0EDEEF8E184918F010F5F1F4F8823B3
:1068200021F00E947D3DF801F6CFE9E1F7E0849187
:106830008F010F5F1F4F882321F00E947D3DF801DB
:10684000F6CF05EC13E1F80181918F01882319F04F
:106850000E947D3DF8CF8AE00E947D3DCE010196E9
:106860000E94544E1092C5138091090180FF04C10B
:10687000E8EAF9E084918F01882309F415C8082E0D
:10688000000C990B0E9423740F5F1F4FF801849135
:10689000F3CF8FE40E942EB5811106C883E40E94D5
:1068A0002EB502C883E50E942EB5811159C08FE430
:1068B0000E942EB5882319F080E799E007C084E58F
:1068C0000E942EB5882349F088E499E09093FC0C4F
:1068D0008093FB0C0E94A93D43C083E40E942EB527
:1068E000882319F08FE199E0F1CF81E50E942EB560
:1068F000882319F087EF98E0E9CF88E40E942EB54D
:106900008823C9F0E3EFF8E084918F01882351F0E8
:10691000082E000C990B0E9423740F5F1F4FF80183
:106920008491F4CF8DE090E00E9423748AE090E09F
:106930000E94237415C08CE40E942EB5882381F038
:10694000EFEEF8E084918F01882361F3082E000CAC
:10695000990B0E9423740F5F1F4FF8018491F4CFAD
:10696000E7EBF9E084918F01882311F40C94542C07
:10697000082E000C990B0E9423740F5F1F4FF80123
:106980008491F2CF80910B0F80910C0F0C94542CBA
:1069900083E50E942EB5882309F46EC087EC98E049
:1069A0009093FC0C8093FB0C0E94A93DE7EBF9E06F
:1069B00084918F01882311F40C94542C082E000C20
:1069C000990B0E9423740F5F1F4FF8018491F2CF3F
:1069D000E2ECF8E084918F01882351F0082E000C3E
:1069E000990B0E9423740F5F1F4FF8018491F4CF1D
:1069F000EDEBF8E084918F01882311F40C94542C72
:106A0000082E000C990B0E9423740F5F1F4FF80192
:106A10008491F2CF88E50E942EB5811106C089E5E8
:106A20000E942EB5882309F4C3C088E50E942EB5C4
:106A3000882341F08EE59AE09093FC0C8093FB0C48
:106A40000E94A93D89E50E942EB5882341F088E582
:106A50009AE09093FC0C8093FB0C0E94A93D8AE580
:106A60000E942EB5882341F082E59AE09093FC0CB9
:106A70008093FB0C0E94A93D8091901390919113FB
:106A8000019664E070E00E9477CC9093911380931C
:106A9000901380918C1390918D13019690938D1388
:106AA00080938C1310929413109293130C94352BA3
:106AB00040919013509191139F012F5F3F4F30935E
:106AC00094132093931390E6949F9001959F300D1B
:106AD0001124245F3D4EE20FF31F80830C94352B6D
:106AE0000091951310919613780124E0E20EF11CA9
:106AF0006AE270E0C7010E94FACCF80124812F32CB
:106B000021F4B8016B5F7F4F03C02C3339F4B70118
:106B100085EC93E10E940ECD0C94542C1092C51379
:106B2000009719F0FC013197108280919513909194
:106B3000961340E061E004960E945AB3809155118B
:106B4000882389F0E9E7FAE084918F01882309F42A
:106B5000C8CB082E000C990B0E9423740F5F1F4FA7
:106B6000F8018491F3CFE5E7FAE084918F0188235F
:106B700009F4B7CB082E000C990B0E9423740F5F09
:106B80001F4FF8018491F3CF0E946A75E1E7FAE0A4
:106B900084918F01882311F40C94542C082E000C3E
:106BA000990B0E9423740F5F1F4FF8018491F2CF5D
:106BB0008AE50E942EB5811138CF83E40E942EB55C
:106BC000882309F459CF8EE49AE050CF86E40E94DE
:106BD0002EB5882309F44AC10E9449B50E94D7CA3C
:106BE0008B018AE49AE09093FC0C8093FB0CB1D764
:106BF00088E50E942EB5882309F450C00E9449B54B
:106C00002B013C012DEC3CEC4CE45EE30E9464C59E
:106C10009E012F5F3F4F7901181674F020E030E09D
:106C2000A901C301B2010E94B4CB18162CF41F9322
:106C30000F938FE39AE004C12DEC3CEC4CEC5DEB40
:106C4000C301B2010E9464C518167CF020E030E058
:106C500040E85FEBC301B2010E94B4CB18162CF4DC
:106C60001F930F9383E39AE0EBC01F930F93C3012D
:106C7000B2010E94D2CA7F936F9389E29AE09F93F8
:106C80008F93FF92EF920E9436C50FB6F894DEBF45
:106C90000FBECDBFCE01019637D7DFC089E50E9478
:106CA0002EB5882309F441C00E9449B52B013C014F
:106CB0002DEC3CEC4CE45EE30E9464C5FE01319691
:106CC0007F01181674F020E030E0A901C301B20181
:106CD0000E94B4CB18162CF41F930F938EE19AE008
:106CE000AFC02DEC3CEC4CEC5DEBC301B2010E945B
:106CF00064C518167CF020E030E040E85FEBC3018B
:106D0000B2010E94B4CB18162CF41F930F9382E1AA
:106D10009AE096C01F930F93C301B2010E94D2CA9A
:106D20007F936F9388E09AE0AACF8AE50E942EB500
:106D3000882309F441C00E9449B52B013C012DEC88
:106D40003CEC4CE45EE30E9464C5FE0131967F0199
:106D5000181674F020E030E0A901C301B2010E94CE
:106D6000B4CB18162CF41F930F938DEF99E068C0E5
:106D70002DEC3CEC4CEC5DEBC301B2010E9464C510
:106D800018167CF020E030E040E85FEBC301B20170
:106D90000E94B4CB18162CF41F930F9381EF99E047
:106DA0004FC01F930F93C301B2010E94D2CA7F93B9
:106DB0006F9387EE99E063CF85E40E942EB5882318
:106DC00009F44BC00E9449B52B013C012DEC3CEC71
:106DD0004CE45EE30E9464C5FE0131967F01181603
:106DE00074F020E030E0A901C301B2010E94B4CBED
:106DF00018162CF41F930F938CED99E021C02DEC05
:106E00003CEC4CEC5DEBC301B2010E9464C518166A
:106E10007CF020E030E040E85FEBC301B2010E946B
:106E2000B4CB18162CF41F930F9380ED99E008C093
:106E3000C301B2010E94D2CA7F936F9385EC99E09F
:106E40009F938F93FF92EF920E9436C50F900F9001
:106E50000F900F900F900F901DCF81EC99E09093C1
:106E6000FC0C8093FB0C75D60C94542C00E010E0C5
:106E7000B8CE20E030E040E251E46091C50370916B
:106E8000C6038091C7039091C8030E9464C587FF21
:106E900007C08AEB99E09093FC0C8093FB0C59D6C9
:106EA00082E390E09093D0038093CF030E949B7A7B
:106EB00088EC90E00E94C172E7EBF9E084918F01C9
:106EC000882311F40C94542C082E000C990B0E946A
:106ED00023740F5F1F4FF8018491F2CF20E030E060
:106EE00040E251E46091C5037091C6038091C703ED
:106EF0009091C8030E9464C587FF07C080EB99E0AA
:106F00009093FC0C8093FB0C24D680E590E090934A
:106F1000D0038093CF030E949B7A80EF90E00E9481
:106F2000C172E7EBF9E084918F01882311F40C948E
:106F3000542C082E000C990B0E9423740F5F1F4FD6
:106F4000F8018491F2CF80E090E00E94C17210922B
:106F5000D0031092CF030E949B7AECEAF9E084916F
:106F60008F01882311F40C94542C082E000C990BDB
:106F70000E9423740F5F1F4FF8018491F2CF6F9628
:106F80000FB6F894DEBF0FBECDBFDF91CF911F913A
:106F90000F91FF90EF90DF90CF90BF90AF909F90B8
:106FA0008F907F906F905F904F903F902F900895BB
:106FB00090914116E92FF0E0EB58F44F80839F5FEA
:106FC000943018F49093411602C0109241168091AB
:106FD00042168F5F8093421608958091B00A909177
:106FE000B10A981759F0E92FF0E0E05DF54F808184
:106FF0009F5F9F779093B10A90E008958FEF9FEF86
:1070000008950F931F93CF93DF93FC01A685B78557
:107010008D0100581F4FE8018881998101968F7773
:107020009927AD014E575F4FEA0128813981281712
:107030003907D1F3E80128813981A20FB31F6C937E
:10704000A685B785A058BF4F11969C938E93A689AD
:10705000B7892C9181E090E0078C02C0880F991FBE
:107060000A94E2F7822B8C9381E081A30488F5894E
:10707000E02D80818064808381E090E0DF91CF917A
:107080001F910F910895FC0181A1882329F0A48903
:10709000B5898C9186FFFBCF11A20895FC01A485D0
:1070A000B585FD01E058FF4F208131813296808106
:1070B00091812817390779F080819181A80FB91F34
:1070C0008C91208131812F5F3F4F2F773327318380
:1070D000208390E008958FEF9FEF0895DC011C96C8
:1070E000ED91FC911D97DF01A058BF4F2D913C9170
:1070F000119712968D919C9111972817390739F0A5
:107100008D919C91E80FF91F808190E008958FEF99
:107110009FEF0895FC0124853585F901E058FF4F64
:107120008081918132962081318180589F4F821BCE
:10713000930B60E870E00C9477CC0895089580E09C
:1071400090E00895CF93FC0120812B33A1F0209192
:107150004216243080F4C62FBC0180914116F0E61F
:107160008F9FC00111248658944F0E940ECD8C2F02
:107170001FDF81E001C080E0CF9108952F923F9200
:107180004F925F926F927F928F929F92AF92BF9237
:10719000CF92DF92EF92FF920F931F93CF93DF93E3
:1071A00000D000D0CDB7DEB79A8389830E94F2B2B7
:1071B000E981FA81C680D780E084F184C114D104CA
:1071C000E104F10409F0ACC22485222309F469C367
:1071D00032852150248721E0230F228745852413FF
:1071E00001C01286E981FA8124E0329FE00DF11D91
:1071F0001124C684D784E088F188E981FA81C282AB
:10720000D382E482F582DC01CB018C0D9D1DA11D92
:10721000B11D86839783A087B18784819581892B4F
:1072200009F43FC3FFB7FD83F894E981FA81228016
:1072300033802101612C712C0481158180913902E8
:107240008F3121F08F3F09F068C205C0EDE0F7E112
:1072500024912E83DAC08FE180933902EDE0F7E1CB
:1072600084918E838F3F09F458C2823009F469C03B
:1072700030F5882309F44CC0813009F0C6C0109263
:10728000800010928100809181008860809381004D
:1072900080918100816080938100E8EDF2E2E491C9
:1072A000F0E0EE0FFF1FEB57FD4D85919491EEE15D
:1072B000F3E2E491E093DE03E1E0EE8330C19E81EE
:1072C000943009F482C008F460C0953009F09DC084
:1072D00010922001109221018091210188608093F9
:1072E000210180912101816080932101E8EDF2E28A
:1072F000E491F0E0EE0FFF1FEB57FD4D8591949167
:10730000EEE1F3E2E491E093DB0395E09E8307C1B5
:1073100014BC15BC84B5826084BD85B5816085BD13
:10732000E8EDF2E2E491F0E0EE0FFF1FEB57FD4DC8
:1073300085919491EEE1F3E2E491E093DF031E8204
:10734000ABC21092B0001092B1008091B000826088
:107350008093B0008091B10081608093B100E8ED2E
:10736000F2E2E491F0E0EE0FFF1FEB57FD4D859147
:10737000949190935A0B8093590BEEE1F3E2E491D0
:10738000E0935B0BF2E0FE8387C2109290001092B4
:10739000910080919100886080939100809191008C
:1073A000816080939100E8EDF2E2E491F0E0EE0F6D
:1073B000FF1FEB57FD4D85919491EEE1F3E2E491CF
:1073C000E093DD0323E02E83AAC01092A000109268
:1073D000A1008091A10088608093A1008091A1000C
:1073E00081608093A100E8EDF2E2E491F0E0EE0F1D
:1073F000FF1FEB57FD4D85919491EEE1F3E2E4918F
:10740000E093DC0384E08E838AC0EE81E7FD85C1D2
:1074100061E08FE10E94B7B18E818D7F09F083C05A
:107420004801A12CB12C60E072E18AE790E0A5014F
:1074300094010E948ACC29833A834B835C8369013F
:107440007A01F1E0CF1AD108E108F1082FEFC21656
:10745000D104E104F10409F008F44EC060E472E4E0
:107460008FE090E0A50194010E948ACC69017A0125
:1074700081E0C81AD108E108F1089E81923009F52F
:10748000EFEFCE16D104E104F10409F008F4CBC10A
:1074900060E970ED83E090E0A50194010E948ACC40
:1074A00069017A01F1E0CF1AD108E108F1082FEF64
:1074B000C216D104E104F10411F008F041C183E0E7
:1074C00027C08FEFC816D104E104F104B9F0B0F081
:1074D00068E478EE81E090E0A50194010E948ACCF6
:1074E00069017A0191E0C91AD108E108F108EE8139
:1074F000EE2309F49AC163C181E001C082E09E815C
:10750000911106C095B5987F892B85BD7AC085E01D
:107510009091B100987F892B8093B10072C061E097
:107520008FE10E94B7B14801A12CB12C60E072E15B
:107530008AE790E0A50194010E948ACC69017A0152
:10754000E1E0CE1AD108E108F108C114D104F1E05C
:10755000EF06F10488F068E478EE81E090E0A501A0
:1075600094010E948ACC69017A0181E0C81AD1088D
:10757000E108F10883E001C081E09E81913071F45F
:1075800090918100987F892B80938100452846281F
:107590004728D9F52FEF3FEFA90168C0EE81E3300E
:1075A00071F490919100987F892B809391004528E8
:1075B0004628472851F52FEF3FEFA90179C0FE81FA
:1075C000F43071F49091A100987F892B8093A100F1
:1075D000452846284728C9F42FEF3FEFA9017AC074
:1075E0002E81253071F490912101987F892B809311
:1075F000210145284628472841F42FEF3FEFA901F4
:107600007BC045284628472869F0D801AA0FBB1F30
:1076100091010E947EC928EE33E040E050E00E94D4
:1076200052C903C02FEF3FEFA9018E81823081F153
:107630002CF4882361F08130C9F06FC09E819430B2
:1076400009F448C0ACF1953009F456C066C0C7BC17
:107650002093F0033093F1034093F2035093F3032C
:1076600080916E00826080936E0057C0D092890036
:10767000C09288002093EC033093ED034093EE0317
:107680005093EF0380916F00826080936F0045C03C
:10769000C092B30020935C0B30935D0B40935E0B64
:1076A00050935F0B8091700082608093700035C0B2
:1076B000D0929900C09298002093E8033093E90398
:1076C0004093EA035093EB038091710082608093B2
:1076D000710023C0D092A900C092A8002093E403B7
:1076E0003093E5034093E6035093E70380917200E3
:1076F00082608093720011C0D0922901C09228014B
:107700002093E0033093E1034093E2035093E303BB
:1077100080917300826080937300ED81EFBFC1C0E0
:10772000DC01CB018C199D09AE09BF09B7FDB9C0B9
:107730004698E981FA811682178210861186B1C0B7
:1077400068E478EE81E090E0A50194010E948ACC83
:1077500069017A01F1E0CF1AD108E108F1082FEFB1
:10776000C216D104E104F10441F138F164E274EF8E
:1077700080E090E0A50194010E948ACC69017A0121
:10778000F1E0CF1AD108E108F1082FEFC216D104B9
:10779000E104F10409F008F4BACE62E17AE780E08E
:1077A00090E0A50194010E948ACC69017A0181E0F0
:1077B000C81AD108E108F10819C084E0A9CE2FEF5A
:1077C000C216D104E104F10409F008F463C062E1D7
:1077D0007AE780E090E0A50194010E948ACC6901DB
:1077E0007A01F1E0CF1AD108E108F1082FEFC216B3
:1077F000D104E104F104A9F0A0F089819A81AB8160
:10780000BC812AE0B595A795979587952A95D1F7DC
:107810006C017D01F1E0CF1AD108E108F10887E0A1
:1078200077CE86E075CE82E073CEEFEFCE16D10430
:10783000E104F10469F160F162E17AE780E090E04F
:10784000A50194010E948ACC69017A0181E0C81ADD
:10785000D108E108F1089FEFC916D104E104F10451
:10786000A9F0A0F089819A81AB81BC813AE0B595FD
:10787000A795979587953A95D1F76C017D01E1E041
:10788000CE1AD108E108F10885E03CCE84E03ACE7A
:1078900083E038CE84E033CE61E08FE10E94B7B15F
:1078A000BFCD26960FB6F894DEBF0FBECDBFDF91D9
:1078B000CF911F910F91FF90EF90DF90CF90BF90ED
:1078C000AF909F908F907F906F905F904F903F9080
:1078D0002F9008950F931F93CF93DF93CDB7DEB70B
:1078E0002C970FB6F894DEBF0FBECDBFEDEBF3E0E3
:1078F00080859185A285B385448155816681778194
:10790000008111812281338109831A832B833C8377
:107910004D835E836F83788789879A87AB87BC871F
:10792000AE01475F5F4FBE016B5F7F4FCE01019697
:107930000E94C4A729EC33E0AE01475F5F4FBE0150
:107940006B5F7F4FCE0101960E943DB82C960FB61B
:10795000F894DEBF0FBECDBFDF91CF911F910F9185
:1079600008958091AC039091AD03009731F04AE007
:1079700050E060E070E00C94B8C260E070E0CB01D1
:107980000895EFDF97FD0AC0ECDF6F3F71058105B9
:10799000910509F02CF4E5DF862F089580E0089525
:1079A0008FEF08958091AC039091AD03892B31F056
:1079B000E8DF91E0811103C090E001C091E0892FE0
:1079C00008950F931F93CF938091AC039091AD03D3
:1079D000009711F1FC018F01C1912C2F2F7DA9F08F
:1079E000C53411F0C536B9F7F801108260E070E0D7
:1079F0008091AC039091AD030E9465C1F801C083F2
:107A0000562F472F382F292F0BC060E070E0CF9101
:107A10001F910F910C9465C150E040E030E020E0F0
:107A2000652F742F832F922FCF911F910F9108955F
:107A300081548A3108F042C0E82FF0E040916C1682
:107A400050916D1660916E1670916F1604C0769508
:107A50006795579547958A95D2F7842F817040FF97
:107A60002FC0EE5AF94E9081992309F1E091311619
:107A7000F0913216E90FF11D908120ED290F2A3087
:107A800098F09E3211F491810CC09D3211F09B321E
:107A900071F4918120ED290F2A3030F09E3239F4B3
:107AA000928190539A3018F42E2F9F2F02C020E01D
:107AB00090E02093AC039093AD03089580E0089587
:107AC0000895B6DF882341F081E02091AC03309126
:107AD000AD03232B09F480E00895FC0123812111DB
:107AE0000C94C58E089580E1EDEBF3E0AAEDBAE0C9
:107AF00001900D928A95E1F708959091C00095FF4D
:107B0000FCCF8093C6000895EF92FF921F93CF930E
:107B1000DF937C0160E016DB182F882399F0EDEEEF
:107B2000F8E18491EF012196882319F0E6DFFE0148
:107B3000F8CFB70181E19BE00E94074C82E2DDDFD4
:107B40008AE0DBDF812FDF91CF911F91FF90EF90D3
:107B50000895DF92EF92FF920F931F93CF93DF93DD
:107B6000CDB7DEB76E970FB6F894DEBF0FBECDBFB0
:107B70006091FB0C7091FC0C6115710541F14DE1B8
:107B800050E0CE0101967C010E940DC51E8EF701CA
:107B90008F010E191F09D190DD2019F09AE0D9123A
:107BA000F7CFF701E00FF11F1082C701ADDF882387
:107BB00071F0DD20A9F00F5F1F4F8091FB0C9091B9
:107BC000FC0C080F191F1093FC0C0093FB0C81E0B8
:107BD0002091FB0C3091FC0C232B29F480E003C096
:107BE00000E010E0F0CF6E960FB6F894DEBF0FBE47
:107BF000CDBFDF91CF911F910F91FF90EF90DF905C
:107C000008953F924F925F926F927F928F929F92D0
:107C1000AF92BF92CF92DF92EF92FF920F931F939A
:107C2000CF93DF931F92CDB7DEB793DF81116EC282
:107C300080914216843008F047C0CFD9AC0197FF3D
:107C40007CC142C08E3409F0D9C10115110509F477
:107C5000D5C164E47CE0C8010E941CC57C01892B6D
:107C600009F48EC16EE470E0C80104960E94FACC5B
:107C7000009709F485C14AE050E060E070E00196A9
:107C80000E94B8C26093F4037093F5038093F603E7
:107C90009093F70380904E1690904F16A090501638
:107CA000B09051162FEF821A920AA20AB20A6815F2
:107CB00079058A059B0509F465C1EF2809F062C1C1
:107CC00081E19CE00E94FCB48091890F882309F433
:107CD0001DC280914216811102C010925A04EE24F6
:107CE000E394409103125091041260910512709137
:107CF00006128091FF1190910012A0910112B09193
:107D00000212481759076A077B0708F4E12C00E0C4
:107D100010E09924939480E6882E99E4A92E9CE0A3
:107D2000B92E2DE8322E80914216843008F0EEC133
:107D3000E110ECC180915A048111E8C180915A117F
:107D400090915B11A0915C11B0915D118093031231
:107D500090930412A0930512B093061241E050E0F4
:107D6000BE016F5F7F4F82E591E10E944C910197C8
:107D700019F4898190E002C08FEF9FEFF82E4090B8
:107D800003125090041260900512709006124091F8
:107D9000FF11509100126091011270910212EE24B5
:107DA000E394441655066606770608F4E12C44165B
:107DB000550666067706B0F4019609F46AC08AE0B3
:107DC000F81609F489C09DE0F91609F485C023E28C
:107DD000F21619F08AE3F81296C0809159048111C5
:107DE00092C06FC00E94DD6682E591E10E94C58E5F
:107DF00080916D11882359F1815080936D11389EC7
:107E0000C001112441E061E08E589E4E0E945AB399
:107E1000E0916D1194E0E99FF0011124E259FE4ECA
:107E20004081518162817381409303125093041207
:107E3000609305127093061282E591E10E94DB8D3A
:107E400080918A0F8823A9F09092890F12C0109216
:107E5000890F0E946FA30E94CA7C0E94597C6D33D7
:107E600071058105910528F0B092FC0CA092FB0CE5
:107E700070DE8091890F811128C0ECE5FCE08491CF
:107E80006F012FEFC21AD20A8823D9F036DEF6012D
:107E9000F6CFE8EDF8E184916F019FEFC91AD90A96
:107EA000882319F02ADEF601F6CFEDE4FCE0849198
:107EB0006F012FEFC21AD20A882319F01EDEF601D5
:107EC000F6CF83E2F81208C005C023E2F2121BC10C
:107ED00000E010E090925A04109259040115110527
:107EE00019F40E949F7F0CC080914116889E000D5E
:107EF000111D1124F801E658F44F108280E058D883
:107F000000E010E010CF0F35110508F00CCF9BE317
:107F1000F91202C09092590480915904811103CF43
:107F200080914116F801889EE00DF11D1124E6585C
:107F3000F44FF0820F5F1F4FF6CE982F20914C1612
:107F400030914D168A3019F09D3009F0AAC0109278
:107F500058042115310519F40E949F7F69CEF9015B
:107F6000E850FC4F108210924D1610924C1608EFFC
:107F700013E0F8018191803209F064CE8F01F9CFCE
:107F8000C80179CE6AE270E0C8010E9432CD9C013E
:107F9000009701F1982F901BF12C992339F0915003
:107FA000F801E90FF11D8081F826F7CF4AE050E093
:107FB00060E070E0C90101960E94B8C2CF2CD12CBC
:107FC000E12CF12C6C157D058E059F0531F082EFBB
:107FD0009BE078CE88EC9BE075CE8091F403909185
:107FE000F503A091F603B091F70380934E1690939A
:107FF0004F16A0935016B09351160EC08091870F64
:10800000882351F069E773E0C8010E9405CD892BF0
:1080100019F08EE99BE056CE8091410281111FC07C
:1080200067E470E0C8010E94FACC0097C1F04AE012
:1080300050E060E070E001960E94B8C264307105C3
:108040008105910560F4E7E2FBE084917F019FEFF9
:10805000E91AF90A882319F050DDF701F6CF6DE728
:1080600073E0C8010E9405CD892B11F410924002E3
:1080700062E873E0C8010E9405CD892B21F48EE1EE
:108080009BE00E94774E67E873E0C8010E9405CD2F
:10809000892B11F40E94368761E088EF93E052D873
:1080A000C7CD2F3531050CF0C3CD9C35C1F40E94EE
:1080B000ED3797FDBDCD209158042111B9CD209108
:1080C0004C1630914D16A9014F5F5F4F50934D16DE
:1080D00040934C16F901E850FC4F8083A9CD9B33A7
:1080E00019F481E080935804809158048111A0CD47
:1080F000C901019690934D1680934C16F901E850F2
:10810000FC4F408395CD10925904EBCE0F90DF9138
:10811000CF911F910F91FF90EF90DF90CF90BF9084
:10812000AF909F908F907F906F905F904F903F9017
:1081300008958F929F92AF92BF92EF92FF920F930A
:108140001F93CF93DF93CDB7DEB7A0970FB6F89408
:10815000DEBF0FBECDBF611571058105910589F1A7
:1081600000E0842E912CA12CB12C102FEE24E3944E
:10817000F12CEC0EFD1EE00EF11C07FDFA94A5019A
:1081800094010E9452C9F7016083B901CA010F5FCF
:10819000611571058105910541F71F3F21F1E1E06E
:1081A000F0E0EC0FFD1FE10FF11D17FDFA95808146
:1081B0008A3010F097E301C090E3890F9EDC1150E4
:1081C000ECCF80E3A0960FB6F894DEBF0FBECDBF14
:1081D000DF91CF911F910F91FF90EF90BF90AF90E3
:1081E0009F908F908ACCA0960FB6F894DEBF0FBEFA
:1081F000CDBFDF91CF911F910F91FF90EF90BF9076
:10820000AF909F908F900895CF92DF92EF92FF9260
:108210006B017C0197FF0AC08DE26FDCF094E09463
:10822000D094C094C11CD11CE11CF11C4AE0C701D0
:10823000B601FF90EF90DF90CF907BCF8F929F920F
:10824000AF92BF92CF92DF92EF92FF92CF936B01EA
:108250007C01B42E20E030E0A9010E9464C587FFB4
:1082600006C08DE24ADCF7FAF094F7F8F094C0E02B
:1082700060E070E080E09FE3CB1541F02DEC3CEC3A
:108280004CEC5DE30E94C9C5CF5FF6CF9B01AC010A
:10829000C701B6010E948EC96B017C010E94D7CA3A
:1082A0004B015C014AE045DFCC2379F1C501B40103
:1082B0000E9468C59B01AC01C701B6010E948DC92F
:1082C0006B017C018EE219DC20E030E040E251E4F9
:1082D000C701B6010E94C9C54B015C010E94D2CA08
:1082E0006B01770FEE08FF08C701B6018DDFC701EC
:1082F000B6010E946AC59B01AC01C501B4010E9490
:108300008DC96B017C01C150F9F6CF91FF90EF90C0
:10831000DF90CF90BF90AF909F908F9008951F9265
:108320000F920FB60F9211240BB60F922F938F93CB
:108330009F93EF93FF932091B10AE091B00A81E0FF
:108340008E0F8F779091C600281729F0F0E0E05D3E
:10835000F54F9083E82FE093B00AFF91EF919F9142
:108360008F912F910F900BBE0F900FBE0F901F900B
:1083700018959C0197FD0EC08436910584F064E643
:1083800070E00E9477CCCB016AE070E00E9477CC6D
:10839000805D06C03195219531098DE201C080E2F2
:1083A0008093B8032A30310564F0EAE0F0E0C901B7
:1083B000BF010E9477CCCB01BF010E9477CC805DCA
:1083C00001C080E28093B903C9016AE070E00E94B5
:1083D00077CC805D8093BA0388EB93E008951F9279
:1083E0000F920FB60F9211240BB60F922F933F935B
:1083F0008F939F93EF93FF9320916A1430916B14A6
:1084000080916C1490916D142817390731F4809184
:1084100031018F7D8093310114C0E0916C14F09193
:108420006D14E651FC4E208180916C1490916D1476
:1084300001968F77992790936D1480936C142093F5
:108440003601FF91EF919F918F913F912F910F9066
:108450000BBE0F900FBE0F901F9018951F920F929A
:108460000FB60F9211240BB60F922F934F935F9379
:108470008F939F93EF93FF938091300182FD1CC0F7
:10848000209136018091EE149091EF144091F014F8
:108490005091F11401968F7799274817590771F079
:1084A000E091EE14F091EF14E259FB4E208390938B
:1084B000EF148093EE1402C080913601FF91EF918A
:1084C0009F918F915F914F912F910F900BBE0F90C5
:1084D0000FBE0F901F90189580910B0F90910C0F6D
:1084E000891B8F7019F480E090E008959091080F37
:1084F000992351F0833030F48FEF890F19F0809376
:10850000080FF1CF1092080FE0910C0F88E5E89F5B
:10851000F0011124E55AFB4F808180FDE4CF80916A
:108520000C0F8F5F8F708093090F90910C0F8091CB
:108530000A0F981304C08091090F80930A0FCF018E
:1085400008950F930FB70F9300916E000F930B7F59
:1085500000936E0000916F000D7F00936F000F93EA
:108560000BB70F930CB70F921F922F933F934F931C
:108570005F936F937F938F939F93AF93BF93EF938B
:10858000FF9311244AD0FF91EF91BF91AF919F913A
:108590008F917F916F915F914F913F912F911F909C
:1085A0000F900CBF0F910BBF0F910260F8940093D6
:1085B0006F000F9100936E000F910FBF0F911895F0
:1085C0008091E00980FF03C0899A8FEF02C08998EB
:1085D00081E0809310028091E00981FF03C08F98B1
:1085E0008FEF02C08F9A81E0809311028091E009A1
:1085F00082FF08C080910B0182708093090143982B
:108600008FEF08C080910B018095827080930901E3
:10861000439A81E08093120208952F923F924F92E5
:108620005F926F927F928F929F92AF92BF92CF9202
:10863000DF92EF92FF920F931F93CF93DF93CDB70B
:10864000DEB72D970FB6F894DEBF0FBECDBFF894FE
:108650008FEF9FEF90938900809388002AE029870D
:10866000212C312C44244A94542C3201789480914A
:108670002C0A90912D0AA0912E0AB0912F0A892BD5
:108680008A2B8B2B09F010C2809118158823E1F0FA
:10869000109218158091161590911715892B09F4D1
:1086A00003C21092E10910921715109216159091BD
:1086B0000B0F80910C0F981709F4F6C180910C0FE5
:1086C0008F5F8F7080930C0F809116159091171506
:1086D000892B09F4E9C1C090280AD090290AE090BA
:1086E0002A0AF0902B0A4091240A5091250A6091A1
:1086F000260A7091270A0091170A10E020E030E066
:10870000DB01CA018C199D09AE09BF0908171907B9
:108710002A073B0710F4D901C801482F8C0D9D1D75
:10872000AE1DBF1D8093280A9093290AA0932A0AA0
:10873000B0932B0A2091840030918500245E3F4F36
:10874000C090FD09D090FE09E090FF09F090000A6A
:108750008091ED099091EE09A091EF09B091F00997
:108760008C0D9D1DAE1DBF1D8093FD099093FE09CC
:10877000A093FF09B093000AB7FD1CC0889AC0906F
:108780002515D0902615E0902715F090281580919A
:108790001002082E000C990BAA0BBB0B8C0D9D1D13
:1087A000AE1DBF1D8093251590932615A093271508
:1087B000B0932815C090010AD090020AE090030AF5
:1087C000F090040A8091F1099091F209A091F309C7
:1087D000B091F4098C0D9D1DAE1DBF1D8093010A43
:1087E0009093020AA093030AB093040AB7FD1CC039
:1087F0008E9AC0902915D0902A15E0902B15F090F4
:108800002C1580911102082E000C990BAA0BBB0BA2
:108810008C0D9D1DAE1DBF1D8093291590932A15AB
:10882000A0932B15B0932C15C090050AD090060A82
:10883000E090070AF090080A8091F5099091F609F6
:10884000A091F709B091F8098C0D9D1DAE1DBF1DBB
:108850008093050A9093060AA093070AB093080A2A
:10886000B7FD3EC09091DF09809112029923C1F0BB
:108870009091DD0992FF02C087FD05C09091DC094F
:10888000992309F4BEC56091DD097091DE0973FF7B
:1088900002C087FD0CC09091DB09911108C006C091
:1088A00090910B019095987090930901419AC09016
:1088B0002D15D0902E15E0902F15F0903015082E24
:1088C000000C990BAA0BBB0B8C0D9D1DAE1DBF1D83
:1088D00080932D1590932E15A0932F15B0933015DE
:1088E000C090090AD0900A0AE0900B0AF0900C0A96
:1088F0008091F9099091FA09A091FB09B091FC09C6
:108900008C0D9D1DAE1DBF1D8093090A90930A0A10
:10891000A0930B0AB0930C0AB7FD3AC080903115B2
:1089200090903215A0903315B0903415C09013027A
:108930000C2C000CDD08EE08FF08C80CD91CEA1C42
:10894000FB1CC0923115D0923215E0923315F09293
:108950003415C090E909D090EA09E090EB09F09055
:10896000EC098C199D09AE09BF098093090A9093FF
:108970000A0AA0930B0AB0930C0A9091E009809127
:10898000150A93FF02C0815001C08F5F8093150AC2
:108990008091FD099091FE09A091FF09B091000A14
:1089A000B7FD15C0C090E909D090EA09E090EB0945
:1089B000F090EC098C199D09AE09BF098093FD095F
:1089C0009093FE09A093FF09B093000A88988091C4
:1089D000010A9091020AA091030AB091040AB7FD1E
:1089E00015C0C090E909D090EA09E090EB09F09039
:1089F000EC098C199D09AE09BF098093010A909377
:108A0000020AA093030AB093040A8E988091050A83
:108A10009091060AA091070AB091080AB7FD3AC0E2
:108A2000C090E909D090EA09E090EB09F090EC09D8
:108A30008C199D09AE09BF098093050A9093060A17
:108A4000A093070AB093080A8091DF098823E1F018
:108A50008091DD0982FF04C08091120287FD05C06C
:108A60008091DC09882309F4D3C48091DD099091B9
:108A7000DE0993FF04C08091120287FD0BC0809134
:108A8000DB09811107C005C080910B0188708093BC
:108A900009014198415041F08091840090918500F6
:108AA00082179307C8F34CCE80911D0290911E024D
:108AB000A0911F02B0912002892B8A2B8B2B09F0E9
:108AC0008AC08091160A882309F452C08090280A2F
:108AD0009090290AA0902A0AB0902B0AC090110AFF
:108AE000D090120AE090130AF090140A8091150AAF
:108AF000C814D904EA04FB0488F42091E2093091F7
:108B0000E3094091E6095091E7094217530730F411
:108B100081508093150A2150310915C08C149D0491
:108B2000AE04BF04E8F42091E2093091E3094091DA
:108B3000E4095091E5092417350790F48F5F80937D
:108B4000150A2F5F3F4F3093E3092093E2094091CC
:108B5000190250911A0260911B0270911C020BC005
:108B60004092190250921A0260921B0270921C02EB
:108B70004FEF5FEFBA018091150A87FD02C0169A88
:108B800001C016982091840030918500245E3F4FEB
:108B90008091150A8823B9F0149A8091150A87FFED
:108BA00002C08F5F01C081508093150A1498809194
:108BB000150A882369F380918400909185008217BB
:108BC0009307C8F3E5CF40931D0250931E026093B4
:108BD0001F027093200280912C0A90912D0AA0917F
:108BE0002E0AB0912F0A892B8A2B8B2B09F08FC369
:108BF000A0911615B0911715109709F4AEC5C09045
:108C0000280AD090290AE0902A0AF0902B0A409175
:108C1000240A5091250A6091260A7091270AC416E9
:108C2000D506E606F706D0F01092E1091092171566
:108C30001092161590910B0F80910C0F981709F454
:108C40008CC580910C0F8F5F8F7080930C0F00ED9F
:108C5000802E07E0902EA12CB12C8AC14091200AD1
:108C60005091210A6091220A7091230A4C155D05EA
:108C70006E057F0508F46DC040911C0A50911D0AD5
:108C800060911E0A70911F0AD2960D911D912D912F
:108C90003C91D597EE27419FF12D529FC001629FD5
:108CA000900D619F800D911D429FF00D811D9E1FB3
:108CB000519FF00D811D9E1F609FF00D811D9E1F15
:108CC000509FF10D8E1F9E1FF6958E1F9E1F349F85
:108CD000800D911D359F900D1124FD01EA5BFF4F22
:108CE0000081118122813381080F191F211D311D3F
:108CF0000093180A1093190A20931A0A30931B0A3A
:108D00003497C080D180E280F380C016D106E2069D
:108D1000F30640F4C092180AD092190AE0921A0A97
:108D2000F0921B0AC090180AD090190AE0901A0A13
:108D3000F0901B0A80E794E121E0FC01859095907A
:108D4000A590B4908C149D04AE04BF0408F466C3CF
:108D500070C32091110A3091120A4091130A509168
:108D6000140A29833A834B835C832C153D054E05F9
:108D70005F0508F070C040910D0A50910E0A609195
:108D80000F0A7091100A4A875B876C877D87D2969D
:108D90000D911D912D913C91D597EE27419FF12D7D
:108DA000529FC001629F900D619F800D911D429F57
:108DB000F00D811D9E1F519FF00D811D9E1F609F14
:108DC000F00D811D9E1F509FF10D8E1F9E1FF69569
:108DD0008E1F9E1F349F800D911D359F900D112475
:108DE0008C0120E030E08090180A9090190AA09041
:108DF0001A0AB0901B0AFD01E65BFF4F0815190522
:108E00002A053B05A0F440815181628173814D8325
:108E10005E836F837887801A910AA20AB30A841648
:108E20009506A606B70638F44A015B0104C08080A7
:108E30009180A280B38080E794E151E05D83FC01E2
:108E40000591159125913491081519052A053B05C1
:108E500008F473C380C38091150A8823D9F0D8968B
:108E60004D915C91D99760E070E0009119021091EA
:108E70001A0220911B0230911C0240175107620711
:108E8000730741F010921D0210921E0210921F02F1
:108E90001092200240911502509116026091170223
:108EA0007091180277FF5CC0AE5BBF4F8D919D91B2
:108EB0000D90BC91A02D20E734E141E0F901C5906F
:108EC000D590E590F490C816D906EA06FB0658F44A
:108ED000B695A79597958795440F2C5F3F4F74E102
:108EE0002C38370759F74093170A80329105A105AE
:108EF000B10520F480E290E0A0E0B0E08097A10905
:108F0000B109811538E09307A105B10508F4DFC365
:108F100044E0949F9001112420593F4EF90132966C
:108F200045915491EE27859FB001849F610D7E1F6E
:108F300006946E1F7E1F1124CB01A0E0B0E0F90162
:108F40004591549160E070E0481B590B6A0B7B0B14
:108F50004093150250931602609317027093180203
:108F60008090150290901602A0901702B0901802FF
:108F70008091161590911715892B09F0C0C1ACDAB4
:108F80009093171580931615892B09F4B8C1E091B9
:108F90001615F0911715808183FF3EC0858996894B
:108FA000A789B08D8093251590932615A09327153A
:108FB000B0932815818D928DA38DB48D8093291542
:108FC00090932A15A0932B15B0932C15858D968D13
:108FD000A78DB0A180932D1590932E15A0932F15DA
:108FE000B093301581A192A1A3A1B4A180933115B2
:108FF00090933215A0933315B093341590910B0FC5
:1090000080910C0F981709F4BACF80910C0F8F5FE5
:109010008F7080930C0FB3CFC588D688E788F08C0B
:1090200081E0C114D104E104F10409F480E0018D70
:10903000128D238D348D011511052105310509F09F
:109040008260458D568D678D70A141155105610572
:10905000710509F084608093E10910920D0A109265
:109060000E0A10920F0A1092100A10921C0A109207
:109070001D0A10921E0A10921F0A85A196A1A7A18F
:10908000B0A58093240A9093250AA093260AB09352
:10909000270A882499245401881A990AAA0ABB0A23
:1090A0008092090A90920A0AA0920B0AB0920C0AC6
:1090B0008092050A9092060AA092070AB092080AC6
:1090C0008092010A9092020AA092030AB092040AC6
:1090D0008092FD099092FE09A092FF09B092000AC9
:1090E000CC0CDD1CEE1CFF1CC092ED09D092EE09E9
:1090F000E092EF09F092F009000F111F221F331FB9
:109100000093F1091093F2092093F3093093F409C5
:10911000440F551F661F771F4093F5095093F609BA
:109120006093F7097093F80941A152A163A174A15A
:10913000440F551F661F771F4093F9095093FA0992
:109140006093FB097093FC09880F991FAA1FBB1F2E
:109150008093E9099093EA09A093EB09B093EC0995
:109160001092280A1092290A10922A0A10922B0AA9
:1091700082A593A5A4A5B5A58093200A9093210A62
:10918000A093220AB093230A86A597A5A0A9B1A906
:109190008093110A9093120AA093130AB093140AB1
:1091A00081A58093E80997A99093160A992309F15C
:1091B00024AD35AD3093E7092093E60922AD33ADF8
:1091C0003093E5092093E40910921D0210921E02CB
:1091D00010921F021092200240AD51AD60E070E08D
:1091E0004093190250931A0260931B0270931C0261
:1091F00008C04092190250921A0260921B027092AB
:109200001C0296A92091E00992130AC02091140231
:1092100030E0482F082E000C550B4217530729F059
:109220009093E00980931402CBD98091680B81114F
:109230000E94C1A840921502509216026092170235
:1092400070921802E0911615F0911715EA5BFF4F26
:1092500080819181A281B3818093180A9093190A29
:10926000A0931A0AB0931B0A20E734E141E0F90108
:10927000C590D590E590F490C816D906EA06FB068D
:1092800060F4B695A79597958795440F2C5F3F4F4F
:10929000ECE8F4E1E217F30751F74093170A803244
:1092A0009105A105B10520F480E290E0A0E0B0E0D6
:1092B0008097A109B109811558E09507A105B1056D
:1092C00008F428C264E0969F9001112420593F4E73
:1092D000F901329645915491EE27859FB001849F04
:1092E000610D7E1F06946E1F7E1F1124F90185906B
:1092F0009490A12CB12C861A970AA108B1088092EB
:109300002C0A90922D0AA0922E0AB0922F0A009158
:109310002C0A10912D0A20912E0A30912F0A40918B
:109320001D0250911E0260911F0270912002F02ECA
:109330001983F22FE32F401751076207730720F4B8
:10934000F42E5983F62FE72F8F2D9981AF2FBE2F43
:109350000097E1E0AE07B10520F08FEF9FEFA0E0AE
:10936000B0E0081B190B2A0B3B0B00932C0A10933F
:109370002D0A20932E0A30932F0A4F3FFFEF5F07ED
:109380006F077F0761F0481B590B6A0B7B0B4093FB
:109390001D0250931E0260931F0270932002F894E6
:1093A0002091840030918500205F3F4F49854150D6
:1093B0004987442339F0280E391E2216330608F453
:1093C00055C901C019013092890020928800789413
:1093D0002D960FB6F894DEBF0FBECDBFDF91CF91B3
:1093E0001F910F91FF90EF90DF90CF90BF90AF90C3
:1093F0009F908F907F906F905F904F903F902F90B5
:10940000089590910B0190959870909309013BCA33
:1094100080910B0188708093090127CBF694E79423
:10942000D794C794220F0496E4E18C389E0709F084
:1094300084CC2093170AF0E2CF16D104E104F104A2
:1094400028F410E2C12ED12CE12CF12C30E2C31A09
:10945000D108E108F108C11488E0D806E104F1045C
:10946000F8F0E4E0DE9EC001112480599F4EFC011B
:10947000329625913491FC2DEE27F39F8001F29FC7
:10948000010D1E1F06940E1F1E1F1124FC01859046
:109490009490A12CB12C801A910AA108B10822C085
:1094A000970186013695279517950795F801EC7F6A
:1094B0009F012059334FF90185909490F90132961C
:1094C00085919491EC2DE770E89F9001E99F300D14
:1094D0001124F3E036952795FA95E1F7821A930A5D
:1094E000A12CB12C480D591D6A1D7B1D40931C0AEF
:1094F00050931D0A60931E0A70931F0A9091160ADA
:109500008091150A992309F474C0882309F430CD99
:10951000D8968D919C91D997A0E0B0E04091190226
:1095200050911A0260911B0270911C0284179507DA
:10953000A607B70709F060C01BCDB694A79497940F
:1095400087944D81440F4D8304966CE874E168174D
:10955000790709F074CC2D812093170A30E2831625
:109560009104A104B10428F450E2852E912CA12C81
:10957000B12C60E2861A9108A108B108811478E044
:109580009706A104B10408F440C0E4E09E9EC00127
:10959000112480599F4EFC01329625913491F82D6B
:1095A000EE27F39F8001F29F010D1E1F06940E1FF0
:1095B0001E1F1124FC0185909490A12CB12C801ABF
:1095C000910AA108B1084A855B856C857D85480DA7
:1095D000591D6A1D7B1D40930D0A50930E0A60931E
:1095E0000F0A7093100A8091160A811132C080917F
:1095F000150A882309F4BCCC10921D0210921E0299
:1096000010921F0210922002B3CC9501840136956E
:10961000279517950795F801EC7F9F012059334F47
:10962000F90185919491F901329605911491E82DF3
:10963000E770E09F9001E19F300D112443E03695E3
:1096400027954A95E1F74C01821A930AA12CB12C77
:10965000BACF49815A816B817C812D81420F511D86
:10966000611D711D4C155D056E057F05C8F4809167
:10967000150A882309F47CCCD8964D915C91D99732
:1096800060E070E00091190210911A0220911B0213
:1096900030911C02401751076207730709F468CC28
:1096A00010921D0210921E0210921F0210922002B0
:1096B000D8968D919C91D997A0E0B0E08093190243
:1096C00090931A02A0931B02B0931C0251CCAC01E0
:1096D000BD017695679557954795FA01EC7F9F01F7
:1096E0002059334FF90145915491F9013296659112
:1096F00074918770869F9001879F300D1124C90156
:10970000F3E096958795FA95E1F7481B590B60E0D1
:1097100070E01ECCAC01BD017695679557954795D5
:10972000FA01EC7F9F012059334FF9018590949005
:10973000F9013296459154918770849F9001859FDD
:10974000300D1124C901A3E096958795AA95E1F7FC
:10975000881A990AA12CB12CD2CD80ED882E87E0F1
:10976000982EA12CB12C0BCCCF92DF92EF92FF92CE
:10977000CF93DF936A017B01FC018491EF01219675
:10978000882321F00E947D3DFE01F7CF4AE0C7010A
:10979000B601DF91CF91FF90EF90DF90CF900C94C6
:1097A0009940CF92DF92EF92FF92CF93DF936A01BD
:1097B0007B01FC018491EF012196882321F00E9416
:1097C0007D3DFE01F7CF42E0C701B601DF91CF91A9
:1097D000FF90EF90DF90CF900C941E410F931F935A
:1097E000CF93DF938B01FC018491EF0121968823B5
:1097F00021F00E947D3DFE01F7CFB801110F880BCB
:10980000990BDF91CF911F910F910C9404410F930D
:109810001F93CF93DF938B01FC018491EF0121967D
:10982000882321F00E947D3DFE01F7CFE801899158
:10983000882319F00E947D3DFACFDF91CF911F91CF
:109840000F9108950F931F93CF93DF9300D01F9232
:10985000CDB7DEB78C0108960E944AA769837A8348
:109860008B839C83B8016C5F7F4FAE014F5F5F4F6E
:10987000C8010E94E9A59B01AC01F80160857185D2
:10988000828593850E948DC9F801608771878287E0
:1098900093870F900F900F900F90DF91CF911F91B2
:1098A0000F91089586E40E94183D809356158823F1
:1098B00051F00E94E13C60930C0270930D02809382
:1098C0000E0290930F0283E50E94183D882351F009
:1098D0000E94E13C609308027093090280930A029F
:1098E00090930B0282E40E94183D882351F00E945D
:1098F000E13C60930402709305028093060290930A
:10990000070208958FEF8EBD0DB407FEFDCF8EB513
:109910000895CF92DF92EF92FF92CF93DF93EC0105
:10992000C090EA0AD090EB0AE090EC0AF090ED0AC1
:10993000A7019601688179818A819B810E9464C513
:1099400087FF04C0C882D982EA82FB82C090EE0AF7
:10995000D090EF0AE090F00AF090F10AA70196018A
:109960006C817D818E819F810E9464C587FF04C0C8
:10997000CC82DD82EE82FF82C0902702D090280246
:10998000E0902902F0902A02A7019601688179816E
:109990008A819B810E94B4CB181624F4C882D98294
:1099A000EA82FB82C0902B02D0902C02E0902D0224
:1099B000F0902E02A70196016C817D818E819F819E
:1099C0000E94B4CB181624F4CC82DD82EE82FF8292
:1099D000C090F20AD090F30AE090F40AF090F50AF1
:1099E000A7019601688579858A859B850E9464C553
:1099F00087FF04C0C886D986EA86FB86C0902F02FE
:109A0000D0903002E0903102F0903202A70196012E
:109A1000688579858A859B850E94B4CB181624F4C5
:109A2000C886D986EA86FB86DF91CF91FF90EF90BA
:109A3000DF90CF9008954F925F926F927F928F92B6
:109A40009F92AF92BF92CF92DF92EF92FF920F93CD
:109A50001F93CF93DF93D82EC82FD0E0FE01EC5098
:109A6000FA4EC49082E0D81203C081E08093DF09EF
:109A70007E01EE0CFF1CEE0CFF1CF701E851FA4EC4
:109A800045905590659074906C2D0C2C000C770BC4
:109A9000880B990B0E946AC54B015C0120E030E005
:109AA00040EC5FE3C301B2010E94C9C5A501940166
:109AB0000E94C9C5AB01BC0100E010E098018D2DEA
:109AC0000E946E98F701E452FA4E25913591459126
:109AD0005491C501B4010E94C9C54B015C0120E04D
:109AE00030E0A9010E9464C5882309F448C000E061
:109AF00010E09801B501A40170588D2D0E946E9858
:109B0000FE01E752FA4EC491C11117C0EDEEF8E123
:109B10008491EF012196882321F00E947D3DFE0172
:109B2000F7CFE7EBF5E18491EF012196882321F04F
:109B30000E947D3DFE01F7CFCAE0F701E256FC4DE1
:109B400045905590659074906C2F70E080E090E0A7
:109B50000E946AC59B01AC01C301B2010E946ACA9E
:109B60002B013C01A5019401C501B4010E948EC9DD
:109B7000AB01BC01930182018D2D0E946E9882E0A1
:109B8000D81249C04090BB155090BC156090BD15CF
:109B90007090BE1520E030E0A901C301B2010E941F
:109BA000B4CB5301420187FF04C0B7FAB094B7F8B1
:109BB000B09420E030E0A901C501B4010E9464C561
:109BC000882349F120E030E0A901C301B2011C144F
:109BD0002CF40E94B4CB18162CF008C00E9464C567
:109BE00087FF04C081E08093DC0903C081E080939B
:109BF000DB091C1424F4B7FAB094B7F8B09400E071
:109C000010E09801B501A40182E00E946E981092C4
:109C1000DC091092DB091092DF0981E090E00D2C45
:109C200001C0880F0A94EAF79091BC03982B909397
:109C3000BC039091D90A892B8093D90AF701E35389
:109C4000F54F10821182128213828D2D0E94CE9ABE
:109C5000F701E555FA4E85919591A591B491E701EB
:109C6000C354DC4F88839983AA83BB830E946A3CD8
:109C7000F701E652F54F88819981AA81BB818083E3
:109C80009183A283B383DF91CF911F910F91FF90B6
:109C9000EF90DF90CF90BF90AF909F908F907F908C
:109CA0006F905F904F90089525EE32E0FC01318374
:109CB000208304960C946D3D5F9A8091BC038E7F47
:109CC0008093BC038A9A479A8091BC038D7F8093CE
:109CD000BC03809108018095817080930601479AAA
:109CE0008091BC038B7F8093BC03129A0895E8EDAA
:109CF000F8E18491EF012196882321F00E947D3DB7
:109D0000FE01F7CFEBE8F5E18491EF01219688237E
:109D100021F00E947D3DFE01F7CF0E94DF7CCCDF69
:109D2000E7E8F5E18491EF01882349F0082E000C63
:109D3000990B0E9423742196FE018491F5CF8DE04A
:109D400090E00E9423748AE090E00E942374FFEF69
:109D50002BE48DE1F15020408040E1F700C000008D
:109D6000F8949FEFE4E3FCE09150E040F040E1F72D
:109D700000C000000E94DF7CA895FECF2F923F928A
:109D80004F925F926F927F928F929F92AF92BF920B
:109D9000CF92DF92EF92FF920F931F93CF93DF93B7
:109DA00000D01F92CDB7DEB70E942B2A0E94F2B2DC
:109DB0006B017C0110912202112309F47BC0809178
:109DC000BF0A882309F476C04091020B5091030B1F
:109DD0006091040B7091050B46015701841A950A96
:109DE000A60AB70AB7FC78C0833051F134F4813049
:109DF0000CF460C0EDEEF8E106C0843009F05AC002
:109E0000EDEEF8E13BC084919F012F5F3F4F3B8314
:109E10002A83882329F00E947D3DEA81FB81F3CFCC
:109E2000E5E0F5E184919F012F5F3F4F3B832A835B
:109E3000882309F43FC00E947D3DEA81FB81F2CF77
:109E4000EDEEF8E184919F012F5F3F4F3B832A8322
:109E5000882329F00E947D3DEA81FB81F3CFEEEE5D
:109E6000F4E184919F012F5F3F4F3B832A83882336
:109E700009F10E947D3DEA81FB81F3CF84919F012E
:109E80002F5F3F4F3B832A83882329F00E947D3D2B
:109E9000EA81FB81F3CFE6EDF4E184919F012F5F2E
:109EA0003F4F3B832A83882329F00E947D3DEA812E
:109EB000FB81F3CF212F30E0A8EEB3E00E947EC9F2
:109EC000C60ED71EE81EF91EC092020BD092030BDD
:109ED000E092040BF092050B89B182FB882780F990
:109EE0008093E4139091E51398170CF049C080918A
:109EF000E6139091E713A091E813B091E91301964E
:109F0000A11DB11D883B3DE39307A105B1054CF4AC
:109F10008093E6139093E713A093E813B093E913AB
:109F20003BC01092E6131092E7131092E8131092C0
:109F3000E9138091890F882319F00E948B751DC049
:109F4000E7E1F5E18491FB83EA83882371F0082E31
:109F5000000C990B0E9423742A813B812F5F3F4F95
:109F60003B832A83F9018491F0CF8DE090E00E9439
:109F700023748AE090E00E9423748091E4130AC065
:109F8000891751F01092E6131092E7131092E8131C
:109F90001092E9138093E51380914216843010F4F7
:109FA0000E94013E0E94F2B2C090C40AD090C50A3D
:109FB000E090C60AF090C70AC114D104E104F1048C
:109FC00081F10091C00A1091C10A2091C20A30911A
:109FD000C30A0C0D1D1D2E1D3F1D4B015C01801A77
:109FE000910AA20AB30AB7FC1CC0E8EDF8E184911B
:109FF0009F012F5F3F4F3B832A83882329F00E94D4
:10A000007D3DEA81FB81F3CF60913116709132166C
:10A010008DE495E1FCDB8AE00E947D3D84E495E1DE
:10A0200081C0C0902302D0902402E0902502F090DD
:10A030002602C114D104E104F104E9F130910B0FBF
:10A0400020910C0F321749F06093C00A7093C10A37
:10A050008093C20A9093C30A2EC00091C00A109147
:10A06000C10A2091C20A3091C30A0C0D1D1D2E1D7C
:10A070003F1DDC01CB01801B910BA20BB30BB7FD85
:10A080001AC05F9A8091BC038E7F8093BC038A9A2A
:10A09000479A8091BC038D7F8093BC038091080117
:10A0A0008095817080930601479A8091BC038B7FD5
:10A0B0008093BC03129A8091120B9091130B90998C
:10A0C00002C0019604C0181619062CF4019790934B
:10A0D000130B8093120B8091120B9091130B8E3EF9
:10A0E00092400CF1E8EDF8E184919F012F5F3F4F22
:10A0F0003B832A83882329F00E947D3DEA81FB81EE
:10A10000F3CFE4E2F5E184919F012F5F3F4F3B8362
:10A110002A83882329F00E947D3DEA81FB81F3CFC9
:10A120008BE195E1E4DD0E94F2B200910E0B1091FB
:10A130000F0B2091100B3091110B4B015C01801A19
:10A14000910AA20AB30AB7FC4EC08B019C010C53C2
:10A15000164F2F4F3F4F00930E0B10930F0B209372
:10A16000100B3093110B4F9BA9C17A9BA7C1209173
:10A17000060120FFA3C120915B1521119FC1379BD0
:10A180009DC1379B9BC1029B99C100910A0B109105
:10A190000B0B20910C0B30910D0B011511052105B6
:10A1A000310599F0DC01CB01801B910BA20BB30BA5
:10A1B00080569A4EA109B1098827B7FD8395992742
:10A1C000AA27BB27682F619501C060E0262F30E0E9
:10A1D0008091020161118095807180930001B90125
:10A1E00087E00E94F3B190910B0F80910C0F9817AC
:10A1F00091F0E0910C0F28E5E29FF0011124E35566
:10A20000FB4F608180910C0F90910B0F981729F0F4
:10A210008F5F8F70F9CF6091CD0370E089E00E946D
:10A22000F3B180915615882309F4F8C00091080213
:10A230001091090280900A028C8290900B029A82FF
:10A240006091D5037091D6036E5F7F4F072E000C8F
:10A25000880B990B0E946AC59801A4010E9464C5ED
:10A2600087FDDCC0F0900C0F212C312CE12C1982E1
:10A2700080910B0F8F1509F462C08F2D90E038E5A7
:10A28000A32EA89EF001A99EF00D1124E55AFB4FC4
:10A29000458956896789708D452B462B472B81F45C
:10A2A000418D528D638D748D452B462B472B41F488
:10A2B000458D568D678D70A1452B462B472BD1F1CF
:10A2C00028E5B22EB89E9001B99E300D1124C90127
:10A2D000855A9B4F6C01FC0161817281838194815D
:10A2E0000E94F9CB4B015C01F60161A172A183A12F
:10A2F00094A10E9468C52B013C01F60165A176A1DD
:10A3000087A190A50E9468C59B01AC01C301B20161
:10A310000E946ACAA50194010E94C9C55B016C0133
:10A3200091014E2D59810E94B4CB18161CF41501D1
:10A33000EC2CD98281E08F0D8F70F82E99CF20916F
:10A340000C0230910D0240910E0250910F02B101AA
:10A350008E2D99810E94C9C598014C815A810E9415
:10A360008EC96B017C019B01AC01B8018C819A8183
:10A370000E94B4CB1816ACF00091040210910502B3
:10A38000809006028C82909007029A829801A40124
:10A39000B601C7010E94B4CB18161CF08601EC82EE
:10A3A000FA82C090060BD090070BE090080BF0905B
:10A3B000090B98014C815A81C701B6010E94B4CBA8
:10A3C0001816D4F420E037ED43EA5CE3B8018C8141
:10A3D0009A810E94C9C54B015C0128E431EE4AE72D
:10A3E0005FE3C701B6010E94C9C5A50194010E949F
:10A3F0008EC98B018C839A83C801AC81BA8180930A
:10A40000060B9093070BA093080BB093090BB801B0
:10A41000CD010E94D2CACB010E94C1720E949F7FCF
:10A4200089E69FE00E94BE38A090CC0AA982AA20AB
:10A4300009F44DC00E94F2B20091C80A1091C90AF5
:10A440002091CA0A3091CB0ADC01CB01801B910B11
:10A45000A20BB30BB7FD3BC00E94F2B26B017C01B3
:10A46000B9802B2D30E0A8EEB3E00E947EC9C60E65
:10A47000D71EE81EF91EC092C80AD092C90AE092FF
:10A48000CA0AF092CB0A0E94E1798AE00F900F90FD
:10A490000F900F90DF91CF911F910F91FF90EF9050
:10A4A000DF90CF90BF90AF909F908F907F906F90F4
:10A4B0005F904F903F902F900C947D3D60930A0BDE
:10A4C00070930B0B80930C0B90930D0B5ECE0F9043
:10A4D0000F900F900F90DF91CF911F910F91FF90F0
:10A4E000EF90DF90CF90BF90AF909F908F907F9034
:10A4F0006F905F904F903F902F9008952F923F92D2
:10A500004F925F926F927F928F929F92AF92BF9283
:10A51000CF92DF92EF92FF920F931F93CF93DF932F
:10A52000CDB7DEB7CC54D1090FB6F894DEBF0FBE5D
:10A53000CDBF80912102882319F08AED9AE0E9D9F4
:10A540008091510B83FDA9C0C090E60AD090E70A24
:10A55000E090E80AF090E90A2091C9033091CA031B
:10A560004091CB035091CC03C701B6010E9464C552
:10A57000882309F492C08091500B811133C06091FF
:10A58000D7037091D8038091D9039091DA030E9488
:10A59000D2CA20913702309138026217730714F53E
:10A5A000C092C903D092CA03E092CB03F092CC03CD
:10A5B000EDEEF8E184917F019FEFE91AF90A882313
:10A5C00021F00E947D3DF701F5CFEBEBF4E18491A2
:10A5D0007F01AFEFEA1AFA0A882321F00E947D3D3D
:10A5E000F701F5CF8090E60A9090E70AA090E80A7C
:10A5F000B090E90A2091C9033091CA034091CB037E
:10A600005091CC03C501B4010E948DC96B017C013E
:10A6100020E030E0A9010E94B4CB87FF04C0F7FA24
:10A62000F094F7F8F094E091BE0AB4E0EB9FF001EB
:10A630001124ED5CFD4F2081318142815381C7019E
:10A64000B6010E94C9C520E030E048E453E40E940E
:10A65000B4CB181614F58092C9039092CA03A09245
:10A66000CB03B092CC03EDEEF8E184917F019FEF34
:10A67000E91AF90A882321F00E947D3DF701F5CF00
:10A68000ECE9F4E184917F01AFEFEA1AFA0A88233A
:10A6900021F00E947D3DF701F5CF80913B1660903F
:10A6A000020270900302C090DA0AD090DB0AE090B8
:10A6B000DC0AF090DD0A8090DE0A9090DF0AA0901C
:10A6C000E00AB090E10A882309F481C220903C1688
:10A6D00030903D1640903E1650903F1620E030E0FE
:10A6E000A901C201B1010E9464C5882379F02091BB
:10A6F000E20A3091E30A4091E40A5091E50AC2016E
:10A70000B1010E94B4CB18160CF061C2B301770CF2
:10A71000880B990B0E946AC520914B0230914C0224
:10A7200040914D0250914E020E94C9C52AE037ED7A
:10A7300043E25CE30E94C9C56DA77EA78FA798ABD3
:10A740002091BD033091BE034091BF035091C003DF
:10A75000C701B6010E948DC92B013C012091C103A4
:10A760003091C2034091C3035091C403C501B401A9
:10A770000E948DC925966CAF7DAF8EAF9FAF259798
:10A7800020E030E0A901C301B2010E9464C581113B
:10A7900041C020E030E0A90125966CAD7DAD8EADC5
:10A7A0009FAD25970E9464C5811134C07090BE0A88
:10A7B00019AA1AAA1BAA1CAAC982DA82EB82FC82F5
:10A7C0008D829E82AF82B8868091E20A9091E30AE0
:10A7D000A091E40AB091E50A89879A87AB87BC8784
:10A7E000AE01475F5F4FBE016B5F7F4FCE010196A9
:10A7F0000E94C4A7FE01F1966F01E72C8E01035D54
:10A800001F4F26EE3AE0AE01475F5F4FBE016B5F20
:10A810007F4F2AC22091C5033091C6034091C703E0
:10A820005091C8036091E20A7091E30A8091E40AB2
:10A830009091E50A0E948DC929966CAF7DAF8EAFCD
:10A840009FAF29972091C9033091CA034091CB0350
:10A850005091CC036091E60A7091E70A8091E80A72
:10A860009091E90A0E948DC921966CAF7DAF8EAFA1
:10A870009FAF2197A3019201C301B2010E94C9C5F4
:10A880006B017C0125962CAD3DAD4EAD5FAD25979E
:10A89000CA01B9010E94C9C59B01AC01C701B6013B
:10A8A0000E948EC96B017C0129962CAD3DAD4EAD49
:10A8B0005FAD2997CA01B9010E94C9C59B01AC01CE
:10A8C000C701B6010E948EC90E94F9CB6B017C01C1
:10A8D0002DEB37E346E855E30E9464C587FF17C0B8
:10A8E00020E030E0A90121966CAD7DAD8EAD9FAD2D
:10A8F00021970E94B4CB2196CCACDDACEEACFFAC82
:10A90000219787FF04C0F7FAF094F7F8F0942DEB45
:10A9100037E346E855E3C701B6010E9464C587FDE9
:10A92000A6C120E030E040EA50E4C701B6010E9431
:10A930006ACA0E94D7CA1B01672B19F422242394E8
:10A94000312CB10180E090E00E9468C59B01AC0110
:10A9500060E070E080E89FE30E946ACA4B015C01FE
:10A960009B01AC01C701B6010E94C9C52D966CAF11
:10A970007DAF8EAF9FAF2D97A5019401C301B201AA
:10A980000E94C9C5698B7A8B8B8B9C8BA501940126
:10A9900025966CAD7DAD8EAD9FAD25970E94C9C546
:10A9A0006D8B7E8B8F8B988FA501940129966CAD52
:10A9B0007DAD8EAD9FAD29970E94C9C5698F7A8FF5
:10A9C0008B8F9C8FA501940121966CAD7DAD8EADD2
:10A9D0009FAD21970E94C9C56D8F7E8F8F8F98A3E1
:10A9E00080E1EDEBF3E0DE01119601900D928A9586
:10A9F000E1F799249394F1E02F1A310809F04BC044
:10AA0000E090BE0A2D968CAD9DADAEADBFAD2D973D
:10AA100089AF9AAFABAFBCAF8091DA0A9091DB0AF5
:10AA2000A091DC0AB091DD0A89A39AA3ABA3BCA3D1
:10AA30008091DE0A9091DF0AA091E00AB091E10ACC
:10AA40008DA39EA3AFA3B8A78091E20A9091E30AD9
:10AA5000A091E40AB091E50A89A79AA7ABA7BCA781
:10AA6000AE01475D5F4FBE016B5D7F4FCE018196AA
:10AA70000E94C4A7DE01D9966D018E01035D1F4FB0
:10AA800026EE3AE0AE01475D5F4FBE016B5D7F4F42
:10AA9000CE018196EBC08091FA0A811112C00E940A
:10AAA000F2B2DC01CB0188539F4FAF4FBF4F809371
:10AAB000F60A9093F70AA093F80AB093F90A9092D5
:10AAC000FA0A0E949F7F0E94F2B2C090F60AD090CC
:10AAD000F70AE090F80AF090F90ADC01CB018C1932
:10AAE0009D09AE09BF09B7FD11C00E94F2B2DC0199
:10AAF000CB0188539F4FAF4FBF4F8093F60A90937F
:10AB0000F70AA093F80AB093F90A38D96E01B1E1B7
:10AB1000CB0ED11CFE0131967F015601D6012D913D
:10AB20003D914D915D916D01F7016081718182814F
:10AB300093810E948EC9D7016D937D938D939D93D0
:10AB40007D01AA16BB0651F7E090BE0A2D968CAD8A
:10AB50009DADAEADBFAD2D978DAB9EABAFABB8AFDE
:10AB600089819A81AB81BC8189A39AA3ABA3BCA341
:10AB70008D819E81AF81B8858DA39EA3AFA3B8A719
:10AB800089859A85AB85BC8589A79AA7ABA7BCA701
:10AB9000AE01475D5F4FBE016B5D7F4FCE01819679
:10ABA0000E94C4A7DE01D5966D018E01035D1F4F83
:10ABB0009E01235F3F4FAE01475D5F4FBE016B5D5E
:10ABC0007F4FCE018196D6D0811115CF19CFB30119
:10ABD000770C880B990B0E946AC520914B0230912B
:10ABE0004C0240914D0250914E020E94C9C52AE08C
:10ABF00037ED43E25CE30E94C9C569AB7AAB8BAB2E
:10AC00009CAB7090BE0A8091E20A9091E30AA091F9
:10AC1000E40AB091E50AC982DA82EB82FC82898A71
:10AC20009A8AAB8ABC8A89A39AA3ABA3BCA31DA6AC
:10AC30001EA61FA618AAAE014F5D5F4FBE016F5E34
:10AC40007F4FCE0101960E94C4A7FE01BD966F0101
:10AC5000E72C8E010F5C1F4F26EE3AE0AE014F5DF0
:10AC60005F4FBE016F5E7F4FCE01019683D080E1C2
:10AC7000EAEDFAE0ADEBB3E001900D928A95E1F7D1
:10AC8000C45BDF4F0FB6F894DEBF0FBECDBFDF91C0
:10AC9000CF911F910F91FF90EF90DF90CF90BF90D9
:10ACA000AF909F908F907F906F905F904F903F906C
:10ACB0002F900895CF93DF9380E00E9442A3C2EBD0
:10ACC000DAE0688379838A839B8381E00E9442A3D0
:10ACD0006C837D838E839F8382E00E9442A368877A
:10ACE00079878A879B87DF91CF910895CF93DF93F0
:10ACF000E0914016F0E0EB58F44F8081882381F01A
:10AD0000E9E9F4E18491EF012196882321F00E9482
:10AD10007D3DFE01F7CF8AE0DF91CF910C947D3D20
:10AD2000DF91CF910895CF93DF938091B00A809304
:10AD3000B10AE0E9F4E18491EF012196882321F042
:10AD40000E947D3DFE01F7CF80914E1690914F16E7
:10AD5000A0915016B0915116BC01CD016F5F7F4F8D
:10AD60008F4F9F4F0E9404418AE00E947D3DDF91FA
:10AD7000CF91BCCF2F923F924F925F926F927F9272
:10AD80008F929F92AF92BF92CF92DF92EF92FF92FB
:10AD90000F931F93CF93DF93CDB7DEB7C857D10979
:10ADA0000FB6F894DEBF0FBECDBFE0915815F091FD
:10ADB0005915EF2B11F00C94835F2896DFAECEAEC1
:10ADC00028976E2C79016A015B01FC012081318199
:10ADD000428153816C962CAF3DAF4EAF5FAF6C9705
:10ADE0002091A9163091AA164091AB165091AC163D
:10ADF0006C966CAD7DAD8EAD9FAD6C970E94C9C554
:10AE00000E94BFCBE0966CAF7DAF8EAF9FAFE09757
:10AE1000D5018D919D910D90BC91A02DA0968CAFE8
:10AE20009DAFAEAFBFAFA0972091AD163091AE16DB
:10AE30004091AF165091B016BC01CD010E94C9C51A
:10AE40000E94BFCBE4966CAF7DAF8EAF9FAFE4970F
:10AE5000D6012D913D914D915C91A4962CAF3DAFC3
:10AE60004EAF5FAFA4972091B1163091B2164091CA
:10AE7000B3165091B416A4966CAD7DAD8EAD9FAD5A
:10AE8000A4970E94C9C50E94BFCBE8966CAF7DAF66
:10AE90008EAF9FAFE897D7012D913D914D915C9179
:10AEA00022962CAF3DAF4EAF5FAF22972091B516E3
:10AEB0003091B6164091B7165091B81622966CADE7
:10AEC0007DAD8EAD9FAD22970E94C9C50E94BFCBBC
:10AED00060966CAF7DAF8EAF9FAF60978091510B46
:10AEE00083FF1CC060962CAD3DAD4EAD5FAD60974D
:10AEF00020933D0F30933E0F40933F0F5093400FF0
:10AF000022968CAD9DADAEADBFAD229780932D0F37
:10AF100090932E0FA0932F0FB093300FD801BC91B8
:10AF2000BDA3F801F181F9ABD8011296BC91BEAB7B
:10AF3000F801F381FAAF80910B0F90910C0F891BF0
:10AF40008F708F3019F40E94BE4EF5CF00910B0F19
:10AF5000E9960FAFE99780910B0F082F10E01CA323
:10AF60000BA38091310F9091320FA091330FB091CC
:10AF7000340FE0968CAC9DACAEACBFACE097881AB9
:10AF8000990AAA0ABB0A8091350F9091360FA091B9
:10AF9000370FB091380FE4962CAC3DAC4EAC5FACA3
:10AFA000E497281A390A4A0A5B0A8091390F90916E
:10AFB0003A0FA0913B0FB0913C0FE8962CAD3DAD00
:10AFC0004EAD5FADE897281B390B4A0B5B0B2DA7E5
:10AFD0003EA74FA758AB80913D0F90913E0FA09197
:10AFE0003F0FB091400F60960CAD1DAD2EAD3FAD43
:10AFF0006097081B190B2A0B3B0B09A71AA72BA755
:10B000003CA7012B022B032B09F4BCC08091500BF1
:10B0100081114BC06091D7037091D8038091D903FF
:10B020009091DA030E94D2CA2091370230913802FF
:10B03000621773070CF039C060962CAD3DAD4EAD74
:10B040005FAD609720933D0F30933E0F40933F0FCD
:10B050005093400F22968CAD9DADAEADBFAD229703
:10B0600080932D0F90932E0FA0932F0FB093300F3E
:10B07000EDEEF8E184918F010F5F1F4F811103C046
:10B08000E6E1F6E104C00E947D3DF801F3CF849132
:10B090008F010F5F1F4F882321F00E947D3DF80133
:10B0A000F6CF19A61AA61BA61CA694E0699E8001DD
:10B0B00011240D5C1D4F69A57AA58BA59CA50E9446
:10B0C0006AC5D8012D913D914D915C910E94C9C5F1
:10B0D0006B017C0120E030E0A9010E94B4CB87FF26
:10B0E00004C0F7FAF094F7F8F0946091B5167091F7
:10B0F000B6168091B7169091B8160E94D2CA9B01DD
:10B10000AC01A8ECB0E00E9474C90E946AC5A70116
:10B1100096010E9464C587FF39C060960CAD1DADD5
:10B120002EAD3FAD609700933D0F10933E0F2093DF
:10B130003F0F3093400F22962CAD3DAD4EAD5FAD2D
:10B14000229720932D0F30932E0F40932F0F509363
:10B15000300FEDEEF8E184918F010F5F1F4F8111E9
:10B1600003C0E7EFF5E104C00E947D3DF801F3CF95
:10B1700084918F010F5F1F4F882321F00E947D3D36
:10B18000F801F6CF19A61AA61BA61CA6D501C40164
:10B190008827B7FD83959927AA27BB27782E57FEC6
:10B1A00003C0382F3260732E8DA59EA5AFA5B8A918
:10B1B000B7FF03C0972D9460792E09A51AA52BA57A
:10B1C0003CA537FF03C0172D1860712E24E0629E46
:10B1D000800111240D5C1D4F69A57AA58BA59CA546
:10B1E0000E946AC5D8012D913D914D915C910E94BC
:10B1F000C9C56B017C0120E030E0A9010E94B4CBFD
:10B2000087FF04C0C701B601905802C0C701B6014C
:10B2100020E030E040E05FE30E948EC90E94D7CA80
:10B220006AAB7BAB8CAB9DAB88E50BA11CA1809F6F
:10B23000F001819FF00D1124E55AFB4F108276AA90
:10B24000B501A401B7FE07C044275527BA01481924
:10B2500059096A097B0988E50BA11CA1809FF001AF
:10B26000819FF00D1124E55AFB4F458B568B678B60
:10B27000708F2C962CAE3DAE4EAE5FAE2C9757FE27
:10B280000DC088279927DC0182199309A409B50903
:10B290002C968CAF9DAFAEAFBFAF2C9728E50BA11E
:10B2A0001CA1209FF001219FF00D1124E55AFB4FB6
:10B2B0002C968CAD9DADAEADBFAD2C97818F928F8E
:10B2C000A38FB48F0DA51EA52FA538A937FF07C0E2
:10B2D00030952095109501951F4F2F4F3F4FE8E572
:10B2E0007E2EABA1BCA17A9EF0017B9EF00D1124B5
:10B2F000E55AFB4F058F168F278F30A38AA99BA98C
:10B30000ACA9BDA981A392A3A3A3B4A323964FAFD5
:10B310002397752EF62FE72F2C968CAD9DADAEADF5
:10B32000BFAD2C97481759076A077B0778F4299611
:10B330009FAD299723969FAF23972A967FAC2A9794
:10B340002B96FFAD2B972C96EFAD2C9723968FADB8
:10B350002397972DAF2FBE2F80179107A207B30712
:10B3600010F4D901C8010AA91BA92CA93DA980176D
:10B370009107A207B30710F4D901C80128E50BA172
:10B380001CA1209FF001219FF00D1124E55AFB4FD5
:10B3900085A396A3A7A3B0A70697A105B10508F4B6
:10B3A000ABC5DF01AE5ABF4F8091CD039091CE0364
:10B3B0008D939C9361A6452B462B472B09F05F98F4
:10B3C00088E50BA11CA1809FF001819FF00D112445
:10B3D000E55AFB4F818D928DA38DB48D892B8A2BDD
:10B3E0008B2B11F08A98479888E50BA11CA1809FB0
:10B3F000F001819FF00D1124E55AFB4F858D968D4C
:10B40000A78DB0A1892B8A2B8B2B31F0809108015D
:10B4100081708093060147982AA93BA94CA95DA990
:10B42000232B242B252B09F470C58091560B8823E0
:10B4300019F081508093560B611004C0129880E27D
:10B440008093560B60904C0B70904D0B00914E0BFF
:10B4500010914F0B9301A8016DA179A98EA99AAD06
:10B460000E9464C587FF04C06DA279AA0EAB1AAF13
:10B47000C501B4010E946AC52091991630919A16AF
:10B4800040919B1650919C160E94C9C526966CAFA0
:10B490007DAF8EAF9FAF2697698B7A8B8B8B9C8B02
:10B4A000C201B1010E946AC520919D1630919E167D
:10B4B00040919F165091A0160E94C9C52B013C01D6
:10B4C0006D8B7E8B8F8B988F6DA57EA58FA598A990
:10B4D0000E946AC52091A1163091A2164091A31630
:10B4E0005091A4160E94C9C54B015C01698F7A8FE7
:10B4F0008B8F9C8F2091A5163091A6164091A71690
:10B500005091A816C701B6010E94C9C56B017C0104
:10B510006D8F7E8F8F8F98A388E50BA11CA1809FD4
:10B52000F001819FF00D1124E55AFB4F25893689E2
:10B530004789508D2DA73EA74FA758AB2630310520
:10B540004105510508F4EAC42896AEADBFAD289771
:10B55000CD90DD90ED90FC9020E030E0A901C70196
:10B56000B6010E9464C58111F8C426962CAD3DAD8C
:10B570004EAD5FAD2697CA01B9010E94C9C56B01E6
:10B580007C01A3019201C301B2010E94C9C59B01C4
:10B59000AC01C701B6010E948EC96B017C01A501F7
:10B5A0009401C501B4010E94C9C59B01AC01C7014A
:10B5B000B6010E948EC90E94F9CB28E50BA11CA1FF
:10B5C000209FF001219FF00D1124E55AFB4F658764
:10B5D00076878787908B88E50BA11CA1809FF0015F
:10B5E000819FF00D1124E55AFB4F458456846784F2
:10B5F0007088A301920160E070E080E89FE30E9400
:10B600006ACA64966CAF7DAF8EAF9FAF64972DA171
:10B6100039A94EA95AAD0E94C9C54B015C01809160
:10B620000B0F9091090F891B8F7027968FAF27976B
:10B63000A501940160E074E284E799E40E946ACA7B
:10B640000E94BFCB6B017C0127968FAD279782505C
:10B65000863008F491C4A5019401C301B2010E948F
:10B66000C9C59B01AC010E94C9C568966CAF7DAF8E
:10B670008EAF9FAF689788E5ABA1BCA18A9F800180
:10B680008B9F100D1124055A1B4F68962CAD3DADB4
:10B690004EAD5FAD6897D80111962D933D934D93B4
:10B6A0005C93149795962D913D914D915C9198974F
:10B6B0002EAB3FAB48AF59AFCA01B9010E9468C574
:10B6C0006AAF7BAF8CAF9DAF9B01AC01C501B401EC
:10B6D0000E94C9C50E9454CA0E94D7CAA8966CAFDE
:10B6E0007DAF8EAF9FAFA897F801EE5BFF4F6083F1
:10B6F0007183828393838E010F5E1F4F2A961FAF43
:10B700000EAF2A970051110924961FAF0EAF249750
:10B7100004E31BE0AC961FAF0EAFAC978E010F5D3C
:10B720001F4F1AA309A324960EAD1FAD2497AA9606
:10B730001FAF0EAFAA97312C212C10E81DA30FE3E9
:10B7400009AB2A96AEADBFAD2A972D913D914D9193
:10B750005D912A96BFAFAEAF2A97C501B4010E9492
:10B76000C9C56B017C01AA96EEADFFADAA976193A6
:10B77000719381939193AA96FFAFEEAFAA9720E0C1
:10B7800030E0A9010E94B4CB87FF04C0F7FAF0941F
:10B79000F7F8F094AC96AEADBFADAC974D905D9020
:10B7A0006D907D90AC96BFAFAEAFAC97A701960100
:10B7B000C301B2010E9464C587FD18C409A11AA182
:10B7C0002A962EAD3FAD2A970217130709F0B9CF7D
:10B7D00020E030E040E85FE3632D722D8DA199A950
:10B7E0000E9464C587FF58C07E0131E1E30EF11C61
:10B7F00024960EAD1FAD2497232D322D4DA159A9AE
:10B80000D8016D917D918D919C910E94C9C5F801DF
:10B8100061937193819391938F01EE16FF0661F707
:10B8200028E50BA11CA1209FC001219F900D112490
:10B830009C01255A3B4F790189010E5B1F4FA89649
:10B840006CAD7DAD8EAD9FADA8970E9468C5232DD0
:10B85000322D4DA159A90E94C9C50E94D7CAD8014D
:10B860006D937D938D939C931397232D322D4DA132
:10B8700059A9632D722D8DA199A90E94C9C56896F9
:10B880002CAD3DAD4EAD5FAD68970E94C9C5F701C7
:10B8900061837283838394832AAD3BAD4CAD5DADF0
:10B8A00064966CAD7DAD8EAD9FAD64970E94C9C5A9
:10B8B0006DA37EA38FA398A70DA51EA52FA538A9BC
:10B8C000012B022B032B09F0A9C388E52BA13CA176
:10B8D000829F8001839F100D1124055A1B4FF80190
:10B8E000818D928DA38DB48D892B8A2B8B2B09F0A2
:10B8F00095C3858D968DA78DB0A1892B8A2B8B2B17
:10B9000009F08CC32091300B3091310B4091320BF8
:10B910005091330B6DA17EA18FA198A50E94C9C53E
:10B920000E9454CA0E94D7CA2B013C01D801D79665
:10B930001C9288E52BA13CA1829F8001839F100D62
:10B940001124055A1B4FF801E25BFF4F40825182E0
:10B9500062827382C301B2010E9468C56B017C01DF
:10B960002DA13EA14FA158A50E946ACA6AAF7BAF24
:10B970008CAF9DAFD80151966D937D938D939C9321
:10B9800054972DEB37E346E051E4C701B6010E941E
:10B99000C9C50E94D7CAF80162AB73AB84AB95AB43
:10B9A00087A9882371F1FE962091240B3091250BF5
:10B9B0004091260B5091270B608171818281938188
:10B9C0000E94C9C52AAD3BAD4CAD5DAD0E94C9C555
:10B9D0002091B5163091B6164091B7165091B81611
:10B9E0000E94C9C59B01AC0160E074E284EF99E458
:10B9F0000E946ACA0E94D7CAD801D9967C936E93D6
:10BA0000D89788E50BA11CA1809FF001819FF00DC4
:10BA10001124E55AFB4F21813281438154812C96B8
:10BA20002CAF3DAF4EAF5FAF2C97CA01B9010E945A
:10BA3000F9CB362E272E8C0144E15BE062965FAF96
:10BA40004EAF62973E0151E1650E711C84E19BE0AF
:10BA50009FAB8EAB24964EAC5FAC249739A62DA637
:10BA60000DA319AB1AAAD201CD90DD90ED90FD90F7
:10BA70002D0120E030E0A901C701B6010E94B4CB3E
:10BA800087FF04C0F7FAF094F7F8F094EEA9FFA945
:10BA900081909190A190B190FFABEEABA701960180
:10BAA000C501B4010E9464C587FDD4C56414750442
:10BAB000D1F627965FAD2797552309F444C6C09069
:10BAC0000D0FD0900E0FE0900F0FF090100F2DEB98
:10BAD00037E346E855E3C701B6010E9464C587FD18
:10BAE00032C6C701B6010E94F9CB6B017C019B01F4
:10BAF000AC01632D722DC8010E9464C587FD03C08F
:10BB00003C2C2D2C87019601A701632D722DC801B5
:10BB10000E946ACA68966CAF7DAF8EAF9FAF689780
:10BB200081E19FE028969FAF8EAF289720E030E01C
:10BB300040E85FE32AAB3BAB4CAB5DAB1EAA28965B
:10BB4000AEADBFAD28972D913D914D915D91289659
:10BB5000BFAFAEAF289768966CAD7DAD8EAD9FAD93
:10BB600068970E94C9C54B015C012496EEADFFADFC
:10BB70002497C190D190E190F1902496FFAFEEAF61
:10BB80002497FEA9FF2391F02AA93BA94CA95DA9FE
:10BB90000E94C9C54B015C012AA93BA94CA95DA91A
:10BBA000C701B6010E94C9C56B017C01A7019601BE
:10BBB000C501B4010E94B4CB20E030E0A901181601
:10BBC0000CF08EC5C701B6010E94B4CB18160CF458
:10BBD00082C520E030E0A901C501B4010E9464C51E
:10BBE00087FD79C52601370177FA709477F870944C
:10BBF000A3019201C501B4010E94B4CB181614F43C
:10BC0000240135016296AEADBFAD6297CD90DD9057
:10BC1000ED90FD906296BFAFAEAF6297A301920127
:10BC2000C701B6010E9464C587FF15C0A301920138
:10BC3000C701B6010E946ACA9B01AC016AA97BA92F
:10BC40008CA99DA90E94C9C56AAB7BAB8CAB9DAB8F
:10BC5000BEA9BF5FBEABE1E2FFE028962EAD3FADCF
:10BC60002897E217F30709F06ACF3EA9332361F062
:10BC70002AA93BA94CA95DA9632D722DC8010E9478
:10BC8000C9C5362E272E8C0124EA30E74DE75FE345
:10BC9000632D722DC8010E94C9C56B017C012091E2
:10BCA000520B3091530B4091540B5091550B0E9405
:10BCB00064C587FD3EC589A59DA5ADA1B9A98093A1
:10BCC000520B9093530BA093540BB093550B28E554
:10BCD0004BA15CA1249FC001259F900D1124DC0184
:10BCE000A55ABB4F7D01232D322DA801632D722D46
:10BCF000C8010E94C9C5F70161877287838794874D
:10BD00006AAD7BAD8CAD9DAD90589B01AC010E949E
:10BD10008EC9D7011D962D913D914D915C91509703
:10BD20000E94C9C59B01AC016BE077ED83E29BE308
:10BD30000E948DC99B01AC018BE097EDA3E2BBE3B0
:10BD4000F70185839683A783B08710812C966CAD0D
:10BD50007DAD8EAD9FAD2C970E9464C518160CF476
:10BD6000F7C483E0182B88E52BA13CA1829FF0014A
:10BD7000839FF00D1124E55AFB4F108380E1FE01F3
:10BD80003196A1E1BFE001900D928A95E1F72C96E2
:10BD90008CAD9DADAEADBFAD2C9780930D0F909344
:10BDA0000E0FA0930F0FB093100FE0960CAD1DADCA
:10BDB0002EAD3FADE0970093310F1093320F2093DB
:10BDC000330F3093340FE4962CAD3DAD4EAD5FADE7
:10BDD000E4972093350F3093360F4093370F5093ED
:10BDE000380FE8968CAD9DADAEADBFADE8978093B2
:10BDF000390F90933A0FA0933B0FB0933C0F60968E
:10BE00000CAD1DAD2EAD3FAD609700933D0F10936F
:10BE10003E0F20933F0F3093400F6C962CAD3DADFD
:10BE20004EAD5FAD6C972093210F3093220F40935E
:10BE3000230F5093240FA0968CAD9DADAEADBFAD3A
:10BE4000A0978093250F9093260FA093270FB09370
:10BE5000280FA4960CAD1DAD2EAD3FADA497009359
:10BE6000290F10932A0F20932B0F30932C0F22961B
:10BE70002CAD3DAD4EAD5FAD229720932D0F30938D
:10BE80002E0F40932F0F5093300F90910B0F8091F6
:10BE90000C0F981303C084E68093080FE9968FADCA
:10BEA000E9978F5F8F7080930B0F80910B0F9091AC
:10BEB0000A0F81508F7089134DC410910C0F1BA372
:10BEC00000910B0F09A728E51BA109A51013CDC4EC
:10BED000812C912CA12CB12C1DA61DA219AA1EAE3D
:10BEE000212C312C00E010E029A53BA12313CAC46A
:10BEF0002114310409F079C580916F00826080932C
:10BF00006F0081E0E2C680E0E0C66090480B709070
:10BF1000490B00914A0B10914B0B9CCA818D928D5D
:10BF2000A38DB48D0697A105B10508F00DCB858DC5
:10BF3000968DA78DB0A10697A105B10508F004CB99
:10BF400020E030E0A901C701B6010E94B4CB87FF11
:10BF500004C0F7FAF094F7F8F09488E50BA11CA15F
:10BF6000809FF001819FF00D1124E55AFB4FC5869B
:10BF7000D686E786F08A2FCB8091440B9091450BB3
:10BF8000A091460BB091470BC816D906EA06FB06EE
:10BF900008F061CB8C199D09AE09BF09BC01CD0128
:10BFA000660F771F881F991F27964FAD2797042F7D
:10BFB00010E020E030E0A90198010E9452C9CA01B6
:10BFC000B9010E9468C50E94BFCB6C0D7D1D8E1DFE
:10BFD0009F1D0E9468C59B01AC0160E074E284E78C
:10BFE00099E40E946ACA4B015C0135CBA701960116
:10BFF000C301B2010E946ACA7B018C019B01AC01A2
:10C00000632D722D8DA199A90E94B4CB18160CF046
:10C01000D5CB3E2C2F2C0DA319ABD0CB0AA91BA935
:10C020002CA93DA9012B022B032B49F020912C0BAD
:10C0300030912D0B40912E0B50912F0B08C0209169
:10C04000280B3091290B40912A0B50912B0B6DA19D
:10C050007EA18FA198A50E94C9C50E9454CA0E94C2
:10C06000D7CA2B013C012AA93BA94CA95DA9232BC6
:10C07000242B252BC9F020E030E0A9016091240B8E
:10C080007091250B8091260B9091270B0E9464C51F
:10C09000882351F081E009A51AA52BA53CA510160F
:10C0A0001106120613060CF080E098E52BA13CA1C6
:10C0B000929F8001939F100D1124055A1B4FD801A8
:10C0C000D7968C93882309F4B2C02091210F309128
:10C0D000220F4091230F5091240F6C966CAD7DADD3
:10C0E0008EAD9FAD6C970E948DC969A77AA78BA76B
:10C0F0009CA72091250F3091260F4091270F50913A
:10C10000280FA0966CAD7DAD8EAD9FADA0970E941F
:10C110008DC94B015C012091290F30912A0F40916C
:10C120002B0F50912C0FA4966CAD7DAD8EAD9FADB5
:10C13000A4970E948DC96B017C0129A53AA54BA546
:10C140005CA5CA01B9010E94C9C569A77AA78BA7D6
:10C150009CA7A5019401C501B4010E94C9C59B011A
:10C16000AC0169A57AA58BA59CA50E948EC94B013F
:10C170005C01A7019601C701B6010E94C9C59B01D8
:10C18000AC01C501B4010E948EC90E94F9CB6B01BC
:10C190007C0120912D0F30912E0F40912F0F509147
:10C1A000300F22966CAD7DAD8EAD9FAD22970E9473
:10C1B0008DC9A70196010E946ACA6B017C01F80132
:10C1C000FE96608371838283938320E030E040E4B5
:10C1D00050E40E94B4CB18161CF4F80117AA27C02B
:10C1E0002091240B3091250B4091260B5091270B69
:10C1F000C701B6010E94C9C59B01AC016091200B2B
:10C200007091210B8091220B9091230B0E946ACA9E
:10C210002DA13EA14FA158A50E94C9C50E94D7CA11
:10C22000641575058605970510F42B013C01809176
:10C23000751690917616A0917716B09178160EA982
:10C240001FA928AD39AD80179107A207B30708F4DD
:10C25000DFC02DA53EA54FA558A9232B242B252BA8
:10C2600041F16091791670917A1680917B169091C8
:10C270007C166415750586059705D8F42EA93FA987
:10C2800048AD59AD0E9443C96B017C012DA53EA567
:10C290004FA558A9C301B2010E9443C9C616D706CB
:10C2A000E806F90630F4C701B6010E9452C9290117
:10C2B0003A0188E50BA11CA1809FF001819FF00D40
:10C2C0001124E55AFB4FC18CD28CE38CF48CC11441
:10C2D000D104E104F10431F160917D1670917E1674
:10C2E00080917F16909180166415750586059705D7
:10C2F000C8F42EA93FA948AD59AD0E9443C94B01CE
:10C300005C01A7019601C301B2010E9443C98616D0
:10C310009706A806B90630F4C501B4010E9452C9B7
:10C3200029013A0188E50BA11CA1809FF001819FA2
:10C33000F00D1124E55AFB4FC58CD68CE78CF0A08C
:10C34000C114D104E104F10431F1609181167091BE
:10C350008216809183169091841664157505860562
:10C360009705C8F42EA93FA948AD59AD0E9443C90D
:10C370004B015C01A7019601C301B2010E9443C9B0
:10C3800086169706A806B90630F4C501B4010E94C6
:10C3900052C929013A0188E50BA11CA1809FF00137
:10C3A000819FF00D1124E55AFB4FC1A0D2A0E3A05C
:10C3B000F4A0C114D104E104F10409F4BACA6091F3
:10C3C000851670918616809187169091881664154F
:10C3D00075058605970508F0ACCA2EA93FA948AD9A
:10C3E00059AD0E9443C94B015C01A7019601C301ED
:10C3F000B2010E9443C986169706A806B90608F03E
:10C4000098CAC501B4010E9452C929013A0191CAD2
:10C410002DA53EA54FA558A9232B242B252BC9F1CB
:10C420006091791670917A1680917B1690917C16A6
:10C43000641575058605970560F50E9468C52AADE7
:10C440003BAD4CAD5DAD0E94C9C56B017C016DA5D6
:10C450007EA58FA598A90E9468C54B015C01C30108
:10C46000B2010E9468C5A50194010E94C9C59B0143
:10C47000AC01C701B6010E9464C587FF0AC0A501CF
:10C480009401C701B6010E946ACA0E94D7CA2B0153
:10C490003C0188E50BA11CA1809FF001819FF00D5C
:10C4A0001124E55AFB4F818C928CA38CB48C81149F
:10C4B0009104A104B104B9F160917D1670917E16CA
:10C4C00080917F16909180166415750586059705F5
:10C4D00050F50E9468C52AAD3BAD4CAD5DAD0E94E4
:10C4E000C9C56B017C01C501B4010E9468C54B013F
:10C4F0005C01C301B2010E9468C5A50194010E94BC
:10C50000C9C59B01AC01C701B6010E9464C587FF84
:10C510000AC0A5019401C701B6010E946ACA0E941F
:10C52000D7CA2B013C0188E50BA11CA1809FF0011B
:10C53000819FF00D1124E55AFB4F858C968CA78CBA
:10C54000B0A081149104A104B104B9F160918116E5
:10C5500070918216809183169091841664157505EA
:10C560008605970550F50E9468C52AAD3BAD4CADD8
:10C570005DAD0E94C9C56B017C01C501B4010E947B
:10C5800068C54B015C01C301B2010E9468C5A501E9
:10C5900094010E94C9C59B01AC01C701B6010E946C
:10C5A00064C587FF0AC0A5019401C701B6010E94B6
:10C5B0006ACA0E94D7CA2B013C0188E50BA11CA1C5
:10C5C000809FF001819FF00D1124E55AFB4FC1A01F
:10C5D000D2A0E3A0F4A0C114D104E104F10409F451
:10C5E000A8C96091851670918616809187169091E2
:10C5F0008816641575058605970508F09AC90E9486
:10C6000068C52AAD3BAD4CAD5DAD0E94C9C54B01BF
:10C610005C01C701B6010E9468C56B017C01C301C2
:10C62000B2010E9468C5A70196010E94C9C59B017D
:10C63000AC01C501B4010E9464C587FF7AC9A70196
:10C640009601C501B4010E946ACA0E94D7CA2B0193
:10C650003C016FC9FAA9FF2331F1A5019401632DB3
:10C66000722DC8010E94C9C54B015C0129A53DA5D9
:10C670004DA159A9C701B6010E94C9C59B01AC01D2
:10C68000C501B4010E9464C587FF22C0A7019601BD
:10C69000C501B4010E946ACA69A77DA78DA399ABA1
:10C6A00021E02AAB03CAA7019601C501B4010E948B
:10C6B0006ACA9B01AC0169A57DA58DA199A90E94BB
:10C6C000C9C569A77DA78DA399AB31E03AABEEC987
:10C6D00041E04AABEBC9A7019601C501B40113C003
:10C6E000C701B6010E9464C587FD09C020E030E0A3
:10C6F000A901C501B4010E94B4CB18164CF4A501E0
:10C700009401C701B6010E948DC92B013C017ACA70
:10C710002401350177FA709477F87094A30192019F
:10C72000C701B6010E9464C587FD6CCA26013701A6
:10C7300069CA29A53DA54DA159A9C701B6010E9405
:10C7400064C587FFB8CA39A42DA40DA119A9B3CA1D
:10C7500081E008CBF0900B0F8FEF8F0D8F708BA3C4
:10C76000B0900A0F80910B0FB81609F454C0C12C79
:10C77000D12C0BA10B1509F44EC0602E712C28E5AD
:10C78000269D8001279D100D1124055A1B4FD801AD
:10C790008C9183FD2BC00EAF1AAB0115110541F131
:10C7A0001996BC91B9A7F801F285FDA7D8011B968F
:10C7B000BC91BDA3F801F485F9ABD80115962D9075
:10C7C0003D904D905C901897A201910169A57DA5BF
:10C7D0008DA19F2F0E9464C5811180C1C114D10415
:10C7E00039F0F601808180FD79C102C0CEAEDAAAAF
:10C7F0008BA181508F708BA380910A0F8B1103C086
:10C80000CEACDAA8B6CF0BA10B1529F081E08B0DC9
:10C810008F70B82EF1CF10910A0F1BA3C12CD12C11
:10C8200080910B0F0BA1801709F447CB802E912C20
:10C8300028E5289D8001299D100D1124055A1B4FC4
:10C84000D8018C9183FD0AC05801C114D10439F07C
:10C85000C6010E941783811102C0BFC156018BA17E
:10C860008F5F8F708BA36501DBCF802F81508F701E
:10C87000289FF0011124E55AFB4F908193FF28CBAC
:10C8800089A722CB48E5439FC0011124DC01A55AAA
:10C89000BB4F1D018C9183FD19C015966D917D9143
:10C8A0008D919C9118970E94F9CBF62EE72ED82EE9
:10C8B000C92E0115110509F48AC0F801808180FD97
:10C8C0000AC0D1018C9180FD06C081C0FDA4EDA0FD
:10C8D000D9A8CEAC81C0F801808181608083C80175
:10C8E0000E94178381116FC0F80161817281838179
:10C8F00094810E94F9CB2B013C019B01AC0160E0CB
:10C9000070E080E89FE30E946ACA4B015C019B01D2
:10C91000AC016F2D7E2D8D2D9C2D0E94C9C5698384
:10C920007A838B839C832DA53DA149A95EADC5016A
:10C93000B4010E94C9C5698B7A8B8B8B9C8BAE012D
:10C940004F5F5F4FBE016F5E7F4FC8010E9412A410
:10C95000D801D7968C918823B1F12091240B309186
:10C96000250B4091260B5091270BF801FE96608114
:10C970007181828193810E94C9C52091B516309141
:10C98000B6164091B7165091B8160E94C9C54B0112
:10C990005C019B01AC01C301B2010E94C9C50E94A8
:10C9A000D7CAF80173AF62AFA50194016F2D7E2D38
:10C9B0008D2D9C2D0E94C9C50E94D7CAD801DD9635
:10C9C0007C936E93DC97F80180818E7F80838F2C1F
:10C9D0009E2CAD2CBC2C81018BA18F5F8F708BA303
:10C9E000FDA6EDA2D9AACEAE7FCAD1018C918160FD
:10C9F0008C93C8010E94178381116BC0F101618182
:10CA00007281838194810E94F9CB6B017C019B012F
:10CA1000AC0160E070E080E89FE30E946ACA2B01ED
:10CA20003C012DEC3CEC4CE45DE30E94C9C56983FC
:10CA30007A838B839C839401A501C301B2010E9478
:10CA4000C9C5698B7A8B8B8B9C8BAE014F5F5F4F17
:10CA5000BE016F5E7F4FC1010E9412A4D101D79623
:10CA60008C918823B1F12091240B3091250B4091BA
:10CA7000260B5091270BF101FE9660817181828116
:10CA800093810E94C9C52091B5163091B616409188
:10CA9000B7165091B8160E94C9C54B015C019B01A5
:10CAA000AC01C701B6010E94C9C50E94D7CAF101F5
:10CAB00073AF62AF2DEC3CEC4CE45DE3C501B40117
:10CAC0000E94C9C50E94D7CAD101DD967C936E939E
:10CAD000DC97F10180818E7F80830ECA28E5269D38
:10CAE000F001279DF00D1124E55AFB4F808181FD57
:10CAF00043C0C114D10441F0D6011596CD90DD900C
:10CB0000ED90FC90189708C08BE0C82E87EDD82ECA
:10CB100083E2E82E8BE3F82EB8E5B69DF001B79DD1
:10CB2000F00D1124E55AFB4F81899289A389B489BC
:10CB3000BC01CD0190589B01AC010E948EC9F80147
:10CB400025853685478550890E94C9C59B01AC0162
:10CB5000C701B6010E948DC9E62E872E982EA92EF8
:10CB6000262F372F482F592F69A57DA58DA199A96B
:10CB70000E9464C587FF04C0E9A48DA49DA0A9A854
:10CB80002E2D382D492D5A2DC201B1010E9464C5A8
:10CB9000882309F42DCEF8E5F69DC001F79D900D90
:10CBA00011249C01255A3B4F6901D9018C91816068
:10CBB0008C93C8010E941783882329F0F601808195
:10CBC0008E7F808315CE8E2D982DA92DBA2DF6013E
:10CBD00085839683A783B0870BCED6018C9181FD88
:10CBE00052C0D60115962D913D914D915C911897AB
:10CBF00029A73AA74BA75CA71501B5E02B0E311C5E
:10CC0000F8014580568067807084A301920169A570
:10CC10007AA58BA59CA50E9464C587FF34C0F60148
:10CC200081899289A389B489BC01CD0190589B0167
:10CC3000AC010E948EC9D6011D962D913D914D915A
:10CC40005C9150970E94C9C59B01AC0169A57AA56A
:10CC50008BA59CA50E948DC96B017C019B01AC0139
:10CC6000C301B2010E94B4CB18166CF4D8018C91A8
:10CC700081608C93C5010E9417838823E1F0F8013D
:10CC800080818E7F808318E5189DF001199DF00D3D
:10CC90001124E55AFB4F21853285438554856581F2
:10CCA0007681878190850E9464C58111D8CD0BA1C2
:10CCB00000930A0FD4CDD101CD92DD92ED92FC927A
:10CCC00013970BA100930A0FDECFC858DF4F0FB6A2
:10CCD000F894DEBF0FBECDBFDF91CF911F910F91B2
:10CCE000FF90EF90DF90CF90BF90AF909F908F908C
:10CCF0007F906F905F904F903F902F90089580911C
:10CD00000B0F90910C0F891B8F708F3019F40E94BC
:10CD1000BE4EF5CF80910B0F8F5F8F70E0910B0FA0
:10CD200098E59E9FF0011124E55AFB4FDF011D920B
:10CD30009A95E9F798E090834091310F5091320F26
:10CD40006091330F7091340F458B568B678B708FCA
:10CD50004091350F5091360F6091370F7091380F19
:10CD6000418F528F638F748F4091390F50913A0FDA
:10CD700060913B0F70913C0F458F568F678F70A36A
:10CD800040913D0F50913E0F60913F0F7091400FC9
:10CD900041A352A363A374A320910B0F90910C0F96
:10CDA000291303C094E69093080F80930B0F809192
:10CDB0006F00826080936F00089590910B0F8091B7
:10CDC0000C0F981306C08091581590915915892B16
:10CDD00019F00E94BE4EF1CF0895CF93DF938B3DA3
:10CDE0009240B1F0E8EDF8E18491EF0121968823BB
:10CDF00021F00E947D3DFE01F7CFE1E3F6E1849151
:10CE0000EF012196882331F00E947D3DFE01F7CF8E
:10CE100080E001C081E0DF91CF9108952F923F9291
:10CE20004F925F926F927F928F929F92AF92BF923A
:10CE3000CF92DF92EF92FF920F931F93CF93DF93E6
:10CE4000CDB7DEB7C757D1090FB6F894DEBF0FBE16
:10CE5000CDBF2DB63EB6A7961FAE1EAEA79784E6F1
:10CE600090E0A9969FAF8EAFA99701E09E012B5944
:10CE70003F4F44E050E0BE01655A7F4FCE018959D3
:10CE80009F4F0E947EA99E012B593F4F42E050E0E8
:10CE9000BE0167597F4FCE0189599F4F0E947EA9DD
:10CEA00043E050E0BE01655A7F4F87ED92E00E945B
:10CEB00015CD892B09F43FC06F968FAD6F978823EE
:10CEC00039F08FE36C968FAF6C976D961FAE6D97B0
:10CED000EDEEF8E184917F012FEFE21AF20A811161
:10CEE00003C0E4EFF6E104C00E947D3DF701F2CFFC
:10CEF00084917F013FEFE31AF30A882321F00E9417
:10CF00007D3DF701F5CFBE01655A7F4F8BEE96E16F
:10CF10000E94074CEDEDF6E184917F019FEFE91A45
:10CF2000F90A882321F00E947D3DF701F5CF81E0C9
:10CF30008093570B54C5EDB7FEB7E696FFAFEEAF43
:10CF4000E6976B961CAE1DAE1EAE1FAE6B97A796F6
:10CF50001FAE1EAEA79701E09E012B593F4F41E047
:10CF600050E0BE0160597F4FCE0189599F4F0E940A
:10CF70007EA980E1E3E5F2E0DE01919601900D9259
:10CF80008A95E1F780E1E3E6F2E0DE015196019057
:10CF90000D928A95E1F780E1E3E7F2E0DE01119678
:10CFA00001900D928A95E1F7E1964FADE19750E03F
:10CFB0004D5F5F4F440F551F440F551F2DB73EB7B0
:10CFC000241B350B0FB6F8943EBF0FBE2DBF8DB797
:10CFD0009EB701967C0100E09E012B593F4FBC019A
:10CFE000CE0189599F4F0E947EA99E012B593F4F28
:10CFF00044E050E064E47BE0CE0189599F4F0E94F9
:10D000007EA9E1968FACE197912C93E0890E911C5B
:10D01000880C991C880C991CEDB7FEB7E819F90922
:10D020000FB6F894FEBF0FBEEDBF2DB73EB72F5F12
:10D030003F4F69018DB79EB7881999090FB6F894CB
:10D040009EBF0FBE8DBFEDB7FEB731965F019E014B
:10D050002B593F4FA401B601CE0189599F4F0E9421
:10D060007EA99E012B593F4FA401B501CE018959DC
:10D070009F4F0E947EA91091580B112309F4A7C05D
:10D0800000E09E012B593F4F44E050E06CE27BE012
:10D09000CE0189599F4F0E947EA99E012B593F4F77
:10D0A00044E050E060E37BE0CE0189599F4F0E944D
:10D0B0007EA99E012B593F4F44E050E068E27BE09F
:10D0C000CE0189599F4F0E947EA99E012B593F4F47
:10D0D00044E050E06CE47BE0CE0189599F4F0E9410
:10D0E0007EA99E012B593F4F44E050E068E47BE06D
:10D0F000CE0189599F4F0E947EA99E012B593F4F17
:10D1000040E150E064E17BE0CE0189599F4F0E94ED
:10D110007EA99E012B593F4F44E050E0BE01695A61
:10D120007F4FCE0189599F4F0E947EA99E012B59A6
:10D130003F4F4CE050E069E67BE0CE0189599F4FBC
:10D140000E947EA99E012B593F4F44E050E067EBBF
:10D1500075E1CE0189599F4F0E947EA99E012B59EE
:10D160003F4F44E050E0BE01695A7F4FCE018959DC
:10D170009F4F0E947EA901E09E012B593F4F41E045
:10D1800050E0BE0161597F4FCE0189599F4F0E94E7
:10D190007EA99E012B593F4F41E050E0BE016259EC
:10D1A0007F4FCE0189599F4F0E947EA911118AC0DD
:10D1B0006B968CAD9DADAEADBFAD6B978093BF153B
:10D1C0009093C015A093C115B093C2157BC0E19692
:10D1D0008FADE19790E0029624E33BE0E4963FAF09
:10D1E0002EAFE497B501DE011196E9EA8E2EE6E155
:10D1F0009E2EAE014F5E5F4FF9E8AF2EF6E1BF2ED7
:10D20000E896FFAEEEAEE8977E0131E2E30EF11C48
:10D2100020E030E0821793072CF0E896EEADFFADEA
:10D22000E89701C0F7014080518062807380F5016A
:10D2300041925192619271925F018217930714F0AB
:10D24000F60101C0FA014080518062807380F401D0
:10D2500041925192619271924F018217930734F07B
:10D26000FB01408051806280738005C04D905D90CD
:10D270006D907C901397E496EEADFFADE4974192EC
:10D28000519261927192E496FFAFEEAFE4972F5FF7
:10D290003F4F6C5F7F4F1496F4E0CF0ED11C4C5F74
:10D2A0005F4FE896EEADFFADE8973496E896FFAF96
:10D2B000EEAFE897F4E0EF0EF11C2430310509F0F1
:10D2C000A9CFDECEE0968FADE097853099F4AF968A
:10D2D0008FADAF97853071F400E09E012B593F4F21
:10D2E00044E650E063EC75E1CE0189599F4F0E94FE
:10D2F0007EA924C0111102C00E94B1A8E0968FAD92
:10D30000E097AF96CFACAF978C9D60011124E12CD4
:10D31000F12CEC14FD0491F000E09E012B593F4FDD
:10D3200044E050E0BE01695A7F4FCE0189599F4FBA
:10D330000E947EA92FEFE21AF20AEBCF00E09E01D5
:10D340002B593F4F44E050E0BE016D5A7F4FCE0154
:10D3500089599F4F0E947EA91AE0115079F000E090
:10D360009E012B593F4F44E050E0BE01695A7F4F68
:10D37000CE0189599F4F0E947EA9EFCF01E09E0107
:10D380002B593F4F41E050E0BE0163597F4FCE0122
:10D3900089599F4F0E947EA99E012B593F4F41E022
:10D3A00050E0BE0164597F4FCE0189599F4F0E94C2
:10D3B0007EA900E09E012B593F4F44E050E0BE01A2
:10D3C000635C7F4FCE0189599F4F0E947EA99E01C9
:10D3D0002B593F4F44E050E0BE016F5C7F4FCE01C0
:10D3E00089599F4F0E947EA9AE968FADAE97AD969C
:10D3F000CFACAD978C9D60011124E12CF12C00E0A5
:10D400009E012B593F4FCE14DF0471F044E050E0F1
:10D41000BE01695A7F4FCE0189599F4F0E947EA954
:10D420003FEFE31AF30AEBCF41E050E0BE016F5843
:10D430007F4FCE0189599F4F0E947EA99E012B5993
:10D440003F4F41E050E0BE0165597F4FCE01895901
:10D450009F4F0E947EA99E012B593F4F44E050E010
:10D46000BE01695A7F4FCE0189599F4F0E947EA904
:10D470009E012B593F4F44E050E0BE01695A7F4F57
:10D48000CE0189599F4F0E947EA99E012B593F4F83
:10D4900044E050E06BEB75E1CE0189599F4F0E944B
:10D4A0007EA99E012B593F4F44E050E0BE01615BD5
:10D4B0007F4FCE0189599F4F0E947EA99E012B5913
:10D4C0003F4F44E050E0BE01655B7F4FCE0189597C
:10D4D0009F4F0E947EA99E012B593F4F44E050E090
:10D4E000BE01695B7F4FCE0189599F4F0E947EA983
:10D4F00010E000E09E012B593F4F44E050E0BE0198
:10D50000695A7F4FCE0189599F4F0E947EA9111100
:10D5100010C06B96CCACDDACEEACFFAC6B9720E0F2
:10D5200030E84BE355E4C701B6010E9464C58111A0
:10D5300003C054E0F52E33C08091580B811108C010
:10D54000C0924A15D0924B15E0924C15F0924D15B1
:10D5500000E09E012B593F4F44E050E066E475E146
:10D56000CE0189599F4F0E947EA99E012B593F4FA2
:10D5700044E050E06EE475E1CE0189599F4F0E946E
:10D580007EA99E012B593F4F44E050E0BE01695AED
:10D590007F4FCE0189599F4F0E947EA912C0FA94F5
:10D5A000FF2079F000E09E012B593F4F44E050E00E
:10D5B000BE01695A7F4FCE0189599F4F0E947EA9B3
:10D5C000EECF1F5F153009F094CF00E09E012B597C
:10D5D0003F4F42E050E0BE016D597F4FCE01895967
:10D5E0009F4F0E947EA99E012B593F4F44E050E07F
:10D5F000BE01695A7F4FCE0189599F4F0E947EA973
:10D600006B96CCACDDACEEACFFAC6B9720E030E8B9
:10D610004BE355E4C701B6010E9464C5882329F194
:10D620008091580B811108C0C0924215D0924315C9
:10D63000E0924415F092451500E09E012B593F4FB2
:10D6400044E050E06EE375E1CE0189599F4F0E949E
:10D650007EA99E012B593F4F44E050E06AE375E1FB
:10D66000CE0189599F4F0E947EA900E09E012B594F
:10D670003F4F42E050E0BE016F597F4FCE018959C4
:10D680009F4F0E947EA99E012B593F4F41E050E0E1
:10D69000BE016F587F4FCE0189599F4F0E947EA9CE
:10D6A00019E0115000E09E012B593F4F112359F012
:10D6B00044E050E0BE01695A7F4FCE0189599F4F27
:10D6C0000E947EA9EECF41E050E067E276E1CE0114
:10D6D00089599F4F0E947EA9F12C00E09E012B5991
:10D6E0003F4F44E050E0BE01695A7F4FCE01895957
:10D6F0009F4F0E947EA91091580B111110C0F1107C
:10D700000EC06B968CAD9DADAEADBFAD6B978093EB
:10D710002C1690932D16A0932E16B0932F16F394DB
:10D7200085E0F812DACF111102C00E94E0424CE00D
:10D73000F42EFA94F11003C03CE0F32E0FC000E089
:10D740009E012B593F4F42E050E0BE01615A7F4F8E
:10D75000CE0189599F4F0E947EA9EBCFFA9400E039
:10D760009E012B593F4FFF2059F044E050E0BE018D
:10D770006D5B7F4FCE0189599F4F0E947EA9EECFEE
:10D7800046E050E0BE01635C7F4FCE0189599F4F58
:10D790000E947EA99E012B593F4F44E050E064E275
:10D7A0007BE0CE0189599F4F0E947EA99E012B5993
:10D7B0003F4F4CE050E0BE016F5C7F4FCE01895976
:10D7C0009F4F0E947EA92CE1F22EFA94F11003C023
:10D7D00094E0F92E1DC000E09E012B593F4F44E01C
:10D7E00050E0BE01695A7F4FCE0189599F4F0E9478
:10D7F0007EA9EBCF00E09E012B593F4F44E050E063
:10D80000BE01695A7F4FCE0189599F4F0E947EA960
:10D81000FA94F110EFCF8BE0F82EFA94FF2079F014
:10D8200000E09E012B593F4F44E050E0BE01695A91
:10D830007F4FCE0189599F4F0E947EA9EECFA996B6
:10D840008EAD9FADA99784569109C7DA8093570B87
:10D85000882309F1EDEEF8E184917F019FEFE91A49
:10D86000F90A882321F00E947D3DF701F5CFA996A2
:10D870006EAD7FADA9976456710985ED96E10E9462
:10D88000EE4B6BED72E08DEC96E10E94EE4B8AE080
:10D890000E947D3D99C0A7962EAD3FADA797AB9650
:10D8A0008EAD9FADAB972817390709F44BC081E0C7
:10D8B0008093570BE8EDF8E184917F012FEFE21A96
:10D8C000F20A811103C0EDEAF6E104C00E947D3D39
:10D8D000F701F2CF84917F013FEFE31AF30A882327
:10D8E00021F00E947D3DF701F5CFAB966EAD7FAD87
:10D8F000AB9780E090E04AE00E949940E8EAF6E1C8
:10D9000084917F019FEFE91AF90A882321F00E9490
:10D910007D3DF701F5CFA7966EAD7FADA79780E06F
:10D9200090E04AE00E949940E8E9F6E184917F01A5
:10D930002FEFE21AF20A882309F446C00E947D3DC7
:10D94000F701F4CF111142C0EDEEF8E184917F01AF
:10D950003FEFE31AF30A811103C007ED12E004C0A0
:10D960000E947D3DF701F2CFF80181918F0188235C
:10D9700019F00E947D3DF8CFA9966EAD7FADA997B5
:10D98000645671098BE796E10E94EE4BA7964EAD67
:10D990005FADA79760E070E08EE696E10E94B44B21
:10D9A000EBE6F6E184917F012FEFE21AF20A811192
:10D9B00007C08091570B811109C00E943DAA06C083
:10D9C0000E947D3DF701EECF112399F3E6968EADCF
:10D9D0009FADE6970FB6F8949EBF0FBE8DBF8091A6
:10D9E000580B811102C00E944D9D9091570B81E010
:10D9F00089270FB6F8943EBE0FBE2DBEC958DF4F23
:10DA00000FB6F894DEBF0FBECDBFDF91CF911F914F
:10DA10000F91FF90EF90DF90CF90BF90AF909F90CD
:10DA20008F907F906F905F904F903F902F900895D0
:10DA300081E08093580BF2D91092580B8111EEC9F6
:10DA40000E94E1A181E008958F929F92AF92BF92D0
:10DA5000CF92DF92EF92FF920F931F93CF93DF93BA
:10DA6000CDB7DEB7CA5AD1090FB6F894DEBF0FBEE4
:10DA7000CDBFE9961CAE1DAE1EAE1FAEE9978091DC
:10DA80008C0390918D03A0918E03B0918F03ED963E
:10DA90008CAF9DAFAEAFBFAFED97C556DF4F1982CC
:10DAA0001882CB59D04084E690E0C356DF4F99836B
:10DAB0008883CD59D0401092570B9E0125563F4F79
:10DAC00044E050E0BE0167587F4FCE0183569F4F20
:10DAD0000E94CAA9C356DF4F88819981CD59D04091
:10DAE0000296C356DF4F99838883CD59D040C556DF
:10DAF000DF4F19821882CB59D04081E0CD55DF4FDE
:10DB00008883C35AD0409E0125563F4F41E050E0E4
:10DB1000BE016D557F4FCE0183569F4F0E94CAA90B
:10DB20009E0125563F4F40E150E069E876E1CE0185
:10DB300083569F4F0E94CAA99E0125563F4F44E03D
:10DB400050E064E47BE0CE0183569F4F0E94CAA957
:10DB50009E0125563F4F40E150E069EA76E1CE0153
:10DB600083569F4F0E94CAA99E0125563F4F40E110
:10DB700050E064E37BE0CE0183569F4F0E94CAA928
:10DB80009E0125563F4F44E050E06CE27BE0CE0121
:10DB900083569F4F0E94CAA99E0125563F4F44E0DD
:10DBA00050E060E37BE0CE0183569F4F0E94CAA9FC
:10DBB0009E0125563F4F44E050E068E27BE0CE01F5
:10DBC00083569F4F0E94CAA99E0125563F4F44E0AD
:10DBD00050E06CE47BE0CE0183569F4F0E94CAA9BF
:10DBE0009E0125563F4F44E050E068E47BE0CE01C3
:10DBF00083569F4F0E94CAA99E0125563F4F40E180
:10DC000050E064E17BE0CE0183569F4F0E94CAA999
:10DC10008AE097EDA3EABCE3E9968CAF9DAFAEAF87
:10DC2000BFAFE9979E0125563F4F44E050E0BE014B
:10DC30006B587F4FCE0183569F4F0E94CAA99E0109
:10DC400025563F4F4CE050E069E67BE0CE0183561D
:10DC50009F4F0E94CAA980913C1690913D16A091B9
:10DC60003E16B0913F16C358DF4F88839983AA832D
:10DC7000BB83CD57D0409E0125563F4F44E050E036
:10DC8000BE0163587F4FCE0183569F4F0E94CAA9A1
:10DC900085E0CC55DF4F8883C45AD040CB55DF4F49
:10DCA0008883C55AD0409E0125563F4F44E050E03E
:10DCB0006FEB75E1CE0183569F4F0E94CAA99E016A
:10DCC00025563F4F41E050E0BE016C557F4FCE01DD
:10DCD00083569F4F0E94CAA99E0125563F4F41E09F
:10DCE00050E0BE016B557F4FCE0183569F4F0E947F
:10DCF000CAA99E0125563F4F44E650E063EC75E10A
:10DD0000CE0183569F4F0E94CAA9CF57DF4F18827A
:10DD100019821A821B82C158D0409E0125563F4F5E
:10DD200044E050E0BE016F577F4FCE0183569F4FB6
:10DD30000E94CAA9E9961CAE1DAE1EAE1FAEE997A1
:10DD40001AE0115071F09E0125563F4F44E050E01B
:10DD5000BE016B587F4FCE0183569F4F0E94CAA9C8
:10DD6000F0CF83E0CA55DF4F8883C65AD040C955EB
:10DD7000DF4F8883C75AD040CB57DF4F18821982B4
:10DD80001A821B82C558D040C757DF4F18821982AC
:10DD90001A821B82C958D040E9961CAE1DAE1EAE39
:10DDA0001FAEE9979E0125563F4F41E050E0BE016E
:10DDB0006A557F4FCE0183569F4F0E94CAA99E018C
:10DDC00025563F4F41E050E0BE0169557F4FCE01DF
:10DDD00083569F4F0E94CAA99E0125563F4F44E09B
:10DDE00050E0BE0167577F4FCE0183569F4F0E9480
:10DDF000CAA99E0125563F4F44E050E0BE016B5733
:10DE00007F4FCE0183569F4F0E94CAA90AE010E0BF
:10DE10000150110971F09E0125563F4F44E050E03A
:10DE2000BE016B587F4FCE0183569F4F0E94CAA9F7
:10DE3000EFCFC855DF4F1882C85AD0408FEFC75573
:10DE4000DF4F8883C95AD0409E0125563F4F41E09D
:10DE500050E0BE0168557F4FCE0183569F4F0E9410
:10DE6000CAA99E0125563F4F41E050E0BE016755CB
:10DE70007F4FCE0183569F4F0E94CAA9E9961CAEE0
:10DE80001DAE1EAE1FAEE9979E0125563F4F44E0E2
:10DE900050E0BE016B587F4FCE0183569F4F0E94CA
:10DEA000CAA99E0125563F4F44E050E0BE016B5881
:10DEB0007F4FCE0183569F4F0E94CAA99E012556CF
:10DEC0003F4F44E050E06BEB75E1CE0183569F4F2E
:10DED0000E94CAA98091830290918402A091850238
:10DEE000B0918602C357DF4F88839983AA83BB838F
:10DEF000CD58D0408091870290918802A0918902EC
:10DF0000B0918A02CF56DF4F88839983AA83BB835F
:10DF1000C159D040CB56DF4F19821882C559D04025
:10DF2000C956DF4F19821882C759D0409E01255625
:10DF30003F4F44E050E0BE0163577F4FCE01835610
:10DF40009F4F0E94CAA99E0125563F4F44E050E0D2
:10DF5000BE016F567F4FCE0183569F4F0E94CAA9C4
:10DF60009E0125563F4F44E050E0BE016B567F4F67
:10DF7000CE0183569F4F0E94CAA910E0C12C80E8B1
:10DF8000D82E8BE3E82E85E4F82E812C912C90E896
:10DF9000A92E9FE3B92E111138C09E0125563F4F7F
:10DFA00044E050E06AE475E1CE0183569F4F0E9441
:10DFB000CAA99E0125563F4F44E050E066E475E152
:10DFC000CE0183569F4F0E94CAA99E0125563F4FFE
:10DFD00044E050E06EE475E1CE0183569F4F0E940D
:10DFE000CAA9E9968CAE9DAEAEAEBFAEE9979E01D2
:10DFF00025563F4F44E050E0BE016B587F4FCE01A5
:10E0000083569F4F0E94CAA92AC0E996CCAEDDAEC6
:10E01000EEAEFFAEE9979E0125563F4F44E050E03B
:10E02000BE016B587F4FCE0183569F4F0E94CAA9F5
:10E03000E9961CAE1DAE1EAE1FAEE99704E001507E
:10E0400071F09E0125563F4F44E050E0BE016B58F1
:10E050007F4FCE0183569F4F0E94CAA9F0CF1F5F0A
:10E06000153009F098CF84E190E0C156DF4F9983D5
:10E070008883CF59D0409E0125563F4F42E050E063
:10E08000BE0161567F4FCE0183569F4F0E94CAA9A1
:10E090009E0125563F4F44E050E062E475E1CE0119
:10E0A00083569F4F0E94CAA99E0125563F4F44E0C8
:10E0B00050E06EE375E1CE0183569F4F0E94CAA9DE
:10E0C0009E0125563F4F44E050E06AE375E1CE01E2
:10E0D00083569F4F0E94CAA980E290E0CF55DF4F40
:10E0E00099838883C15AD0409E0125563F4F42E014
:10E0F00050E0BE016F557F4FCE0183569F4F0E9467
:10E10000CAA9C655DF4F1882CA5AD04080E2EBE850
:10E11000F2E0DE019D9601900D928A95E1F79E0155
:10E1200025563F4F41E050E0BE0166557F4FCE017E
:10E1300083569F4F0E94CAA99E0125563F4F40E239
:10E1400050E0BE01635D7F4FCE0183569F4F0E941A
:10E15000CAA99E0125563F4F41E050E067E276E1B3
:10E16000CE0183569F4F0E94CAA910E011110EC024
:10E1700080912C1690912D16A0912E16B0912F16ED
:10E18000E9968CAF9DAFAEAFBFAFE9979E01255624
:10E190003F4F44E050E0BE016B587F4FCE018356A5
:10E1A0009F4F0E94CAA91F5F153001F7BE01635B34
:10E1B0007F4F86E1FB0111928A95E9F79E01255672
:10E1C0003F4F46E150E0CE0183569F4F0E94CAA9BF
:10E1D0008CE2EBEAF2E0DE01119601900D928A9555
:10E1E000E1F79E0125563F4F4CE250E0BE016F5FC4
:10E1F0007F4FCE0183569F4F0E94CAA9BE0161592D
:10E200007F4F86E0FB0111928A95E9F79E01255622
:10E210003F4F46E050E0CE0183569F4F0E94CAA96F
:10E220009E0125563F4F44E050E064E27BE0CE0182
:10E2300083569F4F0E94CAA9BE016D597F4F8CE043
:10E24000FB0111928A95E9F79E0125563F4F4CE05C
:10E2500050E0CE0183569F4F0E94CAA9E9961CAE9A
:10E260001DAE1EAE1FAEE9971CE1115071F09E016C
:10E2700025563F4F44E050E0BE016B587F4FCE0122
:10E2800083569F4F0E94CAA9F0CFE9961CAE1DAEDF
:10E290001EAE1FAEE99714E0115071F09E01255695
:10E2A0003F4F44E050E0BE016B587F4FCE01835694
:10E2B0009F4F0E94CAA9F0CFE9961CAE1DAE1EAEBC
:10E2C0001FAEE9971BE0115071F09E0125563F4F9C
:10E2D00044E050E0BE016B587F4FCE0183569F4F04
:10E2E0000E94CAA9F0CF8091570B811167C0C35615
:10E2F000DF4FE880F980CD59D040F4E6EF1AF108FD
:10E30000C556DF4F88819981CB59D040C756DF4F22
:10E3100099838883C959D04084E690E0C356DF4F83
:10E3200099838883CD59D0409E0125563F4F44E0C4
:10E3300050E067ED72E0CE0183569F4F0E94CAA95C
:10E340009E0125563F4F42E050E0BE0167567F4F89
:10E35000CE0183569F4F0E94CAA9EDEEF8E1849149
:10E360008F010F5F1F4F882321F00E947D3DF80130
:10E37000F6CFB70189E596E10E94EE4BC756DF4F15
:10E3800048815981C959D04060E070E08CE496E141
:10E390000E94B44BE9E4F6E184918F010F5F1F4FB7
:10E3A000882321F00E947D3DF801F6CFC7010E942D
:10E3B000ED669091570B892B8093570B9091570BDB
:10E3C00081E08927C655DF4F0FB6F894DEBF0FBE38
:10E3D000CDBFDF91CF911F910F91FF90EF90DF9014
:10E3E000CF90BF90AF909F908F900895CF92DF9283
:10E3F000EF92FF920F931F93CF93DF936C017A01FB
:10E400008B01C0E0D0E0CE15DF0581F0D8016D9121
:10E410008D01D601ED91FC910190F081E02DC601B6
:10E420001995892B11F02196EECF7E01C701DF915E
:10E43000CF911F910F91FF90EF90DF90CF900895B3
:10E440000E94BACC1F920F920FB60F9211240BB6F6
:10E450000F922F933F934F935F936F937F938F937D
:10E460009F93AF93BF93EF93FF9380915C0B909139
:10E470005D0BA0915E0BB0915F0B892B8A2B8B2BD0
:10E4800059F190915B0BE091590BF0915A0B8081FF
:10E490008927808380915C0B90915D0BA0915E0B2E
:10E4A000B0915F0B181619061A061B060CF056C021
:10E4B00080915C0B90915D0BA0915E0BB0915F0B16
:10E4C0000197A109B10980935C0B90935D0BA09318
:10E4D0005E0BB0935F0B42C080913902EDE0F7E133
:10E4E000E4919FEF90933902E230C9F050F4EE23AB
:10E4F00099F0E13081F590916F009D7F90936F00CE
:10E500002AC0E43019F1E0F0E53029F5909173006C
:10E510009D7F909373001FC010926E001CC090915D
:10E5200070009D7F9093700091E09093B000909167
:10E53000B100987F94609093B1001092B3000BC02B
:10E54000909171009D7F9093710005C09091720031
:10E550009D7F9093720060E00E9489B1FF91EF91DE
:10E56000BF91AF919F918F917F916F915F914F91EB
:10E570003F912F910F900BBE0F900FBE0F901F90E9
:10E5800018959093D6038093D50380E00C94E77A96
:10E590008F929F92AF92BF92CF92DF92EF92FF92B3
:10E5A0001F93CF93DF93C82F8BE291E19093070FD6
:10E5B0008093060F1092471182E090E0A0E0B0E057
:10E5C0008093301190933111A0933211B093331195
:10E5D0001092050F1092010F1092020F1092030F6C
:10E5E0001092040F8FEF9FEFDC018093FD0E90934C
:10E5F000FE0EA093FF0EB093000FCC2379F1C5302F
:10E6000008F0F8C040E060E070E0CB010E9424AB6D
:10E61000882309F4EFC020E1C29FC0011124835177
:10E62000934FFC01E254FE4F20812F7709F0E2C0A6
:10E630003C96408151816281738144365105610568
:10E64000710508F4D7C03497C080D180E280F38090
:10E65000C114D104E104F10421F4CCC0C12CD12CAB
:10E66000760140E0C701B6010E9424AB182F882331
:10E6700009F4C0C08091080D9091090D8115924058
:10E6800009F0B8C0A0910D0DAA2309F4B3C06091A0
:10E690000B0D70910C0D6115710509F4ABC0209143
:10E6A0000A0D222309F4A6C0A0934211209334112D
:10E6B00080E030E041E050E0C82FFA01082E02C0AF
:10E6C000EE0FFF1F0A94E2F72E173F0739F08F5F16
:10E6D000C83091F789E080933D118CC080933D1143
:10E6E0002091130D3091140D2115310519F040E0E2
:10E6F00050E008C02091210D3091220D4091230D52
:10E700005091240D209335113093361140933711D9
:10E710005093381146015701860E971EA11CB11C5B
:10E720008092431190924411A0924511B0924611EB
:10E73000E0910E0DF0910F0DF0934911E093481107
:10E74000B0E00E9474C9860E971EA81EB91E809262
:10E750004A1190924B11A0924C11B0924D1185E04C
:10E76000EE0FFF1F8A95E1F7E150FE4FEF2FFF27D5
:10E77000E6958E0E9F1EA11CB11C80923E119092B8
:10E780003F11A0924011B09241112091100D309193
:10E79000110D2115310521F0A90160E070E008C0DC
:10E7A00040911D0D50911E0D60911F0D7091200D17
:10E7B000D701C60188199909AA09BB09840F951FB9
:10E7C000A61FB71F04C0B695A79597958795CA95BC
:10E7D000D2F78093391190933A11A0933B11B093E3
:10E7E0003C11853F2FE09207A105B10528F48CE08C
:10E7F0008093471110E01AC0853F9F4FA105B105D6
:10E8000010F480E111C08091290D90912A0DA09102
:10E810002B0DB0912C0D80934A1190934B11A09326
:10E820004C11B0934D1180E280934711812FDF91FD
:10E83000CF911F91FF90EF90DF90CF90BF90AF905E
:10E840009F908F900895682F82EF94E10C94013887
:10E85000CF92DF92EF92FF921F93CF93DF931092AC
:10E860008A0F8091BD0F882321F08AEB9FE00E94E0
:10E87000C58E10922F1110922C1185E380932B11CD
:10E880000E94F2B2EB01A89561E080912B110E94E9
:10E89000B7B18BE291E10E9426902398229A219AA7
:10E8A000209A289A85E080932D1182E58CBD1DBCAD
:10E8B0001AE08FEF0E942B901150D9F720E030E042
:10E8C000A90160E08BE291E10E943090182F8093C3
:10E8D0002E11813049F00E94F2B26C1B7D0B613D1C
:10E8E000774060F381E054C02AEA31E040E050E034
:10E8F00068E08BE291E10E94309082FF03C01093A8
:10E900002F110EC014E00E94824C80932E111150E2
:10E91000D1F78A3A11F082E03BC082E080932F1158
:10E9200080912F11823021F0C12CD12C760105C0AD
:10E93000C12CD12CE12C80E4F82E20E030E0A9019C
:10E9400067E38BE291E10E943090A701960169E2B2
:10E950008BE291E10E94309080932E11882349F040
:10E960000E94F2B26C1B7D0B613D774030F38AE070
:10E970000FC080912F11823011F520E030E0A90105
:10E980006AE38BE291E10E943090882351F088E0A5
:10E9900080932C118BE291E10E942690EDEEF8E13C
:10E9A00019C00E94824C807C803C19F483E08093E3
:10E9B0002F110E94824C0E94824C0E94824C8BE25A
:10E9C00091E10E94269010922D1181E0E1DD8111EC
:10E9D00031C015C08491EF012196882321F00E9457
:10E9E0007D3DFE01F7CFEFEDF8E18491EF01219637
:10E9F000882309F456C00E947D3DFE01F6CF80E0D9
:10EA0000C7DD811117C0E8EDF8E18491EF0121968F
:10EA1000882321F00E947D3DFE01F7CFE4ECF8E170
:10EA20008491EF012196882309F43BC00E947D3D2B
:10EA3000FE01F6CF60E371E18AEB9FE00E94728EE7
:10EA4000811116C0E8EDF8E18491EF012196882349
:10EA500021F00E947D3DFE01F7CFE3EBF8E18491C8
:10EA6000EF0121968823E9F00E947D3DFE01F7CF5A
:10EA700081E080938A0FEDEEF8E18491EF01219619
:10EA8000882321F00E947D3DFE01F7CFE7EAF8E1FF
:10EA90008491EF012196882321F00E947D3DFE01A3
:10EAA000F7CF8BE1EAEBFFE0A9EDBFE001900D921B
:10EAB0008A95E1F78091B80F9091B90F9093D80F94
:10EAC0008093D70FDF91CF911F91FF90EF90DF9050
:10EAD000CF90089580919713823041F482E998E1B4
:10EAE0009093FC0C8093FB0C0E94A93D0E94F2B213
:10EAF00060939B1370939C1380939D1390939E132C
:10EB000080918A0F882319F081E08093890F81E03A
:10EB1000809397130895CF93DF931092890F83E02A
:10EB2000809397138091E4138823B1F0EAE8F8E129
:10EB30008491EF01882341F0082E000C990B83DEAD
:10EB40002196FE018491F6CF8DE090E07CDE8AE094
:10EB500090E0DF91CF9177CEEEE8F8E18491EF017C
:10EB6000882391F3082E000C990B6DDE2196FE018F
:10EB70008491F6CF8F929F92AF92BF92CF92DF9205
:10EB8000EF92FF920F931F93CF93DF9300D01F92CA
:10EB9000CDB7DEB7FC018381813079F5818181FFBA
:10EBA0002CC081899289A389B489892B8A2B8B2BCC
:10EBB00009F448C07F0140E050E0BA01CF010E9453
:10EBC000DB8D8823D1F0F70185889688A788B08CE3
:10EBD000C18CD28C82E090E0A0E0B0E0F6018083AE
:10EBE0009183A283B3839E012F5F3F4FB501A401A0
:10EBF000C6010E94EDAB811102C080E03CC000E084
:10EC000010E09801B501A401C6010E945CAB882305
:10EC1000A1F389809A80AB80BC80F601878980311E
:10EC200041F4F8EF8F16FFEF9F06A104B10460F4E2
:10EC3000DACF88EF88168FEF9806A8068FE0B8061F
:10EC400018F4D1CF81E017C0F701158A168A178A08
:10EC5000108E118A128A138A148A818180688183B6
:10EC6000C7010E943BAD882341F240E050E0BA0169
:10EC7000C7010E94DB8D0F900F900F900F90DF91D6
:10EC8000CF911F910F91FF90EF90DF90CF90BF90A9
:10EC9000AF909F908F90089510928C0F1092890FD3
:10ECA00080915511882321F082E591E10C94C58E65
:10ECB00008952F923F924F925F926F927F928F9220
:10ECC0009F92AF92BF92CF92DF92EF92FF920F93FB
:10ECD0001F93CF93DF93CDB7DEB7C257D1090FB6DD
:10ECE000F894DEBF0FBECDBF8C013B014A014DB78A
:10ECF0005EB7E1965FAF4EAFE197AD961FAEAD97B1
:10ED00001B0154E0250E311C7E018FE5E80EF11C3D
:10ED100095EE492E92E0592EE0E4F0E0EC0FFD1F55
:10ED20003496E396FFAFEEAFE397F301878182302D
:10ED300008F462C184859585A685B7858F7199276A
:10ED4000AA27BB27892B8A2B8B2B09F055C1109240
:10ED50009A0F4AE95FE0BE016F5F7F4FC1010E94D9
:10ED6000D3AC18160CF048C18C85982F987190314F
:10ED700029F4209107122150223078F4298122238E
:10ED800009F43AC1253E89F22E3279F220919A0F88
:10ED90002E3259F28A7049F6B8C04DB75EB7AF96B9
:10EDA0005FAF4EAFAF97BE016F5F7F4FC7010E944D
:10EDB000CEAA0115110521F0F801808181119BC0B7
:10EDC00021E081E090E0F70101900020E9F7319720
:10EDD000EE19FF098E0F9F1F02964DB75EB7481BB5
:10EDE000590B0FB6F8945EBF0FBE4DBF8DB79EB7DF
:10EDF00001965C01211102C0B80102C06AE173E012
:10EE0000C5010E940ECDB701C5010E94EFCC6AE199
:10EE100073E0C5010E94EFCC25961FAE259728967A
:10EE20001FAE289724961FAE1EAE249722965FAE83
:10EE30004EAE229721E0A701B101E3968EAD9FADC2
:10EE4000E3970E94589481112AC080910712811182
:10EE500026C0EDEEF8E184916F019FEFC91AD90A3F
:10EE6000882321F00E947D3DF601F5CFE6E7F8E129
:10EE700084916F012FEFC21AD20A882321F00E94D9
:10EE80007D3DF601F5CF6701F60181916F01882381
:10EE900019F00E947D3DF8CF8AE00E947D3D8BE114
:10EEA000FE01EC5BFF4FDE01959601900D928A9575
:10EEB000E1F724968EAD9FAD24979CA38BA35AA215
:10EEC00049A240E050E0BE016F5D7F4FC501F1DE19
:10EED000CE0181960E94544ECE01805C9F4F0E94CD
:10EEE000544EAF964EAD5FADAF970FB6F8945EBF80
:10EEF0000FBE4DBF1ACFF80101900020E9F73197FE
:10EF0000CF01801B910B20E05ECF81E0903109F0B2
:10EF100080E080938B0F903141F08985873409F030
:10EF200004CF8A858E3709F400CF80910712813093
:10EF300029F08230D9F18111F8CE0AC080910812EF
:10EF40009091091201969093091280930812EDCEC8
:10EF5000BE016F5F7F4F8DE89FE00E94CEAA011532
:10EF6000110529F48DE8C82E8FE0D82E09C068015C
:10EF7000F60181916F018823A9F30E947D3DF8CFAE
:10EF8000F60181916F01882319F00E947D3DF8CF31
:10EF900080E20E947D3D6D8D7E8D8F8D98A14AE02F
:10EFA0000E9499408AE00E947D3DBFCEBE016F5F06
:10EFB0007F4F8DE89FE00E94CEAA8114910441F01A
:10EFC0006DE87FE0C4010E94DCCC892B69F414C099
:10EFD000AD96FFADAD978F2F90E020911415309135
:10EFE00015158217930741F0AD962FADAD972F5FA2
:10EFF000AD962FAFAD9799CEE1968EAD9FADE197CF
:10F000000FB6F8949EBF0FBE8DBFCE58DF4F0FB620
:10F01000F894DEBF0FBECDBFDF91CF911F910F914E
:10F02000FF90EF90DF90CF90BF90AF909F908F9028
:10F030007F906F905F904F903F902F9008950F9327
:10F040001F93CF93DF93CDB7DEB76F970FB6F894CA
:10F05000DEBF0FBECDBF8B0122E02093071290933D
:10F0600015158093141589ED9FE00E9422908BE185
:10F07000E9EDFFE0DE01159601900D928A95E1F72A
:10F080008091D70F9091D80F9C838B8385EE92E06F
:10F090009A838983A801BE016F5F7F4F80E090E073
:10F0A00008DECE0101960E94544E6F960FB6F8947A
:10F0B000DEBF0FBECDBFDF91CF911F910F9108959D
:10F0C0002F923F924F925F926F927F928F929F9278
:10F0D000AF92BF92CF92DF92EF92FF920F931F9366
:10F0E000CF93DF93CDB7DEB76F970FB6F894DEBF3F
:10F0F0000FBECDBF6C012DB63EB61D8218861C8298
:10F100001B8285EE92E09A838983FB0180819E01B8
:10F110002F5F3F4F39018F3241F085ED9FE0F601BF
:10F1200091838083F62E172F64C086EB9FE0F60153
:10F13000918380838B010F5F1F4F0115110509F427
:10F1400056C04DB65EB66FE270E0C8010E94FACCC0
:10F150004C010817190708F048C07C01E01AF10AB1
:10F16000FF24C70101962DB73EB7281B390B0FB6F8
:10F17000F8943EBF0FBE2DBF8DB79EB701965C01C0
:10F18000A701B8010E9423CDF501EE0DFF1D1082ED
:10F19000F601608171816115710511F06C5F7F4F1F
:10F1A00021E0A501CE0105960E945894811111C05D
:10F1B000B50182E698E10E94074C8EE20E947D3DF7
:10F1C0008AE00E947D3D0FB6F8945EBE0FBE4DBE34
:10F1D0000EC0F6017182608284010F5F1F4F0FB66F
:10F1E000F8945EBE0FBE4DBEA8CFF02E02C0F12C2B
:10F1F00010E0C3010E94544E8F2D912F0FB6F8944A
:10F200003EBE0FBE2DBE6F960FB6F894DEBF0FBE8A
:10F21000CDBFDF91CF911F910F91FF90EF90DF90C5
:10F22000CF90BF90AF909F908F907F906F905F90A6
:10F230004F903F902F900895FF920F931F93CF937D
:10F24000DF938C01EB01F42E80E20E947D3D8FEF75
:10F25000F81611F084E501C082E40E947D3D8AE346
:10F260000E947D3DF801608171818281938142E03D
:10F270000E941E41488159816A817B818EE89BE111
:10F280000E94D14B62E070E080E090E0DF91CF918E
:10F290001F910F91FF900C94BAB28F929F92AF92F0
:10F2A000BF92CF92DF92EF92FF920F931F93CF9373
:10F2B000DF93F0E2FF2EE12CAE2DB0E0BD016F0D2B
:10F2C000711D759567956E1511F0F6120BC0E1E78B
:10F2D000F9E165917491072E000C880B990B0E943F
:10F2E0006AC562C09B0121503109220F331F220FD2
:10F2F000331FF901ED50F74E05911491AB01440F06
:10F30000551F440F551FFA01ED50F74EC591D4918A
:10F310008017910714F4F62ED1CFC817D90714F42B
:10F32000E62ECACFF901EB50F74EE590F490FA01C2
:10F33000EB50F74EC590D490BC01601B710B072EAB
:10F34000000C880B990B0E946AC54B015C01B60149
:10F350006E197F09072E000C880B990B0E946AC555
:10F360009B01AC01C501B4010E94C9C54B015C0100
:10F37000C01BD10BBE01DD0F880B990B0E946AC523
:10F380009B01AC01C501B4010E946ACA4B015C013A
:10F39000B701FF0C880B990B0E946AC59B01AC0159
:10F3A000C501B4010E948EC9DF91CF911F910F91C9
:10F3B000FF90EF90DF90CF90BF90AF909F908F9095
:10F3C00008950F931F93CF93DF93CDB7DEB72897A0
:10F3D0000FB6F894DEBF0FBECDBF6091D50370911C
:10F3E000D603072E000C880B990B0E946AC56D830B
:10F3F0007E838F8398878091D7039091D803A091C3
:10F40000D903B091DA0389839A83AB83BC834DEF30
:10F41000BE016B5F7F4FCE0101960EDF6091CF037F
:10F420007091D003072E000C880B990B0E946AC5BF
:10F430006D837E838F8398878091D1039091D203CF
:10F44000A091D303B091D40389839A83AB83BC8307
:10F450004FEFBE016B5F7F4FCE010196EDDEE6E917
:10F46000FBE184918F010F5F1F4F882321F00E94E1
:10F470007D3DF801F6CFE0915C15F0E0E65AFA4EDA
:10F48000608170E080E090E00E940441E1E9FBE1EE
:10F4900084918F010F5F1F4F882321F00E947D3DD3
:10F4A000F801F6CF60915B1570E080E090E00E947B
:10F4B000044128960FB6F894DEBF0FBECDBFDF9192
:10F4C000CF911F910F9108950F930FB70F93009154
:10F4D0006E000B7F00936E0078940F930BB70F9321
:10F4E0000CB70F921F922F933F934F935F936F939D
:10F4F0007F938F939F93AF93BF93EF93FF931124C9
:10F50000DAD2FF91EF91BF91AF919F918F917F914F
:10F510006F915F914F913F912F911F900F900CBF72
:10F520000F910BBF0F910460F89400936E000F9140
:10F530000FBF0F911895CF92DF92EF92FF92C0907C
:10F54000D103D090D203E090D303F090D403609124
:10F55000CF037091D00366507109072E000C880B01
:10F56000990B0E946AC59B01AC01C701B6010E94BC
:10F5700064C587FF1FC020E030E040E050E4C701D1
:10F58000B6010E948EC90E94D7CA709394156093E9
:10F5900093150E94F2B2DC01CB01805A9541AF4F26
:10F5A000BF4F80938F1590939015A0939115B093B2
:10F5B000921508C010928F15109290151092911507
:10F5C00010929215FF90EF90DF90CF900895CF9218
:10F5D000DF92EF92FF92C090D703D090D803E090D3
:10F5E000D903F090DA036091D5037091D603665089
:10F5F0007109072E000C880B990B0E946AC59B01AC
:10F60000AC01C701B6010E9464C587FF1FC020E09E
:10F6100030E040E050E4C701B6010E948EC90E946C
:10F62000D7CA70938E1560938D150E94F2B2DC01DB
:10F63000CB01805E914BAF4FBF4F80938915909364
:10F640008A15A0938B15B0938C1508C0109289155C
:10F6500010928A1510928B1510928C15FF90EF90D6
:10F66000DF90CF9008958F929F92AF92BF92CF92EA
:10F67000DF92EF92FF920F931F93CF93DF93F0E40B
:10F68000FF2EE12CAE2DB0E0BD016F0D711D759503
:10F6900067956E1511F0F6120BC0E3EEFAE1659175
:10F6A0007491072E000C880B990B0E946AC562C0EA
:10F6B0009B0121503109220F331F220F331FF90103
:10F6C000EB51F64E05911491AB01440F551F440FB9
:10F6D000551FFA01EB51F64EC591D4918017910751
:10F6E00014F4F62ED1CFC817D90714F4E62ECACFDA
:10F6F000F901E951F64EE590F490FA01E951F64E20
:10F70000C590D490BC01601B710B072E000C880BB8
:10F71000990B0E946AC54B015C01B6016E197F0905
:10F72000072E000C880B990B0E946AC59B01AC0147
:10F73000C501B4010E94C9C54B015C01C01BD10BBE
:10F74000BE01DD0F880B990B0E946AC59B01AC01BD
:10F75000C501B4010E946ACA4B015C01B701FF0CEC
:10F76000880B990B0E946AC59B01AC01C501B401CD
:10F770000E948EC9DF91CF911F910F91FF90EF9062
:10F78000DF90CF90BF90AF909F908F90089560E0F2
:10F7900080919F159091A01580DD6093D7037093A1
:10F7A000D8038093D9039093DA0380919D159091AB
:10F7B0009E1559DF6093D1037093D2038093D303D6
:10F7C0009093D403A8951092571508957F928F9225
:10F7D0009F92AF92BF92CF92DF92EF92FF920F93E0
:10F7E0001F93CF93DF9320E030E048E452E4609130
:10F7F000D7037091D8038091D9039091DA030E94C6
:10F80000B4CB18164CF4E9E7F9E1E491C1E001C08A
:10F81000CC0FEA95EAF701C0C0E083E7E82E89E162
:10F82000F82E09E719E196E0A92E912CD0E0CC241E
:10F83000C394D12CF7017490F801849077FC23C015
:10F84000892D90E0082C02C0959587950A94E2F7DF
:10F8500080FD19C0BE01082C02C0759567950A94F9
:10F86000E2F76170B62EB1946B2D872D0E9489B19D
:10F870006B2D70E0872D0E94F3B1C60101C0880F87
:10F880008A94EAF7982AAA94FFEFEF1AFF0A0F5F0B
:10F890001F4FA110CFCFDF91CF911F910F91FF90FC
:10F8A000EF90DF90CF90BF90AF909F908F907F9020
:10F8B00008950F931F9380913915813019F40E9498
:10F8C000F2B208C0609135157091361580913715E8
:10F8D0009091381500916115109162152091631572
:10F8E00030916415601B710B820B930B28EE33E093
:10F8F00040E050E00E9452C980915D1590915E15E4
:10F90000A0915F15B0916015BC01CD01620F731F0E
:10F91000841F951F1F910F91089510923915109211
:10F920006115109262151092631510926415109271
:10F930003515109236151092371510923815109211
:10F940005D1510925E1510925F1510926015089566
:10F95000809139158130E1F0823051F4AADF609353
:10F960005D1570935E1580935F159093601501C0CF
:10F97000D4DF81E0809339150E94F2B26093611563
:10F9800070936215809363159093641581E00895D8
:10F9900080E00895809139158150823010F080E028
:10F9A0000895109239150E94F2B260933515709344
:10F9B0003615809337159093381581E0089510928D
:10F9C000561580E090E00E94C1721092D003109210
:10F9D000CF03B1DDDFDF80E090E00E94C1721092C2
:10F9E0005A152C981092D0031092CF0310925B15E9
:10F9F000809102018072809300010895DF92EF925E
:10FA0000FF920F931F93CF93DF93F82ED62EE72EFE
:10FA10008A0180914102882309F439C0E8EDF8E1B8
:10FA20008491EF012196882321F00E947D3DFE0103
:10FA3000F7CFED2DFE2D8491EF012196882321F043
:10FA40000E947D3DFE01F7CFE4E8F9E18491EF01EA
:10FA50002196882321F00E947D3DFE01F7CFF7FC1F
:10FA60000BC06F2DFF0C770B880B990B0E94044184
:10FA70008AE00E947D3D0BC0EFE7F9E18491EF0140
:10FA80002196882321F00E947D3DFE01F7CF8091D1
:10FA90006515811108C01092410281E080936515BF
:10FAA000C8010E94774EDF91CF911F910F91FF9077
:10FAB000EF90DF9084CFEF92FF920F931F93CF933D
:10FAC000DF93809144028F37A0F08F5790915A15A1
:10FAD0009093B015992311F02C9A01C02C98209185
:10FAE0005B152093AF1590910201222369F0909548
:10FAF0000BC09091B015891708F02C989091AF1514
:10FB0000891728F0909102019072909300018F5F05
:10FB1000809344029091AE1581E089278093AE15C1
:10FB20008091430285301CF4C1E0C80F01C0C0E0E1
:10FB3000823009F4B4C054F4882301F1813009F013
:10FB4000E3C088E080937B0085E4C0C0843009F482
:10FB5000C5C00CF4B7C0853009F0D6C09091AD1582
:10FB6000911102C08093AD158091AD1581508093A5
:10FB7000AD15882309F4C8C0C5E0C6C08091420213
:10FB80008F5F80311CF480934202BEC0109242020B
:10FB900080915715811113C08091A3159091A415E0
:10FBA0009093A01580939F158091A1159091A21517
:10FBB00090939E1580939D1581E0809357158AE060
:10FBC000E3EAF5E1DF011D928A95E9F71092A215AB
:10FBD0001092A11500919F151091A01511950195F6
:10FBE00011098091D5039091D603D1E0181619061A
:10FBF0002CF080915A15811101C0D0E08091630BE7
:10FC00009091640B9195819591098017910734F437
:10FC10004CE15BE16DE37BE180E0F0DE80913C0252
:10FC200090913D029195819591090817190744F427
:10FC3000DD2331F04FE45BE160E77BE180E0DEDE75
:10FC40008091CF039091D00311E0181619062CF083
:10FC500080915B15811101C010E0E0909D15F0903E
:10FC60009E158091610B9091620B8E159F0534F06B
:10FC70004CE25BE16DE37BE18FEFC0DE80913A0205
:10FC800090913B02E816F9060CF43EC01123E1F115
:10FC90004FE55BE160E77BE18FEFB0DE35C080913F
:10FCA0007A0086FD2EC08091780090917900209195
:10FCB000A3153091A415820F931F9093A4158093E0
:10FCC000A31522C088E080937B0086E480937C00AB
:10FCD00080917A00806480937A0016C080917A00C7
:10FCE00086FD11C080917800909179002091A11536
:10FCF0003091A215820F931F9093A2158093A115A6
:10FD000003C0C2E001C0C4E0C09343028091680B0D
:10FD100081110E94C1A880915815909159150097A2
:10FD2000A9F001979093591580935815892B71F478
:10FD300082E89BE19093FC0C8093FB0CDF91CF91C8
:10FD40001F910F91FF90EF900C94A93DDF91CF91FF
:10FD50001F910F91FF90EF9008952F923F924F9235
:10FD60005F926F927F928F929F92AF92BF92CF924B
:10FD7000DF92EF92FF920F931F93CF93DF9300D008
:10FD80001F92CDB7DEB75C017A8369834A01170100
:10FD900007FD07C0802F002E000C990B9C838B83DE
:10FDA00004C0E1E0F0E0FC83EB83F9014080518086
:10FDB000628073808B819C81880F991F880F991FA7
:10FDC0009C838B838B569A4E7C01A3019201FC018C
:10FDD00060817181828193810E9464C5882391F042
:10FDE000F701408251826282738211E020E030E0AC
:10FDF000A901C301B2010E94B4CB18160CF010E0A7
:10FE0000F5011083F50180818230D1F0833009F44F
:10FE10005EC0813009F07CC0EB81FC81EB56FA4E6C
:10FE20002081318142815381F4016081718182811D
:10FE300093810E9464C587FD6BC082E0F5018083D9
:10FE40008B819C818B569A4E9C838B83B60180E07C
:10FE500090E00E9468C59B01AC01EB81FC81608150
:10FE60007181828193810E948DC99B01AC01F40153
:10FE700060817181828193810E94B4CB87FD14C01F
:10FE80000E94F2B26B017C019101A8EEB3E00E94E6
:10FE90007EC9C60ED71EE81EF91EE981FA81C0820E
:10FEA000D182E282F38234C00E94F2B2E981FA8107
:10FEB000C080D180E280F380DC01CB018C199D09E8
:10FEC000AE09BF09B7FD24C083E0F50180830F3F71
:10FED00019F045EE5AE102C048EF5AE16CE07BE1CF
:10FEE000802F0F900F900F900F90DF91CF911F9167
:10FEF0000F91FF90EF90DF90CF90BF90AF909F90C9
:10FF00008F907F906F905F904F903F902F9076CD25
:10FF10000F900F900F900F90DF91CF911F910F9145
:10FF2000FF90EF90DF90CF90BF90AF909F908F9019
:10FF30007F906F905F904F903F902F9008954F92D9
:10FF40005F926F927F928F929F92AF92BF92CF9269
:10FF5000DF92EF92FF920F931F93CF93DF93CDB772
:10FF6000DEB760970FB6F894DEBF0FBECDBF8091AD
:10FF70005715811117C060960FB6F894DEBF0FBEFB
:10FF8000CDBFDF91CF911F910F91FF90EF90DF9048
:10FF9000CF90BF90AF909F908F907F906F905F9029
:10FFA0004F900895F4DB0E94F2B24B015C01609126
:10FFB000D5037091D603072E000C880B990B0E9475
:10FFC0006AC569837A838B839C8348E0C42ED12CD5
:10FFD0005CE3E52EF12C00E09E012F5F3F4F47EDE3
:10FFE00053E065E875E184E895E1B7DEC090D7039A
:10FFF000D090D803E090D903F090DA036091650BBC
:020000021000EC
:100000007091660B072E000C880B990B0E946AC535
:100010009B01AC01C701B6010E94B4CB18160CF0CD
:1000200009C160913E0270913F02072E000C880BBF
:10003000990B0E946AC59B01AC01C701B6010E94E1
:1000400064C587FFF7C00091D5031091D603B801AE
:10005000012E000C880B990B0E946AC5A70196011E
:100060000E948DC92B013C0120ED3CEC4CE45DE38A
:1000700060914E1570914F158091501590915115CA
:100080000E94C9C56D837E838F83988720917B15DD
:1000900030917C1540917D1550917E15C701B601B8
:1000A0000E948DC99B01AC016D817E818F819885F5
:1000B0000E94C9C56D837E838F83988723E333E3D2
:1000C00043E75FE36091771570917815809179151A
:1000D00090917A150E94C9C59B01AC016D817E810A
:1000E0008F8198850E948EC96D837E838F839887C8
:1000F00060937715709378158093791590937A159E
:10010000C0927B15D0927C15E0927D15F0927E1501
:1001100020E030E040E251E4C301B2010E94B4CBE0
:1001200018160CF431C220E030E040E251ECC3017B
:10013000B2010E9464C587FD2FC2012B09F42CC2B5
:100140008091761581112CC2209172153091731512
:10015000409174155091751529873A874B875C87B4
:1001600020914A1530914B1540914C1550914D15E9
:10017000C301B2010E94C9C56B017C01A3019201B8
:1001800069857A858B859C850E948EC969877A8767
:100190008B879C8760937215709373158093741589
:1001A000909375152091461530914715409148154B
:1001B000509149150E94C9C5A70196010E948EC998
:1001C0002D813E814F8158850E948DC96B017C0134
:1001D00020E030E04FE753E40E94B4CB20E030E071
:1001E000A90118160CF4E3C1C701B6010E9464C549
:1001F00087FD07C0C701B6010E94D2CA75956795F1
:100200001AC020E030E0A901C301B2010E9464C518
:1002100087FF10C0A301920169857A858B859C8533
:100220000E948DC960937215709373158093741535
:100230009093751560E060935A158091891590919F
:100240008A15A0918B15B0918C150097A105B10569
:1002500021F1A5019401281B390B4A0B5B0B57FDBB
:100260001CC060918D1570918E1580E090E00E9409
:1002700068C59B01AC016091D7037091D803809150
:10028000D9039091DA030E9464C587FF82C144ECD0
:1002900059E166ED79E180E0B1DB809152159091F2
:1002A0005315A0915415B0915515A5019401281B23
:1002B000390B4A0B5B0B57FD0FC088DAD501C4011F
:1002C0008C53964FAF4FBF4F809352159093531559
:1002D000A0935415B093551580918F15909190155A
:1002E000A0919115B09192150097A105B10511F15A
:1002F000881A990AAA0ABB0AB7FC1CC06091931518
:100300007091941580E090E00E9468C59B01AC015B
:100310006091D1037091D2038091D3039091D40363
:100320000E9464C587FF20C142EA59E165EB79E18B
:100330008FEF64DB6091CF037091D003072E000C28
:10034000880B990B0E946AC569837A838B839C838F
:1003500092E0C92ED12C24E1E22EF12C0FEF9E0168
:100360002F5F3F4F41ED53E06FE775E183E895E183
:10037000F4DCC090D103D090D203E090D303F0908E
:10038000D40320E030E040EA50E4C701B6010E9407
:10039000B4CB87FDE5C020E030E04CED52E4C7016E
:1003A000B6010E9464C518160CF4DAC06091CF0340
:1003B0007091D003072E000C880B990B0E946AC520
:1003C000A70196010E948DC94B015C012091421545
:1003D0003091431540914415509145150E94C9C56F
:1003E00069877A878B879C8720916E1530916F156E
:1003F0004091701550917115C501B4010E948EC9CC
:100400006D837E838F83988760936E1570936F15CD
:10041000809370159093711520913E1530913F1582
:1004200040914015509141150E94C9C56D877E8746
:100430008F87988B20ED3CEC4CE45DE360913A159E
:1004400070913B1580913C1590913D150E94C9C556
:100450002B013C0120916A1530916B1540916C1570
:1004600050916D15C701B6010E948DC99B01AC0169
:10047000C301B2010E94C9C52B013C0123E333E350
:1004800043E75FE360916615709167158091681589
:10049000909169150E94C9C59B01AC01C301B201CD
:1004A0000E948EC92B013C016093661570936715FD
:1004B0008093681590936915C0926A15D0926B1558
:1004C000E0926C15F0926D152D853E854F8558890B
:1004D00069857A858B859C850E948EC9A3019201CE
:1004E0000E948DC96B017C0120E030E04FE753E4AE
:1004F0000E94B4CB20E030E0A9011816C4F5C50174
:10050000B4010E94B4CB181684F4A50194016D8146
:100510007E818F8198850E948DC960936E1570933E
:100520006F1580937015909371156FE71AC020E0D6
:1005300030E0A901C501B4010E9464C587FF10C065
:10054000A50194016D817E818F8198850E948DC95E
:1005500060936E1570936F1580937015909371155D
:1005600060E060935B1507CD0E949B7AE3CEC701E4
:10057000B6010E9464C587FDDACFC701B6010E94AB
:10058000D2CA75956795EDCF81E0809376156FE7B8
:1005900052CE80E01CD881CE81E0809376154ACE81
:1005A0001092761519861A861B861C86D9CDC30132
:1005B000B2010E94B4CB181654F7A30192016985C9
:1005C0007A858B859C850E948DC960937215709386
:1005D000731580937415909375156FE72CCE9091D9
:1005E0006F00292F227091FF05C090916F009D7FB1
:1005F00090936F0034E0839FC0011124FC01EB5DF8
:10060000FA4E4081518162817381FC01E75EFA4EAE
:10061000408351836283738381E080931815222382
:1006200029F080916F00826080936F000895BC0173
:1006300020911615309117154091161550911715E8
:100640002417350711F09A01F7CF81E026173707F5
:1006500009F080E008952F923F924F925F926F923F
:100660007F928F929F92AF92BF92CF92DF92EF9242
:10067000FF920F931F93CF93DF93CDB7DEB76297AF
:100680000FB6F894DEBF0FBECDBF8091D90A982F68
:100690009270E92EE82FE470FE2EF82FF170DF2E15
:1006A00080FF04C0992311F0E11152C0EDEEF8E192
:1006B00084918F010F5F1F4F811103C0E2E5FEE1BE
:1006C00004C00E947D3DF801F3CF84918F010F5F3C
:1006D0001F4F882321F00E947D3DF801F6CFD110F5
:1006E0000CC0E0E5FEE184918F010F5F1F4F88236E
:1006F00021F00E947D3DF801F6CFE1100CC0EEE440
:10070000FEE184918F010F5F1F4F882321F00E942B
:100710007D3DF801F6CFF11003C0ECE4FEE103C02B
:10072000E4E4FEE10AC084918F010F5F1F4F88232C
:10073000B9F30E947D3DF801F6CF84918F010F5FE0
:100740001F4F882309F4C7C00E947D3DF801F5CFF3
:100750000BEA15E18DEB93E09A8B898BFE013196C4
:100760005F0194EF892E95E1992E1F01F8016591A3
:10077000759185919491E989FA89C190D190E19020
:10078000F190FA8BE98BA70196010E948DC92B018C
:100790003C01F101608371838283938320E030E028
:1007A00040EA51EC0E94B4CB87FD0AC020E030E063
:1007B00040EA51E4C301B2010E9464C518162CF44A
:1007C000F401849118160CF47CC0F101C190D19011
:1007D000E190F1901F0120E030E040EA51ECC701C8
:1007E000B6010E94B4CB87FD0AC020E030E040EAA9
:1007F00051E4C701B6010E9464C5181614F5E8ED6E
:10080000F8E184918F010F5F1F4F811103C0E8E56C
:10081000FEE104C00E947D3DF801F3CF84918F0179
:100820000F5F1F4F882321F00E947D3DF801F6CF16
:1008300088E290E0988B8F8788EC90E09E878D8788
:1008400038C00C5F1F4FFFEF8F1A9F0A85E1073BEF
:10085000180709F08BCF89E6E82E8BE0F82E10E020
:10086000F50181919191A191B1915F01F70181937E
:100870009193A193B1937F01812F0E94CE9A1F5F24
:10088000133071F70E94459583E992E0988B8F872A
:1008900004E610E01E870D87BE01615F7F4FCE0129
:1008A0000D960E9410B18AEB92E0988B8F871E877D
:1008B0000D87BE01615F7F4FCE010D960E9410B182
:1008C0000AC0F7FAF094F7F8F094F101C082D182EF
:1008D000E282F3827ACF62960FB6F894DEBF0FBE43
:1008E000CDBFDF91CF911F910F91FF90EF90DF90DF
:1008F000CF90BF90AF909F908F907F906F905F90C0
:100900004F903F902F900895CF92DF92EF92FF92F9
:100910000F931F93CF93DF9388E50E94183DD82E45
:1009200089E40E94183DC82E882319F00E94B13C2A
:100930001CC0DD20C1F00E94E13C20E030E040E23C
:1009400051E40E948DC920E030E04CEB51E40E945C
:100950008EC921E43CE44EEA5CE30E94C9C50E94D2
:10096000D2CA653010F01FEF01C0162F89E50E9432
:10097000183D082F8AE40E94183DC82F882319F0DB
:100980000E94B13C1CC00023C1F00E94E13C20E069
:1009900030E040E251E40E948DC920E030E04CEBB1
:1009A00051E40E948EC921E43CE44EEA5CE30E94DB
:1009B000C9C50E94D2CA653010F0DFEF01C0D62F42
:1009C0008AE50E94183DE82E811105C081E50E944C
:1009D000183DF82E01C0F12CC11001C0C0E02C2F31
:1009E00030E0D11001C000E0200F311D2130310571
:1009F00021F4E1101AC0F11018C0E8EDF8E184917B
:100A0000EF012196811103C0E4E2FEE104C00E94DF
:100A10007D3DFE01F4CF8491EF012196882309F4F6
:100A200055C00E947D3DFE01F6CF17FD02C0D7FFE5
:100A300017C0E8EDF8E18491EF012196811103C020
:100A4000E5E0FEE104C00E947D3DFE01F4CF84910B
:100A5000EF0121968823D1F10E947D3DFE01F7CF61
:100A60000E94E13C9B01AC01012F110F110BAD2F36
:100A7000DD0FBB0BFF2099F085E0809FF001819F87
:100A8000F00D1124EA0FFB1FEE0FFF1FEE0FFF1FEB
:100A9000ED53FA4E608171818281938103C060E0E1
:100AA00070E0CB01E5E0E09FE001E19FD00D112473
:100AB000CA0FDB1FCC0FDD1FCC0FDD1FCD53DA4E6D
:100AC0000E948EC9688379838A839B83DF91CF914B
:100AD0001F910F91FF90EF90DF90CF9008952F928C
:100AE0003F924F925F926F927F928F929F92AF92BE
:100AF000BF92CF92DF92EF92FF920F931F93CF930B
:100B0000DF93CDB7DEB761970FB6F894DEBF0FBEA7
:100B1000CDBF83E50E94183D882349F00E94D23C56
:100B2000182F811106C080E00E946A9902C01091BE
:100B30003B168091BD039091BE03A091BF03B0917D
:100B4000C00389839A83AB83BC838091C103909156
:100B5000C203A091C303B091C4038D839E83AF836E
:100B6000B8878091C5039091C603A091C703B09147
:100B7000C80389879A87AB87BC870E943D998823E1
:100B800009F49AC083E40E94183D882309F494C0B4
:100B90000E94E13C1B012C0105E0612C712C38EC1A
:100BA000388B82EC898BA12CB12C98EC9E87E2E4E7
:100BB000EF87015080F125E02D87209F400111240F
:100BC0003D8531503D873F3FA1F3F401E30FF11D17
:100BD000EE0FFF1FEE0FFF1FED53FA4EC080D180C6
:100BE000E280F3809601A701B5018E859F850E9462
:100BF000B4CB18161CF45601EE86FF869601A701A9
:100C0000B301888999890E9464C587FFD9CF3601CD
:100C1000E88AF98AD5CF930148895989B5018E852B
:100C20009F850E948EC920E030E040E05FE30E9493
:100C3000C9C5A20191010E948EC92B013C012DEB77
:100C400037E346E855EB0E94B4CB87FD0AC02DEB95
:100C500037E346E855E3C301B2010E9464C51816A4
:100C60005CF580E00E946A9935E0D32E45E0C42E01
:100C7000DA949FEFD91601F105E0CD9C50011124C3
:100C80000150B0F37501E00EF11CC701880F991FE8
:100C9000880F991FFC01ED53FA4E7F01A3019201C9
:100CA00060817181828193810E948DC9F701608387
:100CB000718382839383E4CF86E50E94183D882365
:100CC00099F00E943D99882379F0EFEEFDE184913F
:100CD0007F012FEFE21AF20A882321F00E947D3D66
:100CE000F701F5CF0E94FEA78AE50E94183D8823F0
:100CF00021F00E94E13C0E947BB0812F0E946A9902
:100D0000111103C0EDEEF8E11CC080913B1681117A
:100D1000F9CFE8EDF8E184918F010F5F1F4F882331
:100D200021F00E947D3DF801F6CFE0EDFDE18491D8
:100D30008F010F5F1F4F882329F30E947D3DF8012B
:100D4000F6CF84918F010F5F1F4F882321F00E94FF
:100D50007D3DF801F6CF80913B16811103C06FE015
:100D600073E002C06BE073E082EC9DE10E94074CEF
:100D70008AE00E947D3DEDEEF8E184918F010F5FE6
:100D80001F4F882321F00E947D3DF801F6CFE5EB4F
:100D9000FDE184918F010F5F1F4F882321F00E9496
:100DA0007D3DF801F6CFC0903C16D0903D16E09006
:100DB0003E16F0903F1620E030E0A901C701B601D1
:100DC0000E94B4CB18164CF442E0C701B6010E9451
:100DD0001E418AE00E947D3D0CC0E0EBFDE1849164
:100DE0008F010F5F1F4F882321F00E947D3DF80186
:100DF000F6CF4CE050E06DEB73E0CE0101960E941F
:100E0000C6CC892BD1F061960FB6F894DEBF0FBE29
:100E1000CDBFDF91CF911F910F91FF90EF90DF90A9
:100E2000CF90BF90AF909F908F907F906F905F908A
:100E30004F903F902F900C94459561960FB6F89483
:100E4000DEBF0FBECDBFDF91CF911F910F91FF90FD
:100E5000EF90DF90CF90BF90AF909F908F907F905A
:100E60006F905F904F903F902F90089580916F000A
:100E7000982F927081FF05C080916F008D7F8093C5
:100E80006F0080910C0F80930B0F80930A0F80935B
:100E9000090F84E68093080F28EE33E0309359154C
:100EA00020935815992329F080916F0082608093D8
:100EB0006F0081E0809318150E94DD660E945A56EB
:100EC00080913B16882321F082EB9AE00E94224C0D
:100ED0008CE0E2EBFAE0ADEBB3E001900D928A9585
:100EE000E1F70C946A3C2F923F924F925F926F927F
:100EF0007F928F929F92AF92BF92CF92DF92EF92AA
:100F0000FF920F931F93CF93DF93CDB7DEB7C554F6
:100F1000D1090FB6F894DEBF0FBECDBF85E40E94A5
:100F2000613D882321F00E94B13C7B0102C0E12C8D
:100F3000F12C83E40E94613D882321F00E94B13CA2
:100F40006AA302C005E00AA385E50E94613D8823EB
:100F500019F00E94D23C03C085E50E94183D8CA781
:100F6000F7FC07C0812C912C16E1A12E13E4B12EC1
:100F700006C0812C912CBCE8AB2EB2E4BB2E83E5DD
:100F80000E94613D882321F00E94E13C4B015C01FD
:100F9000E114F10411F410925C151092BF0AED8275
:100FA0000E94F2B22B013C011D8117FD03C004E138
:100FB00010E002C00CE310E0D301C2018C53964F45
:100FC000AF4FBF4F8093521590935315A093541574
:100FD000B093551561E06E0D623080F0E2E7FDE1FF
:100FE00084918F010F5F1F4F1A830983882309F4AF
:100FF0003AC30E947D3DE981FA81F2CFECE9FDE13F
:1010000084917F012FEFE21AF20A882321F00E94D7
:101010007D3DF701F5CF0E94DF7C3D8137FF04C0A5
:101020008FE780935B1508C04D81E42F440FFF0BC1
:10103000E65AFA4E8FE78083C501B4010E94D2CAF6
:10104000072E000C880B990B0E946AC56A877B8764
:101050008C879D879801A8EEB3E00E947EC96DA79A
:101060007EA78FA798ABDC01CB01840D951DA61D33
:10107000B71D8AAF9BAFACAFBDAF81E0809340029C
:101080000D810F3F39F40CED1CE11FAF0EAF06EAE6
:101090001CE106C00AEC1CE11FAF0EAF03E91CE126
:1010A00022961FAF0EAF22974CA25DA26EA27FA226
:1010B00049AA5AAA6BAA7CAA1DAA1EAA1FAA18AEE0
:1010C00019AE188E10E4198F0CE10A8F16E41B8FED
:1010D0001C8E1D8E1E8E1F8E1C8A1D8A1E8A1F8AC4
:1010E000188A198A1A8A1B8A19821A821B821C8200
:1010F0002FE730E040E050E02E833F834887598758
:10110000FFE7CF2ED12CE12CF12C18A619A61AA698
:101110001BA611E01F861E8625961FAE2597212C43
:10112000312C26961FAE26970D81802F000F990B2C
:101130009C01265A3A4E24963FAF2EAF2497880F33
:10114000991F880F991FAC0149525C4F59A348A3BE
:101150008AA1082E000C990B9BA38AA380914002C0
:10116000882309F47EC20E94F2B24B015C01809197
:101170005715882309F4D4C00E94C77B0D8107FD51
:101180000CC0A8A1B9A1BC912596BFAF2597E8A135
:10119000F9A12180328003810BC00091D1032596F3
:1011A0000FAF25972090D2033090D3030091D40342
:1011B00026960FAF269725962FAD2597322D432DD6
:1011C00026965FAD26976C8D7D8D8E8D9F8D0E94AE
:1011D00064C587FF0AC025960FAD25970C8F2D8E0D
:1011E0003E8E26960FAD26970F8F288D398D4A8D0E
:1011F0005B8D25966FAD2597722D832D26969FAD1D
:1012000026970E9464C587FF0AC025960FAD2597D3
:10121000088F298E3A8E26960FAD26970B8F8091D8
:10122000521590915315A0915415B0915515A501E3
:101230009401281B390B4A0B5B0B57FD10C00E9411
:10124000E67BD501C4018C53964FAF4FBF4F8093BF
:10125000521590935315A0935415B0935515259698
:101260002FAD2597322D432D26965FAD26976A85A3
:101270007B858C859D851123E9F10E9464C587FFDC
:101280004FC0B501A4014419550966097709DB016E
:10129000CA0188589341A109B109B7FD41C0D701DE
:1012A000C6010E811F8128853985801B910BA20BF9
:1012B000B30B1D81B595A7959795879517FF03C02B
:1012C00080935B1505C02496EEADFFAD2497808317
:1012D00048A759A76AA77BA70A850C8F1B851D8F76
:1012E0000C850E8F1D851F8F8CA29DA2AEA2BFA262
:1012F00010E016C00E94B4CB181694F4D501C401B6
:101300002CA13DA14EA15FA1821B930BA40BB50B99
:10131000AC01BD01485853416109710977FFC0C153
:1013200020E030E040EA51E46A857B858C859D852C
:101330000E948EC925962FAD2597322D432D2696D6
:101340005FAD26970E9464C587FF10C0EEEFFCE1F9
:1013500084918F010F5F1F4F1A830983882309F43B
:1013600080C10E947D3DE981FA81F2CFD501C4019F
:1013700029A93AA94BA95CA9821B930BA40BB50B15
:10138000B7FD8BC00E94E1798AE00E947D3DD501C6
:10139000C4018053984FAF4FBF4F89AB9AABABABF3
:1013A000BCAB0DA9011158C02EA93FA948AD59AD3C
:1013B00025966FAD2597722D832D26969FAD269786
:1013C0000E94B4CB1816BCF520E030E040E050E4B9
:1013D00025966FAD2597722D832D26969FAD269766
:1013E0000E948EC96EAB7FAB88AF99AF2DA53EA58D
:1013F0004FA558A9280D391D4A1D5B1D2AAF3BAFCB
:101400004CAF5DAF20E030E040EC50E46A857B8576
:101410008C859D850E948DC925962FAD2597322DEF
:10142000432D26965FAD26970E9464C5881F8827A6
:10143000881F8DAB32C0D501C4012AAD3BAD4CAD88
:101440005DAD821B930BA40BB50BB7FD26C04EAD53
:101450005FAD6FEE7CE11EC020E030E040EA51E479
:101460006A857B858C859D850E948DC99B01AC0119
:1014700025966FAD2597722D832D26969FAD2697C5
:101480000E9464C587FF09C022964EAD5FAD2297CA
:101490006AEB7CE18D810E94FE7CD501C401880F3E
:1014A000991FAA1FBB1F2CA13DA14EA15FA1821BAA
:1014B000930BA40BB50B84199509A609B7098138BC
:1014C0009F44A241B10580F0E5E7FCE184918F01E2
:1014D0000F5F1F4F1A830983882309F4C2C00E943B
:1014E0007D3DE981FA81F2CF2AA13BA14E855F853E
:1014F000241735070CF032CEE8E1FCE184918F012E
:101500000F5F1F4F1F830E83882329F00E947D3DAC
:10151000EE81FF81F3CF1D8117FD03C00EE013E0C4
:1015200002C000E913E01F830E836E817F8187E094
:101530009CE10E94074C49815A816B817C8183E048
:101540009CE10E94D14B8AE00E947D3D6E817F81AB
:1015500082EF9BE10E94074C488959896A897B89FF
:101560008EEE9BE10E94D14B8AE00E947D3D6E8110
:101570007F818DED9BE10E94074C4C895D896E89CE
:101580007F8989ED9BE10E94D14B8AE00E947D3DDD
:101590001CA5112309F467C00D8107FF31C0298103
:1015A0003A814B815C8120934215309343154093DF
:1015B0004415509345152CEA35EC47E25EE3688903
:1015C00079898A899B890E94C9C560933E15709369
:1015D0003F1580934015909341152CEA35EC47E276
:1015E0005EE36C897D898E899F890E946ACA6093B7
:1015F0003A1570933B1580933C1590933D1533C07D
:1016000089819A81AB81BC8180934A1590934B1557
:10161000A0934C15B0934D152CEA35EC47E25EE3F0
:10162000688979898A899B890E94C9C56093461512
:101630007093471580934815909349152CEA35EC23
:1016400047E25EE36C897D898E899F890E946ACA20
:1016500060934E1570934F158093501590935115CC
:1016600002C00E94DF7C81E08093BF0ACB5BDF4F2A
:101670000FB6F894DEBF0FBECDBFDF91CF911F91A3
:101680000F91FF90EF90DF90CF90BF90AF909F9021
:101690008F907F906F905F904F903F902F90089524
:1016A0000E851F85012B09F42DC148A459A46AA4F5
:1016B0007BA4480E591E6A1E7B1E28A539A54AA583
:1016C0005BA5281B390B4A0B5B0B6E817F818885DC
:1016D00099850E9443C9A30192010E948ACCDA0134
:1016E000C9018C0D9D1DAE1DBF1D84319105A10545
:1016F000B105FCF06C017D018C3E9105A105B105A1
:101700002CF05BEEC52ED12CE12CF12C20E8C2167A
:10171000D104E104F104DCF08EEF90E0A0E0B0E051
:101720008C199D09AE09BF098E839F83A887B9874D
:1017300012C044E1C42ED12CE12CF12C04E110E0C4
:1017400020E030E00E831F832887398704C0CE82D3
:10175000DF82E886F986EAE6FDE184918F010F5F7A
:101760001F4F882321F00E947D3DF801F6CFC7016D
:10177000B6010E940441E5E6FDE184918F010F5F0F
:101780001F4F882321F00E947D3DF801F6CF6E8126
:101790007F81888599850E940441488D598D6A8D85
:1017A0007B8D8EE59DE10E94D14B4C8D5D8D6E8DC4
:1017B0007F8D87E59DE10E94D14B0E851F8503300B
:1017C00011050CF49FC06E817F81888599850E94E8
:1017D0006AC520E030E040E850E40E94C9C5698352
:1017E0007A838B839C83288D398D4A8D5B8D6C8D9C
:1017F0007D8D8E8D9F8D0E948DC92BED3FE049E43C
:1018000050E40E94C9C520E030E040E05FE30E9460
:10181000C9C59B01AC0169817A818B819C810E9441
:101820006ACA69837A838B839C83C301B2010E9455
:101830006AC52FE632E143E85AE30E94C9C52B018D
:101840003C0149815A816B817C8181E59DE10E9447
:10185000D14BB301A2018BE49DE10E94D14B2AE957
:1018600039E949E15FE369817A818B819C810E943A
:10187000C9C569837A838B839C839B01AC010E94D9
:101880008EC9A30192010E946ACA688B798B8A8BE8
:101890009B8B29813A814B815C81C301B2010E94FB
:1018A000C9C520E030E040E05EE30E94C9C56C8B12
:1018B0007D8B8E8B9F8BEBE3FDE184918F010F5F1E
:1018C0001F4F882321F00E947D3DF801F6CF49810A
:1018D0005A816B817C8185E39DE10E94D14B4889CF
:1018E00059896A897B898FE29DE10E94D14B4C899D
:1018F0005D896E897F8989E29DE10E94D14B8AE0F2
:101900000E947D3D8E819F81A885B9858C0D9D1D8E
:10191000AE1DBF1D1D81B595A7959795879517FF9E
:1019200003C080935B1505C02496EEADFFAD2497F0
:1019300080830E851F850F5F1F4F1F870E871A85B7
:10194000188F0B85098F1C851A8F0D850B8F24012D
:10195000350111E0E5CCCF93DF93EDEEF8E1849112
:10196000EF012196882321F00E947D3DFE01F7CFF3
:1019700083E50E94183D882321F00E94D23C809389
:101980002102E9ECFBE18491EF012196882321F00B
:101990000E947D3DFE01F7CF80912102811103C09D
:1019A000E5ECFBE102C0E1ECFBE18491EF01219663
:1019B000882321F00E947D3DFE01F7CFE9EBFBE19A
:1019C0008491EF012196882321F00E947D3DFE0144
:1019D000F7CF2091A0033091A1034091A203509131
:1019E000A3036091EA0A7091EB0A8091EC0A90914E
:1019F000ED0A0E948EC9AB01BC0187EB9BE10E94FE
:101A0000D14B2091A4033091A5034091A60350919E
:101A1000A7036091EE0A7091EF0A8091F00A90910D
:101A2000F10A0E948EC9AB01BC0184EB9BE10E94CC
:101A3000D14B2091A8033091A9034091AA03509162
:101A4000AB036091F20A7091F30A8091F40A9091CD
:101A5000F50A0E948EC9AB01BC0181EB9BE10E949B
:101A6000D14BE9EAFBE18491EF012196882321F033
:101A70000E947D3DFE01F7CF2091A0033091A1038C
:101A80004091A2035091A303609127027091280214
:101A90008091290290912A020E948EC9AB01BC015B
:101AA00087EA9BE10E94D14B2091A4033091A503CA
:101AB0004091A6035091A70360912B0270912C02D4
:101AC00080912D0290912E020E948EC9AB01BC0123
:101AD00084EA9BE10E94D14B2091A8033091A90395
:101AE0004091AA035091AB0360912F027091300294
:101AF00080913102909132020E948EC9AB01BC01EB
:101B000081EA9BE10E94D14B8AE0DF91CF910C9456
:101B10007D3DFF920F931F93CF93DF93F82E092FF4
:101B2000162FECE9FBE18491EF012196882321F047
:101B30000E947D3DFE01F7CFEF2DF02F8491EF0144
:101B40002196882321F00E947D3DFE01F7CFEAE92E
:101B5000FBE18491EF012196882321F00E947D3DD5
:101B6000FE01F7CF612F70E080E090E00E94044119
:101B70008AE0DF91CF911F910F91FF900C947D3DF2
:101B80000F931F93CF93DF93EB010E94F2B28B016F
:101B90000E94824C8F3F49F00E94F2B2601B710B91
:101BA0006C177D07A8F380E001C081E0DF91CF9141
:101BB0001F910F9108958F929F92AF92BF92CF92F3
:101BC000DF92EF92FF920F931F93CF93DF93EC017D
:101BD0008B81811102C080E078C009891A892B8924
:101BE0003C890417150726073707A8F36A017B010C
:101BF000823029F4C886D986EA86FB860DC0C114D6
:101C0000D104E104F10451F4188619861A861B8662
